:100000000040002049710000897100008B710000E0
:1000100000000000000000000000000000000000E0
:100020000000000000000000000000008D710000D2
:1000300000000000000000008F71000091710000BE
:1000400093710000B5520000C57500009371000067
:100050009371000000000000937100009371000094
:100060009371000095780000BD310000937100008D
:100070009371000093710000937100009371000070
:10008000937100002D7A00009371000093710000BD
:100090009371000093710000937100009371000050
:1000A0009371000093710000000000000000000048
:1000B0000000000000000000000000000000000040
:1000C00010B5064C2378002B07D1054B002B02D02E
:1000D000044800E000BF0123237010BD640200202B
:1000E0000000000068E40000044B10B5002B03D0B2
:1000F0000349044800E000BF10BDC04600000000F6
:100100006802002068E40000164B002B00D1144B5D
:100110009D46402292029A1A924600218B460F4633
:100120001348144A121A0BF029FA0F4B002B00D077
:1001300098470E4B002B00D0984700200021040068
:100140000D000D48002802D00C4800E000BF0BF065
:10015000D5F92000290007F053FA0BF0A9F9C046A1
:100160000000080000400020000000000000000027
:1001700064020020BC2F00200000000000000000EE
:1001800002000120104011D1042A0ED91368180969
:1001900080B2002809D001388000031D11180979A8
:1001A000002902D001309842F8D170470020FCE7C6
:1001B0000378002B03D05AB2002A01DB01307047CC
:1001C0003F229343C03B59424B41C01803789343AD
:1001D000802BF4D10130F9E710B500240378002B0F
:1001E00001D1200010BDFFF7E3FF0134F6E770B541
:1001F000002204000D00411C092003F009FB002827
:1002000006D001236200134343600023A34200DBB6
:1002100070BD9A00A958821891600133F6E770B555
:10022000012803DC1C2001F047F870BD01230D6894
:1002300011201D42F7D04868184206D1042804D97D
:100240000F2302681340042B01D00E20EBE703F0CC
:100250003DF96D100400002D03DDFFF7BDFFA8423E
:1002600006DA1220DFE72000FFF7A2FF0400013DBD
:10027000012DF8D120787F2809DDDF280BDCF82359
:100280003F22DB00800118406378134018430123AC
:1002900040001843C9E7EF280BDCFC226378120109
:1002A0009B0113403F220007000C0343A07810403D
:1002B000ECE7F72812DCFC22637892021B03134060
:1002C000E0228004520310403F221843E378134099
:1002D000FC220343A07812018001E8E7012040429C
:1002E000D5E7F8B54D680F00EB0706D4042D04D907
:1002F0000F232E683340092B03D00B2000F0DCFFC6
:10030000F8BD6B683609B6B25C10731EA3420FD8F5
:100310000321200008F0EEFF6421642803DC0100C3
:10032000032800DA03212800891903F0A3FA050045
:100330002B6800201B099BB2013B9C42E0D23A682B
:10034000A31C9B005A510123013464001C436C60C0
:10035000D6E7F0B585B0012803DC1C2000F0ACFF27
:100360002CE001274B683A000093022806D08B68E6
:100370003B4203D05F10002F00DC17000124009BDC
:10038000234200D0B2E0042B00D8AFE01B680D6818
:100390000F2619003140042925D1254205D1042D0D
:1003A00003D92B681E40042E01D00E20D6E70098FA
:1003B000FFF7E6FEB84203DA0120404205B0F0BD87
:1003C000009803F083F80600280003F07FF801008E
:1003D000781E30180BF088FC0028EDD0801B01300F
:1003E00040002043EAE709293DD1009B5B685B1090
:1003F00001939F42E0DC25422CD1042D2AD92B68A1
:100400003340042B26D1280003F060F803960290B5
:100410007E1C009AB300D058854201D17800E0E7F5
:1004200020420ED104280CD90368039A1340042BF0
:1004300007D103F04BF8010002980BF01FFC0028D5
:10044000ECD0019B37009E42E2DDB5E71F00019B27
:100450009F42B1DC7B1C00999A008A58AA42F5D1D0
:1004600078000124BDE7032940D11A0992B25B0F3D
:1004700092000B40D31A01939F429DDC254229D163
:10048000042D27D92A681640032E19D1100980B2ED
:10049000520F800032402C1D801A019B26181B1A17
:1004A0000193009B781E0433019A904200DD83E79C
:1004B00022001918B2420FD316D101304000D0E704
:1004C000042E07D1280003F001F804002800FFF7EC
:1004D00057FEE2E70F2041E70D78AC461578AC45B2
:1004E00002D101310132E5E70130DDE7212035E7B6
:1004F00010B502F0CFFF43000120184310BD0000EB
:10050000C30711D404280FD90F2302681340032B0B
:100510000AD119400133591AC0234907DB05194094
:10052000024B1A40114301607047C046FFFFFF9F16
:10053000F7B507000E001C20012F06DD4C680123D3
:1005400022001A40009203D10D2000F0B5FE53E0C6
:10055000022F02D08A681A42F6D0012335681D4264
:1005600000D0A9E0042D00D8A6E01C41002C00DC3E
:100570001C000F2029680840092828D16B685B10EF
:100580000093022F05D0B368009A5B109A4200DDF9
:100590000093009B01221D1B0135EB43DB171D401F
:1005A000691C092003F034F9071E09D001236D00EE
:1005B0001D4303003268083345600099A14201DA07
:1005C0003800FEBD0134A100515802C3F5E70428EC
:1005D00045D1280002F07AFFFFF7FEFD0190022FBF
:1005E00004D0B3685B10984200DD0193019BA342E5
:1005F00004DA002003F07EF90700E1E7280002F0AA
:1006000065FF0700009BA34221DB2800009702F052
:100610005DFF05003800FFF7CBFD019B01340700AB
:10062000A342F7DA009BC41A200003F063F9071E07
:10063000C6D002F04BFF0190306802F047FF220065
:10064000009B591B411801980AF07CFFB8E738005D
:10065000FFF7AEFD009B070001330093D2E70328AC
:100660002AD10B099BB2490F9B000140591A022F56
:1006700004D0B2685210914200DD1100A14205DAA7
:1006800000220320110003F0C3F8B5E703200E1B7E
:10069000331DD9170140C9188910002203F0B8F89A
:1006A000071E00D18CE7013631000334FFF728FF25
:1006B000381D29193200C7E7212046E7F8B5002880
:1006C00005DC1C2000F0F8FD05002800F8BD01261F
:1006D0000C6826400FD06410E343DB171C40E11C7C
:1006E00089100022032003F093F8051EEDD02100AD
:1006F000FFF706FFE9E7042C01D80025E5E70F2303
:1007000022681340042B1BD12000FFF739FDC31CC6
:1007100007000320D9170140C9188910320003F0DF
:1007200077F8051ED1D03900FFF7EAFE200002F06D
:10073000CDFE2B1D01003A0018000AF003FFC4E7AC
:10074000092BDAD10320636832005F10FB1CD91734
:100750000140C918891003F05BF8051ECDD039009F
:10076000FFF7CEFEFF20BE42AFDA0122B300E3184E
:100770009B68134208D01341FF2B00DD0300D943CF
:10078000C917AA190B4013710136ECE710B57F2980
:1007900002DC0170013010BD1A4B99420CDC402381
:1007A0008A115B42134303703F230B40802149426F
:1007B000194341700230EEE7134B994210DC2023BD
:1007C0000A135B4213433F24802203708B11524271
:1007D0002340214013430A43437082700330DAE719
:1007E0000A4B9942D7DCF0230370603B4370113B06
:1007F0008A11FF3B1A4382703F2211401943C17096
:100800000430C8E7FF070000FFFF0000FF0F0100F2
:10081000F0B50D0085B0002803DC1C2000F04CFD75
:100820000DE009680122080010400AD002AC114115
:100830002000FFF7ABFF011B200003F067F8040066
:100840001AE004293FD90F230C682340092B3AD121
:100850004B685B10019303239C46019B9A420EDD7B
:1008600003F048F8041E07D02E68012502F02EFE82
:100870002F00019B9D421DDD200005B0F0BD01321F
:100880009300CC580123234001D10D20C6E764100A
:100890007F2C0DDD0D4E0223B44209DD0C4E634664
:1008A000B44205DD00270B4EE30FA6427B419B00BF
:1008B000C018D2E70135AB00F1583942E5D04910F4
:1008C000FFF764FFD5E72120A8E7C046FF07000037
:1008D000FFFF0000FF0F010010B5040001200840D9
:1008E00010D104290DD90F230A681340042B08D115
:1008F000080002F0EBFD010020000BF0BFF94342BD
:10090000584110BD0020FCE7F7B50F00012803DCBB
:100910001C2000F0D1FCFEBD01264D682E4006D102
:10092000042D04D90F222B681A40092A01D00B206C
:10093000EFE76A681B099BB25410A34200D85C1E03
:1009400039681E48FFF7C8FF01230190002813D122
:1009500039681B48FFF7C0FF002811D0002C0DD0CC
:100960000123621C013C9C409200535123436B6065
:1009700004E00136B200AB50B442FADA0020CAE714
:100980003B680D20DA07C4D55B10002B11DD9C42BB
:100990000FDB9B00A200291DEB1889180433994234
:1009A00009D10123013C9C40AA181C4353606C6090
:1009B000E4E71220ADE758681860EFE70FCC0000BD
:1009C00013CC0000002310B50C000B70C30705D535
:1009D0000D49421020000BF015F908E00B490028E2
:1009E00002D0042804D10A4920000BF02BF910BDD5
:1009F0000428FCD90F2302681340042BF7D102F01E
:100A000065FD04490200E5E70CD6000018CC0000A3
:100A10001ECC000023CC0000F0B593B0060002917C
:100A20001C20012E1DDD029B01251B681C002C4093
:100A300000D0ADE0042B00D8E6E01A680F231A407E
:100A4000092A4AD10394039A029992008A581700FE
:100A50002F4005D1042A03D910681840092806D070
:100A6000222000F029FC0190019813B0F0BD5268DB
:100A70005210A418039A013203929642E3D1611CEA
:100A8000012202F0C5FE0190002802D1002301934B
:100A9000EAE7019B6400190025435D600831029A72
:100AA000BB00D05802684368120992B25B109A42A8
:100AB00000D8531E0022934209DCDA43D2171340B8
:100AC0009B00C918039B01379F42E8DBCCE79400E9
:100AD0000519AD6801320D51EDE72700032A59D100
:100AE0000193029ABB00D3582B42B9D1042BB7D93A
:100AF000186801990140032939D1020992B2430FC4
:100B000092000B40D31A1C190137BE42E9D10320D1
:100B1000E31CD9170140C9188910002202F078FEA1
:100B200001900028B2D000252100FFF7E9FC019BCD
:100B30001E1D029AAB00D45801231C421FD1042C65
:100B40001DD90F2123681940032918D1180980B233
:100B50005B0F80000B40C01A0023834213DBC343AA
:100B6000DB17184001353618BD42E2DB7CE704296B
:100B700000D075E71800FFF703FB2418C4E7200036
:100B8000FFF7FEFAE8E7E2181279F2540133E4E7DE
:100B900000273C000F25029ABB00D35801221342C4
:100BA00034D1042B32D9186801002940042935D1E9
:100BB0001800FFF7E5FA24180137BE42EBD12000F8
:100BC00002F098FE0190002800D15FE7029FB60076
:100BD000BB19041D029301233D681D4229D1042D38
:100BE00027D90F262B681E40042E37D12800FFF787
:100BF000C7FA0600280002F069FC0100200032005C
:100C00000AF0A0FCA41922E02700C3E7180005A9F8
:100C1000FFF7D8FE05A80BF03BF8CCE7032900D07E
:100C20001EE7020992B2430F92000B40D31A1C191F
:100C3000C2E705A92800FFF7C5FE05A80BF028F8B4
:100C400005A90500020020000AF07CFC6419029B43
:100C50000437BB42BFD10023237005E7032EF6D132
:100C60001A0992B25B0F92001E40961B291DC5E720
:100C7000F0B50D0095B0002806DC1C2000F01CFB30
:100C80000400200015B0F0BD0C68012123000B40CA
:100C9000009306D1042C04D922680F331A40092A84
:100CA00001D00B20EAE7626852100392002A03DCAD
:100CB000009802F01FFEE3E73F4A019201280BD0A3
:100CC0006868084208D1042806D902681340042B3A
:100CD00002D102F0FBFB019001980AF0D9FF060057
:100CE0000F27039B0834013B04935E43039B029050
:100CF0009B001B19059301232068184251D1042839
:100D00004FD903683B40042B52D1FFF739FA059BBA
:100D100004343618A342EED1300002F0EBFD041E7D
:100D2000AFD02B680593029B002B03D0686802F0BC
:100D3000CDFB0190200002F0C9FB0500009B059A45
:100D40009B00D3189F68380002F0C0FB0123060007
:100D50001F4201D1042F04D807A93800FFF732FE43
:100D600007AE30000AF094FF0700020031002800AF
:100D70000AF0E8FB029BED19002B0AD0049B009AB5
:100D8000934206DD2800029A01990AF0DBFB029BE0
:100D9000ED18009B01330093009A039B9342CDD141
:100DA0006FE707A9FFF70EFE07A80AF071FFAEE78D
:100DB00002F08CFBF9E7C046B0D0000010B500246B
:100DC000A04207DD0B6801341C4003D05C10E343F4
:100DD000DB171C40611C0122092002F019FD0028CC
:100DE00003D0012364001C43446010BD0A6870B541
:100DF00010000125284034D1042A32D90F24136869
:100E000049681C40092C17D154681B099BB22C411E
:100E1000A34200D85C1E844205DC022001339842C4
:100E200006DB00200FE085005519A9600130F2E7CC
:100E3000840011510130F2E7032C12D1294203D171
:100E4000132000F039FA70BD4910FF29F8D81B09AA
:100E50009BB204329B00D3189342E2D91170013245
:100E6000FAE70B2000F028FADBE700000123F7B5D2
:100E700000254E680F0033400093AB420ED11D0099
:100E8000042E0BD90F2233681A40092A10D1726838
:100E90001B099BB25510AB4200D85D1E3968CB07C9
:100EA00017D54C10002C01DDA5421DDA122032E0CE
:100EB000042A04D13000FFF763F90500EEE7009D36
:100EC000032AEBD11D09ADB25B0FAD001340ED1A43
:100ED000E4E72E48FFF700FD002814D00AF02EFEAC
:100EE000290008F0EDFA4C1C009B002B4CD1042E7D
:100EF0004AD932680F331340092B10D10134A400B2
:100F0000A4592000FEBD39682148FFF7E5FC2C00FC
:100F10000028E9D1113000F0CFF90400F1E7042BEB
:100F20002AD1300002F0D2FA0500FFF755F9A042AD
:100F3000BCDB012C1ADC300002F0C8FA009028005B
:100F4000FFF736F9461B300002F0D4FC041ED8D05F
:100F500002F0BCFA0190786802F0B8FA009B320007
:100F6000E91A411801980AF0EDFACAE72800FFF7DC
:100F70001FF9013C0500DCE7032B05D13419E478A7
:100F8000023B64001C43BCE70B20C4E708CC000014
:100F900013CC0000F7B54D680F002A0001210A406C
:100FA0002FD1042D2DD90F242B68BE681C40092C8D
:100FB00014D169681B099BB24C100192A34200D85E
:100FC0005C1E39682A48FFF787FC00282DD00F23C4
:100FD0002A681340092B1DD1012317E0032C10D1DF
:100FE0000E4203D1132000F067F9FEBD721001928A
:100FF000FF2AF7D81A0992B25B0F92001C40141B0B
:10100000DFE70B20EFE701339A00AE509C42FADA9B
:101010000020EAE7032BFBD12B0001335A1BA2422D
:10102000F6DC6A461279DA70F7E73968CB0706D53D
:101030004910002901DD8C4209DA1220D3E70D485E
:10104000FFF74AFC2100002801D11130CBE70F2324
:101050002A681340092B03D1013189004E51D7E78B
:10106000032BD5D16B461B796D18EB70D0E7C046CA
:101070000FCC000013CC000010B5012408682042FA
:101080001AD1042818D90F2102681140092901D169
:10109000406810BD032908D113099BB2500F9B0073
:1010A0000840181A40002043F3E7042904D102F055
:1010B0000DFAFFF791F8F5E70B2000F0FDF8E8E7EF
:1010C00010B5034A0B21034804F0ECF910BDC046EB
:1010D000B0CB0000A8CB0000002070470420704770
:1010E0000120704710B5002002F004FC10BD002064
:1010F0007047002070470020704700207047002094
:1011000070470020704700207047002070470000A3
:1011100010B5034A0C21034804F0C4F910BDC046C1
:1011200098CC0000F8CC000010B50124044002D097
:101130004410200010BD042810D90F23026813406A
:10114000042B07D102F0C2F921000A220AF068FE3E
:101150000400EEE7032B01D10430F5E70D22014B2B
:101160001A70E6E7A4020020012210B5024018D14F
:10117000042802D903681A0992B201230B4012D144
:10118000042902D90B681B099BB20024934206D1A3
:1011900004309B000431C318984206D30124200078
:1011A00010BD0022E9E70023EFE704780A78002C5D
:1011B00001D1002AF2D0013001319442ECD0002458
:1011C000EDE70000F7B50700009101933049314B7E
:1011D000002A02D002220A70013A00261A601B6817
:1011E000CE54BE4200DBF7BD009AB300D058294B65
:1011F000274D1C68C8239B0065191C1B012318423E
:1012000006D0254A4310210028000AF0C9FC09E055
:10121000224A002802D004281BD1214A210028009C
:101220000AF0BEFC1A4C20000AF032FD194A019B5C
:101230001060002B0BD07B1EB34208DD194B984287
:1012400005D8431C1360202222540022E2540136A8
:10125000C7E7042819D90F2301680B40042B04D1D8
:1012600002F034F9104A0300CDE7092B03D143689B
:101270000E4A5B10C7E7032B08D10A0992B2490F47
:1012800092000B40D31A0A4ABDE70123094ABAE784
:10129000A5020020C80500200CD6000018CC0000D4
:1012A0001ECC00001F03000037DC000068CF0000E8
:1012B00077CF000082CF0000014B187000207047EC
:1012C000A402002070B501F067FE094C0100251D45
:1012D0001F2228000AF0F4FC28000AF0D9FC04239D
:1012E00004308008000118432060200070BDC04613
:1012F00080020020C368F0B59D00836889B05D1945
:101300000300183306930369069A9F00069B029018
:10131000DF19436901939B00D3180393CD4B1B78CE
:10132000002B26D17F222B68CB491C1213409B0037
:101330005B58043501929F46029B587804F0DCFC10
:101340000023029A137027E0C24B1B78002B10D1A8
:101350002B68019A1C121340BF4A9B009B5804350E
:10136000E9E7069B3A1DD11ABA4BD82928DD1A2283
:101370001A70029BB74C9B6821780193EA1A029B72
:1013800092109B7812021A43029B587804F0BCFC1E
:101390000023029A23701370029B069A9B68ED1A31
:1013A0000193029BAD10DD60069BFE1A029BB610F6
:1013B0001E61039B9B1A029A9B10536109B0F0BDFA
:1013C0001B783C60002B01D01700D2E72B680199F5
:1013D0001C120B40A0499B005B5817000435AAE77C
:1013E000069B3A1DD11A9B4BD82902DD1A221A708E
:1013F000BFE728681B78291D3860002B02D0170032
:101400000D00B6E76B6801991C120B4092499B00D6
:101410005B58170008358EE7069B3A1DD11A8D4B95
:10142000D82902DD1A221A70A3E7A4001B782C1910
:101430003C60002B01D017009BE72B6801991C1220
:101440000B4085499B005B581700043573E7069BEA
:101450003A1DD11A7F4BD82902DD1A221A7088E76B
:101460007E49A40061581B783960002B01D0170019
:101470007FE72B6801991C120B4077499B005B5852
:101480001700043557E7043F744B3A68A400E25054
:10149000704B1B78002B00D06BE72B68019A1C1255
:1014A00013406D4A9B009B58043544E76B4BA400E6
:1014B000E058FFF739FE043F06003868FFF734FEB6
:1014C00036180120654B76000643E650614B1B78C9
:1014D000002B00D04DE72B68019A1C1213405E4A86
:1014E0009B009B58043526E7069B3A1DD11A594BA1
:1014F000D82902DD1A221A703BE70698039C0121C5
:10150000A04202D221000C3909681B783960002BF7
:1015100001D017002DE72B6801991C120B404E4992
:101520009B005B581700043505E7069B3A1DD11A4E
:10153000484BD82902DD1A221A701AE70699039837
:1015400081420FD203000C3B1B6845495B106418B5
:10155000E41AA40023583B603E4B1B78002B05D0B7
:10156000170006E7182119700023F4E72B6801998A
:101570001C120B4038499B005B5817000435DAE613
:10158000069B039A934219D213000C3B1B68344A02
:10159000043FA4185B10E31A039A39689B00995022
:1015A0002C4B1B78002B00D0E3E62B68019A1C1211
:1015B0001340294A9B009B580435BCE61822254B52
:1015C0001A70EDE7069B039A93422DD2244B3E1FDF
:1015D000E31814000C3C04932368049A5B10D31A9C
:1015E000039A9B009858FFF79FFD07903068FFF71C
:1015F0009BFD2468049B64101C1B079BA4001F1800
:1016000001207F00039B0743E7503700114B1B78F5
:10161000002B00D0ADE62B68019A1C1213400E4A35
:101620009B009B58043586E618220A4B1A70EDE79A
:10163000069B3A1DD11A074BD82902DD1A221A70CF
:1016400097E60399A40061581B783960002B09D0F4
:1016500017008EE6A402002068CD0000882D00202F
:10166000FDFFFF3F2B6801991C120B40D9499B00DD
:101670005B58170004355EE6043F039B3A68A400FC
:10168000E250D54B1B78002B00D072E62B68019AF4
:101690001C121340CF4A9B009B5804354BE6039B1A
:1016A000A4001C192368043F38685E10FFF73CFD56
:1016B00036180120C84B76001B7806432660002BA5
:1016C00000D056E62B68019A1C121340C14A9B00B9
:1016D0009B5804352FE6069BA4003F1BBE4CBB4223
:1016E0000CD82378002B00D043E62B68019A1C12FB
:1016F0001340B84A9B009B5804351CE6B74801F0DC
:10170000D5FE2378002B00D033E62B68019A1C12FB
:101710001340B04A9B009B5804350CE6A300ED181B
:10172000002C00DA38E6AC4B1B78002B00D020E60A
:101730002B68019A1C121340A64A9B009B58043543
:10174000F9E5043F3B68042B04D1A300ED18002CFD
:1017500000DA21E6A04B1B78002B00D009E62B68AD
:10176000019A1C1213409B4A9B009B580435E2E5EA
:10177000043F3B68042B04D0A300ED18002C00DAD2
:101780000AE6954B1B78002B00D0F2E52B68019AF6
:101790001C1213408F4A9B009B580435CBE53A1F1F
:1017A00013685B10013B06D401215B00A4000B43CE
:1017B0002D191360F0E5884B17001B78002B00D023
:1017C000D7E52B68019A1C121340824A9B009B5854
:1017D0000435B0E53A00069B0C32D31AD82B03DD52
:1017E0001A227D4B1A70C4E5FF2361005B0019408B
:1017F000FE3BFF3B19433960029906988968241221
:1018000004916D1A0299AD1089782D020D43039948
:101810009D40091A891099401D430B43BB60029BF0
:101820007D609C70E4B26E4BE4000392E358029A30
:101830009360694A1278002A03D008331D00039F81
:1018400097E51D00019A9B680C351C121340614AF4
:101850009B009B58039F6EE53B1F1C68039A069BE9
:1018600093422DD10A20E3070CD4042C13D90F2363
:1018700022681340042B11D1200001F027FE0AF04A
:1018800007FA0630643003F047FE00280FD1043D0C
:10189000069B039380E50720042CF3D02000431E11
:1018A0009841FA234042FF3318400730EAE7029B91
:1018B0002100587804F03AFA0023029A1370E7E7FF
:1018C000039B039A0C3B1B6802995B109B00D31A85
:1018D0000C3B1C601F1D1300083B1B685A108A70CC
:1018E000D2B23F49D2005B0055589B0A029A9B0036
:1018F0009560ED18039B069A043B1B685B109B00E8
:10190000D3180393344B1B78002B00D031E52B68A0
:10191000019A1C1213402F4A9B009B5804350AE57C
:101920003B1F1868FFF700FCA40006003F1B1E28A1
:1019300027DC00280DDC284B1B78002B00D018E595
:101940002B68019A1C121340224A9B009B580435B5
:10195000F1E401F00FFB033E361801F00BFB214BC5
:10196000801B9842F9D81C4B1B78002B00D000E557
:101970002B68019A1C121340164A9B009B58043591
:10198000D9E40123029A137001F0F4FA029B0A3899
:1019900086195E6000E53B1F1868FFF7C5FBA400D1
:1019A00006003F1B00280DDC0B4B1B78002B00D0E2
:1019B000DFE42B68019A1C121340064A9B009B58D7
:1019C0000435B8E4084B984210DD1D22024B1A7012
:1019D000CFE4C04668CD0000A402002094CF0000F0
:1019E000902500203F420F0080EE36000123029A2E
:1019F000137001F0BFFAFA239B005E43029B0A3E7C
:101A000030185860C8E4A300FF1A002320001A0011
:101A10003900FFF7D7FBD44ED44C3168200001F0D9
:101A200075FFD34B31681860200004F025F8316849
:101A3000200004F082F9CF4B1B78002B00D098E4F3
:101A40002B68019A1C121340CB4A9B009B5804350B
:101A500071E4C84BA4001B783F1B002B00D088E426
:101A60002B68019A1C121340C34A9B009B580435F3
:101A700061E4029803F0B4FDBE4B1B78002B00D04C
:101A800077E42B68019A1C121340BB4A9B009B58B9
:101A9000043550E43B1F1B68002B3ED13B000C3B40
:101AA0001B68DA072CD5390001225B105800083971
:101AB00002430A60002B44DD012259001143381F04
:101AC00001603900083909681141CB1A39000C3915
:101AD0000968114224D09B189340A4001343039A31
:101AE000A350A44B1B78002B00D042E42B68019A32
:101AF0001C121340A04A9B009B580435FFF71BFCA7
:101B0000042B06D90F211A680A40092A01D15B6803
:101B1000C9E71922974B1A702BE45B10013BC9E708
:101B2000042909D90F200A680240092A04D1023386
:101B30009B005B58A400D2E719228E4B1A70FFF766
:101B400018FC0435CDE7A300069AFB189B1AD82B86
:101B500013DC0122631E002C14DC864B1B78002B47
:101B600001D0FFF706FC2B68019A1C121340824A31
:101B70009B009B580435FFF7DEFB1A227D4B1A7041
:101B8000FFF7F7FB3A601C000437E3E7069A3B1DBA
:101B90009B1A784ED82B03DD1A233370FFF7E9FB2D
:101BA000069B039AA40093422AD23B1F1868FFF7B2
:101BB000BBFA011E21DD039B0C3B1A6852108242C6
:101BC0001BDB9007801A6D4B4018C018039B8000E8
:101BD000C2583B1B1A60674B3F1B1B780437002B16
:101BE00001D0FFF7C6FB2B68019A1C121340624A12
:101BF0009B009B580435FFF79EFB20233370EAE7D8
:101C00001823FBE75A4BA4001A683B1B1F001A60FD
:101C1000584B04371B78002B01D0FFF7AAFB2B6829
:101C2000019A1C121340544A9B009B580435FFF73D
:101C300082FB3B1F1A68042A11D1A4002D194D4BB9
:101C40001B78002B01D0FFF794FB2B68019A1C1224
:101C50001340494A9B009B580435FFF76CFB1F005B
:101C6000EDE73A1F1368042B04D0002313603A00F9
:101C7000A4002D193F4B1B78002B02D01700FFF753
:101C800078FB2B6801991C120B403B499B005B5869
:101C900017000435FFF74FFBA3009C46FE1A002CEB
:101CA00017DC1C22334B1A70002333606346FF1A83
:101CB000304B04371B78002B01D0FFF75AFB2B6801
:101CC000019A1C1213402C4A9B009B580435FFF7C5
:101CD00032FB002033685A108300F15801230B4077
:101CE00003D10D21234A1170DFE749108A4200DD3C
:101CF0000A0001308442EFDC012352001343D4E791
:101D0000A3009C46FE1A002C17DC1C22194B1A70EB
:101D1000002333606346FF1A164B04371B78002BF1
:101D200001D0FFF726FB2B68019A1C121340124AC0
:101D30009B009B580435FFF7FEFA002033685A10C9
:101D40008300F15801230B4003D10D21094A117082
:101D5000DFE749108A4200DA0A0001308442EFDCF2
:101D6000012352001343D4E7C8050020A502002038
:101D700008000020A402002068CD0000FCFFFF3F07
:101D80003B00083B1868FFF7CFF93B1F06001868B7
:101D9000FFF7CAF90023864200DA0433A4003A1B95
:101DA00017001360E54B04371B78002B01D0FFF7B9
:101DB000E0FA2B68019A1C121340E14A9B009B58E1
:101DC0000435FFF7B8FA3B00083B1868FFF7ACF999
:101DD0003B1F06001868FFF7A7F9F30FC217B042C0
:101DE0005341A4003A1B17009B001360D34B0437E8
:101DF0001B78002B01D0FFF7BCFA2B68019A1C124C
:101E00001340CF4A9B009B580435FFF794FA3B00E0
:101E1000083B18683B1F1968A600BE1B04238142BB
:101E200002D0042802D80023336018E001239C4626
:101E30001842F8D10F2302681A40042AF3D16346EE
:101E40001942F0D10429EED90B680B321340042B50
:101E5000E9D1FFF789F9431E984180003060B74B04
:101E6000A4001B783F1B0437002B01D0FFF781FA39
:101E70002B68019A1C121340B14A9B009B580435F1
:101E8000FFF759FA3B00083B18683B1F1968A6008A
:101E9000BE1B0023814202D0042802D804233360F1
:101EA00018E001239C461842F8D10F2302681A401B
:101EB000042AF3D163461942F0D10429EED90B6804
:101EC0000B321340042BE9D1FFF74EF9434258413E
:101ED00080003060994BA4001B783F1B0437002B17
:101EE00001D0FFF746FA2B68019A1C121340944A5E
:101EF0009B009B580435FFF71EFA3B00083B18680F
:101F0000FFF712F93B1F06001868FFF70DF9F317EA
:101F1000C20F86425341A4003A1B17009B00136076
:101F2000864B04371B78002B01D0FFF722FA2B6871
:101F3000019A1C121340824A9B009B580435FFF7FC
:101F4000FAF93B00083B1868FFF7EEF83B1F060064
:101F50001868FFF7E9F80023864200DD0433A40087
:101F60003A1B17001360754B04371B78002B01D008
:101F7000FFF7FFF92B68019A1C121340704A9B006F
:101F80009B580435FFF7D7F93B1F1B68A400043B9F
:101F90005A1E93413A1B17009B001360674B04378E
:101FA0001B78002B01D0FFF7E4F92B68019A1C1273
:101FB0001340634A9B009B580435FFF7BCF93B0074
:101FC000083B1868FFF7B0F83B1F06001868FFF7DA
:101FD000ABF832180120A4003B1B1F005200024343
:101FE0001A60564B04371B78002B01D0FFF7C1F95C
:101FF0002B68019A1C121340514A9B009B580435D0
:10200000FFF799F93B00083B1868FFF78DF83B1F75
:1020100006001868FFF788F8321A0120A4003B1B5D
:102020001F00520002431A60444B04371B78002BF8
:1020300001D0FFF79EF92B68019A1C121340404A09
:102040009B009B580435FFF776F93B00083B186866
:10205000FFF76AF83B1F06001868FFF765F80200F3
:102060000120A4003B1B1F007243520002431A6070
:10207000324B04371B78002B01D0FFF77AF92B681D
:10208000019A1C1213402E4A9B009B580435FFF7FF
:1020900052F93B1F1868FFF747F8061E17D11F2398
:1020A000264A1370A4003B1B1F001E60234B0437FD
:1020B0001B78002B01D0FFF75CF92B68019A1C12EA
:1020C00013401F4A9B009B580435FFF734F93B002F
:1020D000083B1868FFF728F8310007F00BF90126D4
:1020E00040000643DEE73B1F1868FFF71DF8061E99
:1020F00017D11F23114A1370A4003B1B1F001E6041
:102100000E4B04371B78002B01D0FFF732F92B68F8
:10211000019A1C1213400A4A9B009B580435FFF792
:102120000AF93B00083B1868FEF7FEFF310007F094
:10213000C7F9012649000E43DEE7C046A40200208D
:1021400068CD00003B1F1868FEF7EEFFC21780182D
:1021500050400122A4003B1B1F00400010431860A8
:10216000F14B04371B78002B01D0FFF702F92B68E5
:10217000019A1C121340ED4A9B009B580435FFF74F
:10218000DAF8A300FE1A3068012C24D1FEF7CCFF48
:102190000494079009F0D2FC0799002900DC012182
:1021A00007F08EF9049BA400C918012349001943C4
:1021B000DD4B3F1B1B7831600437002B01D0FFF74C
:1021C000D8F82B68019A1C121340D84A9B009B58E0
:1021D0000435FFF7B0F8FEF7A7FF04907068FEF72C
:1021E000A3FF049B0130C31A0793D3E7A300FE1A91
:1021F00031002000049301F00FFD049B3060FF1AB2
:10220000C94B04371B78002B01D0FFF7B2F82B68BD
:10221000019A1C121340C54A9B009B580435FFF7D6
:102220008AF83B00083B1868FEF77EFF3B1F06005C
:102230001868FEF779FF02000120A4003B1B1F0075
:102240003240520002431A60B74B04371B78002B10
:1022500001D0FFF78EF82B68019A1C121340B34A85
:102260009B009B580435FFF766F83B00083B186855
:10227000FEF75AFF06003B1F1868FEF755FF3200B5
:1022800002430120A4003B1B1F00520002431A60BE
:10229000A54B04371B78002B01D0FFF76AF82B6899
:1022A000019A1C121340A14A9B009B580435FFF76A
:1022B00042F83B00083B1868FEF736FF06003B1F5C
:1022C0001868FEF731FF320042400120A4003B1B9A
:1022D0001F00520002431A60934B04371B78002BF7
:1022E00001D0FFF746F82B68019A1C1213408F4A61
:1022F0009B009B580435FFF71EF83B1F1868FEF73C
:1023000013FFC0430122A4003B1B1F0040001043E9
:102310001860854B04371B78002B01D0FFF729F894
:102320002B68019A1C121340804A9B009B5804356D
:10233000FFF701F83B00083B1868FEF7F5FE0600C2
:102340003B1F1868FEF7F0FE320082405100012268
:10235000A4003B1B1F000A431A60734B04371B7811
:10236000002B01D0FFF705F82B68019A1C121340CF
:102370006E4A9B009B580435FEF7DDFF3B00083B8F
:102380001868FEF7D1FE06003B1F1868FEF7CCFE6A
:102390003200024151000122A4003B1B1F000A43EE
:1023A0001A60614B04371B78002B01D0FEF7E1FF68
:1023B0002B68019A1C1213405C4A9B009B58043501
:1023C000FEF7B9FF3B000C3B1868FEF7ADFE3B0083
:1023D000083B06001868FEF7A7FEF1170200C317B6
:1023E000300007F0BFF83B1F049005911868FEF716
:1023F0009BFE02000498059907F068F8430001204D
:10240000A4003E1B37001843474B30601B7804374D
:10241000002B01D0FEF7ADFF2B68019A1C12134070
:10242000424A9B009B580435FEF785FFA300FE1A25
:10243000310020000493FEF7C1FC049B3060FF1ABA
:10244000394B04371B78002B01D0FEF792FF2B6825
:10245000019A1C121340354A9B009B580435FEF725
:102460006AFFA300FF1A39002000FEF7BFFC2E4BC5
:102470001B78002B01D0FEF77CFF2B68019A1C1201
:1024800013402A4A9B009B580435FEF754FFA300D3
:10249000FE1A310020000493FEF7E8FC049B306034
:1024A000FF1A214B04371B78002B01D0FEF761FF88
:1024B0002B68019A1C1213401C4A9B009B58043540
:1024C000FEF739FFA300FF1A39002000FEF762FD76
:1024D000154B1B78002B01D0FEF74BFF2B68019AA0
:1024E0001C121340114A9B009B580435FEF723FF32
:1024F000A300FE1A310020000493FEF7BDFD049BEB
:102500003060FF1A084B04371B78002B01D0FEF710
:1025100030FF2B68019A1C121340044A9B009B5801
:102520000435FEF708FFC046A402002068CD000075
:102530003B1F186800F0CAFF3A00083A126803000F
:10254000A400D10729D4042A0CD910680F22104006
:10255000013808280FD806F02FFE052026220E0E7F
:102560000E0E2400EE49180009F088FB4342584142
:102570003B1B80001860EB4B3F1B1B780437002B84
:1025800001D0FEF7F6FE2B68019A1C121340E64AB2
:102590009B009B580435FEF7CEFEE449E3E7E4498F
:1025A000E1E7E449DFE7E449DDE7069B3E1DF31A76
:1025B000DC4CD82B03DD1A232370FEF7DAFE00F083
:1025C000E3FC43000120184323783860002B02D03D
:1025D0003700FEF7CEFE2B68019A1C121340D24A38
:1025E0009B009B5837000435FEF7A5FE069B3E1D59
:1025F000F31ACC4CD82B03DD1A232370FEF7B9FE57
:1026000000F0B8FCCD4B400018400123184323785C
:102610003860002B02D03700FEF7ABFE2B68019A22
:102620001C121340C04A9B009B5837000435FEF72C
:1026300082FE069B3E1DF31ABA4CD82B03DD1A23EB
:102640002370FEF796FE00F09FFCBD4B1A68831ABC
:10265000904201D2BB4A9B1801205B0003433B60C0
:102660002378002B02D03700FEF783FE2B68019AF7
:102670001C121340AC4A9B009B5837000435FEF7F0
:102680005AFE00F081FCAE4BA4001860A54B3F1B26
:102690001B78002B01D0FEF76CFE2B68019A1C12F0
:1026A0001340A14A9B009B580435FEF744FE0123CA
:1026B000A600BE1B20001A003100FEF783FDA24CCD
:1026C0002068643002F028FF002802D1043DFEF7A4
:1026D00063FE029B21685A789C4803F03CFB01236F
:1026E000029A3700137000F045FC994B22681B6872
:1026F000063253431818029B5860FEF74DFEA600A1
:10270000BE1B2000012300223100FEF75BFD8E4C32
:102710002068643002F000FF0028D7D08B4803F017
:102720009BF8DCE7A4003E1BFEF7CCFD37007D4B99
:1027300030601B780437002B01D0FEF71AFE2B689F
:10274000019A1C121340784A9B009B580435FEF7EF
:10275000F2FD744BA4001B783F1B002B01D0FEF749
:1027600008FE2B68019A1C1213406F4A9B009B586D
:102770000435FEF7E0FD03F0B1FAFEF71FFEA400FA
:102780003E1B300000F02FFC3700664B30601B789A
:102790000437002B01D0FEF7ECFD2B68019A1C12C8
:1027A0001340614A9B009B580435FEF7C4FDA4000A
:1027B0003E1B300000F019FC37005A4B30601B788C
:1027C0000437002B01D0FEF7D4FD2B68019A1C12B0
:1027D0001340554A9B009B580435FEF7ACFDA300FF
:1027E000FE1A31002000049300F002FC049B3060CC
:1027F000FF1A4C4B04371B78002B01D0FEF7B9FDB4
:102800002B68019A1C121340474A9B009B580435C1
:10281000FEF791FDA4003F1B380000F01BFC414B6C
:102820001B78002B01D0FEF7A4FD2B68019A1C1227
:1028300013403D4A9B009B580435FEF77CFDA300E6
:10284000FE1A31002000049300F02CFC049B306041
:10285000FF1A344B04371B78002B01D0FEF789FD9B
:102860002B68019A1C1213402F4A9B009B58043579
:10287000FEF761FDA4003F1B380000F055FC294B1A
:102880001B78002B01D0FEF774FD2B68019A1C12F7
:102890001340254A9B009B580435FEF74CFD01214F
:1028A000200000F029FC1F4B1B78002B01D0FEF705
:1028B00060FD2B68019A1C1213401B4A9B009B5819
:1028C0000435FEF738FD0021200000F015FC154B03
:1028D0001B78002B01D0FEF74CFD2B68019A1C12CF
:1028E0001340114A9B009B580435FEF724FDA400B9
:1028F0003E1B300000F03AFC37000A4B30601B787A
:102900000437002B01D0FEF734FD2B68019A1C120E
:102910001340054A9B009B580435FEF70CFDC0464A
:10292000A4CF0000A402002068CD0000ACCF0000BE
:10293000B3CF0000BACF0000BFCF0000FEFFFF7F83
:10294000D005002037894100C8050020A5020020DD
:1029500004000020A4003E1B300000F01BFC3700E8
:10296000EE4B30601B780437002B01D0FEF701FDE1
:102970002B68019A1C121340E94A9B009B580435AE
:10298000FEF7D9FCA4003F1B380000F0DDFBE34B51
:102990001B78002B01D0FEF7ECFC2B68019A1C126F
:1029A0001340DF4A9B009B580435FEF7C4FCA4008B
:1029B0003F1B380003F0EAFCD84B1B78002B01D0FA
:1029C000FEF7D7FC2B68019A1C121340D44A9B00D7
:1029D0009B580435FEF7AFFCA4003E1B300003F00B
:1029E0006FFD3700CD4B30601B780437002B01D0D2
:1029F000FEF7BFFC2B68019A1C121340C84A9B00CB
:102A00009B580435FEF797FCA4003F1B380003F0E9
:102A10006DFCC24B1B78002B01D0FEF7AAFC2B6883
:102A2000019A1C121340BE4A9B009B580435FEF7C6
:102A300082FCA4003E1B300003F06EFC3700B74B55
:102A400030601B780437002B01D0FEF792FC2B6816
:102A5000019A1C121340B24A9B009B580435FEF7A2
:102A60006AFCA300FF1A3900200001F015FCAB4BF3
:102A70001B78002B01D0FEF77CFC2B68019A1C12FE
:102A80001340A74A9B009B580435FEF754FCA30053
:102A9000FF1A3900200001F013FAA04B1B78002B1D
:102AA00001D0FEF766FC2B68019A1C1213409C4A69
:102AB0009B009B580435FEF73EFCA300FF1A39002B
:102AC000200001F021FB954B1B78002B01D0FEF775
:102AD00050FC2B68019A1C121340914A9B009B5892
:102AE0000435FEF728FCA300FF1A3900200001F08E
:102AF00033FB8A4B1B78002B01D0FEF73AFC2B6886
:102B0000019A1C121340864A9B009B580435FEF71D
:102B100012FCA300FE1A31002000049303F068FDAC
:102B2000049B3060FF1A7D4B04371B78002B01D0CB
:102B3000FEF71FFC2B68019A1C121340784A9B0079
:102B40009B580435FEF7F7FBA300FE1A3100200066
:102B5000049303F055FD049B3060FF1A6F4B04375C
:102B60001B78002B01D0FEF704FC2B68019A1C1285
:102B700013406B4A9B009B580435FEF7DCFBA30017
:102B8000FE1A31002000049303F042FD049B3060E4
:102B9000FF1A624B04371B78002B01D0FEF7E9FBCC
:102BA0002B68019A1C1213405D4A9B009B58043508
:102BB000FEF7C1FBA300FE1A31002000049303F0CE
:102BC0004DFB049B3060FF1A544B04371B78002BDD
:102BD00001D0FEF7CEFB2B68019A1C121340504A1D
:102BE0009B009B580435FEF7A6FBA300FF1A390093
:102BF000200001F09DF9494B1B78002B01D0FEF716
:102C0000B8FB2B68019A1C121340454A9B009B5845
:102C10000435FEF790FBA300FF1A3900200001F0F5
:102C2000C3FA3E4B1B78002B01D0FEF7A2FB2B68AA
:102C3000019A1C1213403A4A9B009B580435FEF738
:102C40007AFBA300FE1A31002000049301F028FA59
:102C5000049B3060FF1A314B04371B78002B01D0E6
:102C6000FEF787FB2B68019A1C1213402C4A9B002D
:102C70009B580435FEF75FFBA300FF1A39002000C4
:102C800001F0D6F9254B1B78002B01D0FEF771FB24
:102C90002B68019A1C121340214A9B009B58043553
:102CA000FEF749FB069B029AFB1A9B101361A300D7
:102CB000FF1A3900200002F00DFE184B1B78002B84
:102CC00001D0FEF756FB2B68019A1C121340144AE0
:102CD0009B009B580435FEF72EFB069B029AFB1ABD
:102CE0009B101361A300FE1A31002000049302F030
:102CF000F1FD049B3060FF1A084B04371B78002B52
:102D000001D0FEF736FB2B68019A1C121340044ACF
:102D10009B009B580435FEF70EFBC046A402002022
:102D200068CD00000023F7B55A1E0192002B07DA88
:102D300001F0C8FA02F0FEFE03F06CF819230193CB
:102D400000263000194B1968B14212DD184B1A6881
:102D500001328A420FDAF0241A601D68154F6C4365
:102D6000E35D002B1FD0E419022B06D12000FEF7F3
:102D7000C1FA019BD8E70022EDE7012B0DD1002815
:102D800001D100F0F7F8F0226A43BB185B680A49EA
:102D9000C31A8B4201D80223BB54F0235D43054B79
:102DA000EB5C022BE2D00136CCE7C046CC0500201C
:102DB00000000020301C00203F420F0001220021B3
:102DC0000A4B0B481A61195004301950A2210420F3
:102DD000C9005850C121C0208900800258501A6093
:102DE000044BFC311960044B1A70704700A000407E
:102DF0000405000000E100E0F70500200420704712
:102E0000F8B550C9012322001A40101E2DD03340BE
:102E1000181E2AD0641000201C2C26D81D4B7610BA
:102E200035009E4200DD1D001B4F3B5D012B05D090
:102E30000121200004F07AFD01233B55174B1B783C
:102E4000002B01D1FFF7BAFF0023154A9E420DDC8B
:102E5000FF2514491448D65CB44202D15E0070527A
:102E6000D5540133042BF6D10420F8BDD15C8C423B
:102E700003D10C4A5B009D52F6E70133042BF5D1D8
:102E80000023D15CFF2901D1D454F2E70133042B94
:102E9000F7D1E9E788130000D8050020F7050020E6
:102EA0001C0000200E000020DC05000070B530C9B9
:102EB000012322001A40101E1BD02B40181E18D0D0
:102EC00064101C2C00D90024174E335D012B05D053
:102ED0000121200004F02AFD012333556910080068
:102EE000124A1038124B904204D9012252421A6001
:102EF000042070BD1C600F4806F0FCF90E4B1880D2
:102F00000E4B1B78002B02D1FFF758FFF0E7012290
:102F10000B4B9A64A922D2009A588018A82280B23A
:102F2000D2009850E4E7C046D80500209086010002
:102F30001800002020A107000C000020F705002049
:102F400000A00040030010B50120002B02DC1B3064
:102F5000FEF7B2F910BD0420704710B5002803DC5D
:102F60001C20FEF7A9F910BD0B680020DB07FAD47E
:102F70000D30F6E70122034B1A64A822D2009858BC
:102F80007047C0460080004010B5FFF7F3FFFA21FC
:102F9000890006F025F910BD004870471CD00000DC
:102FA0001D20704770B5054E0400335C0D008B4248
:102FB00002D004F0BBFC355570BDC046D8050020DA
:102FC00070B50024064D635D012B05D10021200062
:102FD00004F0ACFC0023635501341D2CF2D170BD0C
:102FE000D805002070470D2070473B207047000037
:102FF000F8B501240B6806000D00234204D10D2012
:10300000FEF75AF92000F8BD5B102000052BFAD816
:103010000E4A9B009C580E4F3B5D002B05D00021B3
:10302000200004F083FC00233B55012E06DD6B6875
:10303000042B03D10221200004F078FC200004F0CE
:1030400023FB012440002043DDE7C04604D00000FC
:10305000D8050020F8B501260568354202D044683D
:10306000344203D10D20FEF727F9F8BD6D101C2D59
:10307000FBD80A4F7B5D012B04D03100280004F0FF
:1030800055FC7E55064964108C4202DCE143C917A9
:103090002140280004F07EFBE7E7C046D805002069
:1030A000FF03000070B501240D68254204D10D20F6
:1030B000FEF702F9200070BD6D101C2D17D80024FA
:1030C000012804DD4C68043C63425C416400094E05
:1030D000735DA34204D02100280004F027FC74553E
:1030E000280004F057FC03000420012BE3D000204B
:1030F000E1E7C046D805002070B504000D001C288B
:103100000ED8084E335C012B04D0012104F00EFCD4
:1031100001233355290020004D1EA94104F024FC51
:1031200070BDC046D8050020036810B5DA0703D487
:103130000D20FEF7C1F810BD4168581004394A420D
:103140005141FFF7D9FFF6E737B569460A00064B4C
:1031500030CB30C203680220042B02D100F0D4FF30
:1031600037BD00F0F9FFFBE7CCCF000010B5084CED
:103170006379002B05D00021052004F0D7FB002344
:103180006371052004F006FC43425841800010BDE5
:10319000D805002010B5084CE37A002B05D000219B
:1031A0000B2004F0C3FB0023E3720B2004F0F2FBBE
:1031B00043425841800010BDD8050020F7B5304D7E
:1031C000304E6B6C002B15D0A8240023E400375937
:1031D0006B642D4B186800280CDB2C4B19784A4285
:1031E0005141C9B2197004F0BFFB294B1B88DF198C
:1031F000BFB23751AB6C002B39D00021254B264F85
:10320000F458A9643A780C340193244D8A4206D0CC
:103210002B68032B03D8224AD05C04F0A5FB2B6853
:10322000204A0133134004D50422013B5242134388
:1032300001331B4900228C462B60042B18D06046BA
:10324000C05C591CFF2802D10B000122F5E7002ABF
:1032500000D02B60012104F087FB01233B702B6819
:10326000114A5B009B5AE418019BA4B2F450F7BDCD
:1032700001235B422B6000233B700C4BF3E7C046FD
:10328000FCA0004000A0004018000020F60500202F
:103290000C00002044050000F5050020D4050020A6
:1032A0001C000020030000800E000020504600009B
:1032B000084B094AFF201A805A809A80DA8000233E
:1032C000064A07491370074A087048708870C8702A
:1032D000136070470E000020DC050000F50500209B
:1032E0001C000020D40500200122024B52421A602B
:1032F0007047C0461800002010B5034A0621034855
:1033000002F0D0F810BDC046D4CF00003ED7000078
:10331000E12170B54902194803F0AEFF00240122F3
:103320000320174B17491A615C500431585080181C
:10333000083158501A60063004F0A0F9FF21124AF3
:10334000A15401341D2CFBD1012200200F4B0100A0
:103350001A6004230E4A0F4D1468002CFCD02C6810
:103360000002013B20431160002BF5D101220A4BE2
:103370001A6004F03DF901F0F1F870BDB81B0020AF
:103380000080004004050000D805002000D0004067
:1033900000D1004008D5004004D00040F8B50B4EE5
:1033A000070030000D0003F0AFFF0400A84200DD6D
:1033B0002C003D00EB1B9C4205DD300003F0AEFF0E
:1033C00028700135F6E72000F8BDC046B81B002084
:1033D00010B50100014803F057FF10BDB81B0020D5
:1033E00010B5054C200003F05DFFE12120004902EB
:1033F00003F042FF10BDC046B81B0020C3070CD429
:10340000064B1B68834208D8054B1B68984204D8BA
:10341000031F1B68002B00D0180070470006002017
:10342000FC0500200023012210B50A489900013351
:103430004250642BFAD1084C084B00211A6020003E
:10344000074A08F09BF8074B074A6360074B1A606E
:1034500010BDC046882D0020040600200800002072
:10346000D40900003027000008060020F8050020DD
:1034700010B5044B044A1A60044B054A1A60FFF762
:10348000D1FF10BD0006002004060020FC0500202E
:10349000D80F0020044B1B681868000980B202385E
:1034A000C343DB1718407047F805002000B59BB0F8
:1034B0000200054901A808F0A5FB01A802F0E8F9FF
:1034C00002F0A8FCFCE7C046A0D000000B4BC207EE
:1034D00004D4042804D80A4B00D00A4B18007047C3
:1034E0000F2203681A40031D042AF7D0064B092A4D
:1034F000F4D0064B032AF1D0054BEFE77AD0000059
:103500001ECC000018CC000084D0000094D0000035
:103510008BD000000020064A0649131F186013686C
:103520001B099BB202339B00D2188A42F5D3704725
:1035300008060020D80F0020F7B50F240126314BD4
:10354000314A1968314B324D186813681F00274003
:10355000072F26D813681B099BB202339B00D21891
:10356000AA42F2D300242B4EA500AD192868FFF71C
:1035700045FF01342860642CF6D1274C2068FFF702
:103580003DFF2060254C2068002802D0FFF736FF61
:1035900020600025224B1B680093009B9D4214DB9A
:1035A000F7BD1B099BB29B00D3189A42D2D01F686B
:1035B000374208D1B94206D2B84204D3043F3F682B
:1035C000002F00D01F60043BEFE7F0236B43154A48
:1035D0009B181A78002A01D10135DEE71F693C23C8
:1035E00000266B43DB199B0001930136BB1BF3D410
:1035F000019BB4001C1B0B4B1C19A069FFF7FEFEBE
:10360000A061F2E70006002008060020FC0500206B
:10361000D80F0020882D002008000020D80F00209F
:10362000CC050020301C0020F7B50124204246D1F3
:10363000234B1B689C46984241D3224B1B68019345
:1036400098423CD8031F1B68002B38D10200036846
:1036500000941B099BB2002B0FD10099131F196016
:1036600090422CD015682B1F1B68990069180C68B4
:10367000013B14600A602A00EDE79D005519296896
:10368000009C214219D18C4517D8019C8C4214D33F
:103690000E1F3468002C10D10F680F343C40072CEB
:1036A00008D92F60151F2B600B680A601B099BB29D
:1036B0000A00D0E700993160CDE7013BCBE7F7BDC9
:1036C00000060020FC0500200D4970B50A000D4DD4
:1036D0001368141F1B0926689BB2981C002E0BD080
:1036E00000238A4200D00B0023608300C9188000A9
:1036F0001218AA42ECD370BD1B011360F7E7C04655
:1037000008060020D80F0020F8B5124C27000F2221
:103710003B681D09ADB213420DD06E1CB600A74226
:1037200004D032003900200007F015FF0022A31951
:103730000436A4191A600235AD00074B7F199F4269
:10374000E5D31B1B9B10013B1B012360034B1C603B
:10375000F8BDC04608060020D80F0020F80500205C
:10376000F0B59BB0FFF706FC00240700214AA30038
:10377000D0580134FFF758FF642CF7D11E4B18685E
:10378000FFF752FF1D4B1868002801D0FFF74CFFD0
:1037900000261B4B1B689E4217DBFFF795FFFFF7C8
:1037A000CBFEFFF7B1FFFFF7E5FB164BC21B1B6813
:1037B00015491B6801A81B099BB2023B08F022FABD
:1037C00001A802F065F81BB0F0BDF02575430F4B62
:1037D000ED182B78002B01D10136DAE72B695C1E3E
:1037E000002CF9DBA300EB189869FFF71DFF013CE3
:1037F000F6E7C046882D002008000020D80F0020E2
:10380000CC050020F80500205AD00000301C002014
:10381000F7B5174D4F1C2B6806001B680C001B09E1
:103820009BB201929F420BDBFFF79AFF2B681B684C
:103830001B099BB29F4203DB0A20FDF73DFDFEBD45
:103840002868A71CBA00DB1B81181B010B602960CC
:103850000021031F19600F231E400300240126438B
:1038600040C3083A9A189A42E9D9019902C3FAE783
:10387000F8050020F7B503000122134004000D00F5
:103880000193002B2BD1174B1B68834227D8164B73
:103890001B68834223D90F23144F386000681840F7
:1038A000FFF7B6FF019B3C68061E3B6017D02368FC
:1038B00004301B099BB29D4200DD1D00AA00211DA2
:1038C000251F07F03FFEFFF725FE2E60FFF734FEB1
:1038D00000232B602268064B134023603400200035
:1038E000FEBDC04600060020FC050020D80F0020C9
:1038F000F0FF0F000323043010B5C1171940091859
:10390000891000220420FFF783FF10BD70B5050069
:1039100008000C00FFF7EEFF0023002804D170BD63
:10392000E95CC21811710133A342F9DBE343DB17F1
:103930001C40002304192371F1E7F0B50C009BB083
:10394000022804DC1C20FDF7B7FC1BB0F0BD0123EE
:103950000868184206D1042804D90F2601683140AE
:10396000042901D00E20EEE761680D001D40F9D159
:103970000429F7D90A683240042AF3D1A2681A420E
:1039800001D10D20DFE7FFF7A1FD06006068FFF71A
:103990009DFDA768010001AC7F103000257003F089
:1039A00016F839006423220003F076F8200008F0AE
:1039B0006FF901002000FFF7A9FFC6E710B51C4C06
:1039C000A544041E02D1FFF795FF0BE002F018FF9B
:1039D0000138062828D805F0EFFB09091118290439
:1039E000240000208023DB009D4410BD200002F055
:1039F00083FF011B2000FFF789FFF3E7200002F09F
:103A000029FF430001201843ECE780226946D200D9
:103A1000200002F036FF684608F03AF901006846D7
:103A2000E9E704210348E6E70020CCE70420D9E7D2
:103A300000FCFFFFE8D0000070B50C00022803DC9A
:103A40001C20FDF739FC70BD01230868184206D11F
:103A5000042804D90F2501682940042901D00E202B
:103A6000EFE761681942FAD10429F8D90A682A40B7
:103A7000042AF4D1A2681A4201D10D20E1E7FFF730
:103A800025FD05006068FFF721FDA46801006410B2
:103A9000280002F09CFF210002F0D9FFFFF78EFF03
:103AA000D1E770B50D00012803DC1C20FDF704FCF4
:103AB00070BD01240868204206D1042804D90F21D2
:103AC00002680A40042A01D00E20EFE76A68224209
:103AD000FAD1042AF8D913680B40042BF4D1FFF76C
:103AE000F5FC06006868FFF7F1FC0100300002F009
:103AF0006EFF02F0F0FF40002043D9E7F8B5070061
:103B00000C001C20012F0BDD01250868284206D17E
:103B1000042804D90F2102680A40042A03D00E2089
:103B2000FDF7CAFBF8BD62682A42F8D1042AF6D92B
:103B300013680B40042BF2D1FFF7C8FC0600606845
:103B4000FFF7C4FC0100022F14D0A4682C4211D04E
:103B50006410300002F03BFF050002F051FE012826
:103B600011D1002C02DD0135012C06D12800FFF710
:103B700025FFD7E701246442EBE7280002F0C8FEE6
:103B8000013C0500F0E70228F0D1002CEEDD013504
:103B9000012CEBD000222800110002F0EBFE02F015
:103BA000B7FE013C0500F3E710B5012408680440A6
:103BB00016D04410200005F031FE154905F0FCFC3C
:103BC00007F0E2FB04F02AF80022124B06F096FD03
:103BD00003F0CCFF07F068FB43000120184310BD41
:103BE000042810D90F2302681340042B07D1FFF7D4
:103BF0006DFC21000A2208F013F90400DAE7032B18
:103C000001D10430F5E70D20FDF756FBD2E7C046A1
:103C1000D30237390000D040086870B50124050090
:103C2000254006D1042804D90F2302681340042B31
:103C300003D00E20FDF740FB70BDFFF747FC037873
:103C40002900233B5A4253411022C01808F0E8F8DB
:103C500080239B05C218044B9A4201D91420E9E73E
:103C600040002043E8E7C046FFFFFF3F10B5034A8E
:103C70000621034801F016FC10BDC046B8D0000074
:103C8000B1D000000020704710B51E20FDF714FBD6
:103C900010BD10B51E20FDF70FFB10BD10B51E2086
:103CA000FDF70AFB10BD10B51E20FDF705FB10BD8A
:103CB00010B51E20FDF700FB10BD10B51E20FDF74E
:103CC000FBFA10BD10B51E20FDF7F6FA10BD10B5B9
:103CD0001E20FDF7F1FA10BD10B51E20FDF7ECFA1D
:103CE00010BD10B51E20FDF7E7FA10BD10B5034A50
:103CF0000B21034801F0D6FB10BDC04624D10000C3
:103D00007CD100000120034B1860034B1B688340EB
:103D100018437047FC0F0020DC0F0020F0B5EFF3D4
:103D200010810123194083F31088134C134AA446D1
:103D30001268134E013A9340124F134A002B17D0CA
:103D4000146803420FD03D682C60C046C046C04690
:103D5000C046C046C046C046C0460C4C15682468E4
:103D600025605B08EAE765462C6014683460F8E774
:103D700081F31088F0BDC0460805005020000020E7
:103D80000C050050E80F0020F00F0020E40F002089
:103D900030B585B001AD0C220649280007F0D2FBF2
:103DA0000024285D01210134FFF7FCF80C2CF8D128
:103DB00005B030BD11D20000F7B56A46394B01ADF0
:103DC00013801C239370384B2B800A23AB70FFF7B2
:103DD000D1F8364B364CC0182368984201D20023E4
:103DE00023602668002E3DD16B469F5D012138007F
:103DF000FFF7D8F801360021380003F0B5FD032E97
:103E0000F2D10026AF5D01213800FFF7CBF8013673
:103E10000121380003F0A8FD032EF3D1C82001389A
:103E2000C046C046C046C046C046C046C046C04662
:103E3000C046C046C046C046F1D100212878FFF7F1
:103E4000B1F868780021FFF7ADF8A8780021FFF7F6
:103E5000A9F8FFF78FF8FA2300251B01C01820608E
:103E60002800FEBDFFF786F8236800259842F7D3A7
:103E7000032003F009FC0600042003F005FC3618BB
:103E80000A2003F001FC0B4B9B1B181A0A4BA8429B
:103E900006DB18600023094A236013600125DFE771
:103EA0001D60F7E71A1B0000030400001027000044
:103EB000F40F0020E3030000DC0F0020FC0F0020C3
:103EC0000022054B10B51A60044B1B68934201D0C9
:103ED00002F036FC002010BDF80F0020DC1A002094
:103EE00010B5041E10DA00240A4BA400E258012386
:103EF0009340094A09491360094A1160094A0A496D
:103F000011600A4A136010BDFFF74AF8A042EADDCB
:103F1000EAE7C04620DF0000F00F0020080500504F
:103F2000E80F0020E40F00200C0500501805005099
:103F3000F0B53B4B85B01B680C00002B03D1012072
:103F40004042FFF7CDFF246801222700174028D008
:103F5000FF236012184033496714661040431F4026
:103F60001E4005F0C7F9050438002E49784305F0D6
:103F7000C1F90002054330002A49704305F0BAF93F
:103F8000294B28431B68202B06D16400A40E274B25
:103F9000A400E35800021843FFF7C0FE002005B05C
:103FA000F0BD042CFAD90F2321680B40092BF5D161
:103FB000636803925B100193019B9F42EEDABB00A2
:103FC000E3189E68039B1E4228D0FF2370121840FE
:103FD00072101A401349751440431D40009205F0B9
:103FE00089F9030428000F496843029305F082F918
:103FF000029D0002054300980A49404305F07AF902
:10400000094B28431B68202B06D17600B60E074BC0
:10401000B600F55800022843FFF780FE0137CBE7D2
:10402000F00F00205906000020000020F8D3000007
:104030000200086810B5C3070FD540101823012AE5
:1040400003DD4A68042A00D10833054A1360FEF7ED
:10405000C9FFFFF745FF002010BD01204042EDE7FA
:104060002000002010B50124044002D0441020009C
:1040700010BD042810D90F2302681340042B07D168
:10408000FFF724FA21000A2207F0CAFE0400EEE737
:10409000032B01D10430F5E70D20FDF70DF9E6E71C
:1040A0000868F8B5C3071AD5FFF7DCFF0300203B0B
:1040B0005E2B25D80520434301221D180020114EF8
:1040C0009D4219D005211024F75C3C4200D0801895
:1040D0000139520064100029F7D10133F0E70428B8
:1040E0000ED90F2203681A40042A09D11B099BB27A
:1040F000002B05D00379DAE7012340001843F8BD0F
:104100000120FCE71DD2000070B508680D00FFF724
:10411000A9FF04006868FFF7A5FF621E0100042ADA
:1041200014D8451E042D11D805236B439B1801227A
:1041300015009D402B00064805682B430360054B86
:104140001B68002B02D0200002F0FBFA002070BD9B
:10415000F80F0020DC1A002070B508680D00FFF78A
:1041600081FF04006868FFF77DFF621E0100042ADA
:1041700013D8451E042D10D805236B439B1801222C
:104180009A400748036893430360064B1B68002B63
:1041900003D00022200002F0D4FA002070BDC046F7
:1041A000F80F0020DC1A0020F0B5050089B008687F
:1041B0000C00FFF757FF0690022D36DD6068FFF711
:1041C00051FF0190A068FFF74DFF04000127231D58
:1041D000661E0793731C0293079B9E4235D00523EE
:1041E00073430593019B019D05330493049BAB42EC
:1041F0001ED0042E16D86B1E042B13D80122059B4B
:104200002349013B5B199A409446224A0B68106887
:10421000069A3A4003920DD062461A430A60012280
:1042200000280DD17F000135E0E701240194CDE79E
:10423000029ECFE7624693430B600028F2D0039AB8
:104240000299280002F07DFAECE7019B1E1D042E66
:104250001AD8012C18D1002505273B0021006B43FB
:104260009B1999400B000A4A013511689943094B83
:1042700011601B68002B05D0019B0022581D2900EE
:1042800002F05FFA052DE8D1002009B0F0BDC0466C
:10429000F80F0020DC1A0020086810B5C30703D50A
:1042A000FFF7E0FE054B1860054B1B68002B03D0A1
:1042B000024B186802F046FA002010BDF80F0020EB
:1042C000DC1A00207FB5A04C2368002B0AD19F4A3E
:1042D0001268002A06D19E4B1B68002B01D0FFF705
:1042E0006BFD7FBD9B4D2A68002A26D1984A126833
:1042F000002A1BD0FFF760FD0028F2D0FFF748FD31
:10430000924B24681A681C60002A16D0002C14D125
:1043100001AD0C229049280007F014F9285D002116
:104320000134FEF73FFE0C2CF8D1DAE7874A126819
:10433000002AE5D1002BE3D0E0E700211A2003F0AA
:1043400013FB00211B2003F00FFB00211C2003F0B6
:104350000BFB2E68012E5CD0022E00D1A2E0002EB5
:1043600050D101363100794C03202368994303F082
:10437000FBFA0420216801404B42594103F0F4FA52
:10438000102123680A2019404B42594103F0ECFAEE
:1043900080212368090119404B425941062003F04E
:1043A000E3FA80212368090219404B425941072052
:1043B00003F0DAFA80212368490219404B4259413F
:1043C000092003F0D1FA80212368890219404B4269
:1043D0005941192003F0C8FA80212368C902194005
:1043E0004B425941182003F0BFFA802321681B0378
:1043F00019404B425941172003F0B6FA31001A20F8
:1044000003F0B2FA2B680321581C05F059F8296013
:1044100067E702214D4C1720236819404B42594150
:1044200003F0A2FA08212368182019404B42594191
:1044300003F09AFA80212368C90019404B42594180
:10444000042003F091FA80212368490119404B426E
:1044500059410A2003F088FA80212368C9011940D4
:104460004B425941032003F07FFA802123688903DE
:1044700019404B425941092003F076FA8023216804
:104480001B0419404B425941192003F06DFA3100C9
:10449000062003F069FA3100072003F065FA3100C5
:1044A0001B20ADE72021294C1720236819404B42DF
:1044B000594103F059FA40212368182019404B4212
:1044C000594103F051FA80212368192019404B42C9
:1044D000594103F049FA80212368490019404B42B1
:1044E0005941092003F040FA8021236889001940CE
:1044F0004B425941072003F037FA80212368890194
:1045000019404B425941062003F02EFA80212368BE
:10451000490319404B4259410A2003F025FA8021F2
:104520002368C90319404B425941032003F01CFA88
:10453000802321685B0419404B425941042003F059
:1045400013FA01211C205BE7F80F0020EC0F00207C
:10455000FC0F0020E00F002011D20000012010B558
:104560004042FFF7BDFC10BD10B5034A09210348C6
:1045700000F098FF10BDC046F8D4000040D5000000
:104580008023F0B502255B051A690A4C0A4BA12667
:104590001D5103278025F600ED00BA43884202D35F
:1045A00000221A51F0BD5F59002FFCD0985180189D
:1045B000F4E7C0460405000000E0014010B5002803
:1045C00006D1C020B02140028902FFF7D9FF10BDFB
:1045D000B02080218002C902F7E700004342584121
:1045E000064B40421840B0239B02C01803680020CD
:1045F0001A0E532A01D11B02180A704700C0FEFF91
:1046000030B501248025054B054AED009C505C59CE
:10461000002CFCD001600021995030BD00E0014029
:104620000405000043425841074B40421840B02364
:104630009B02C018A62310B50902DB05090A19431D
:10464000FFF7DEFF10BDC04600C0FEFFF0B501243D
:1046500080260D4B0D4DF6005C51002902DC002236
:104660005A51F0BD577814783F02274394782404B8
:104670002743D478043224063C439F59002FFCD0B2
:1046800010C00139E9E7C04600E001400405000020
:1046900070B505004B680A009C1C2100A400FFF7C0
:1046A000D5FF281970BD0000134B1B68002B0CD0E0
:1046B0008022B023D2029B0200280BD11A1D5B6816
:1046C0001B0E522B00D110007047B022C023920263
:1046D0005B02F1E782420DD903681B0E522B09D110
:1046E000436802339B00C018824203D903681B0E43
:1046F000522BE9D00020E7E700110020F0B50020A0
:10470000B7B00024FFF7D0FF270005002600002DDA
:104710002ED1284D2868FFF761FF32003B00019041
:104720000094254904A807F06DFA04A801F0B0F838
:10473000224B64201C682B68A0215A425341204A16
:104740005B421340B02292029B18E41A6043490274
:1047500004F0D0FDA0225202030000921949220069
:1047600004A807F04FFA04A801F092F837B0F0BDA2
:10477000FF226B6829689C460233FF180B12013632
:1047800013409C4200DA1C00FF200A1402400392EE
:104790006246014001920091039A0B4904A807F078
:1047A00031FA04A801F074F82800FFF77DFF050036
:1047B000ADE7C046001100204AD6000004110020D9
:1047C00000C0FEFFF4D5000036D6000070B5002012
:1047D000FFF704FF04000120FFF700FF844200DA26
:1047E00004000A4B1D686A42554128001D60FFF70E
:1047F000E5FEA0226B4252021340054A28009B1896
:10480000044A611C1360FFF70DFF70BD001100200A
:104810000480010004110020F8B50020FFF7DEFE3F
:1048200007000120FFF7DAFE3E00204D0643204C32
:104830000DD18021C020C9024002FFF7A1FE012155
:104840003000FFF7EFFE1B4B2E6023601DE0874218
:1048500009DD0023B0212B60164B890223602368F9
:104860000020012517E0012380212B60124BC90293
:104870002360F4E7120E522A08D0002800D02360EB
:104880000E4801F005F8FFF7A1FFF8BD28005A68AF
:10489000023292009B188B4205D21A68561CE9D14D
:1048A0000028F2D0D1E72160EFE7C04600110020D8
:1048B000041100200480010004C002000FD6000093
:1048C00070B50020FFF7F0FEFF260500002801D19B
:1048D000280070BD03681C143440FFF7E5FEDA2C95
:1048E000F4D10500F2E700008022F0B55200A1B03B
:1048F0000021674806F042FE8022002152006548F0
:1049000006F03CFE644BFF271B681A0004935342D9
:104910005A4110000592FFF751FE049C0020631ECF
:104920009C415E4B64421C405D4BE418FFF7C8FF9E
:104930000600002E2DD10498FFF750FE411C05986B
:10494000FFF770FE059A574D534B2C601A60FEF727
:1049500047FD514B64201B68A0215A4253414F4AE6
:104960005B421340B0222C6892029B18E41A604309
:10497000490204F0BFFCA0225202030000924A49FF
:10498000220007A807F03EF907A800F081FF21B038
:10499000F0BD3268131412123A403B4003921A00E1
:1049A0000A3A092A49D83A4B039A995C002931D12D
:1049B00010223E4806F0E2FD35002B6803991A12DA
:1049C0003A40914209D11A143A400B2A27D0132AAF
:1049D0002DD00A2A01D1354B1D602800FFF764FE57
:1049E000051EEAD1314B196800290FD02000FFF7CE
:1049F0004FFE04002D4B5B195968002903D020009D
:104A0000FFF746FE040004350C2DF3D1204B0121A5
:104A1000039A99543000FFF747FE060089E73B40B0
:104A2000022BDADC214A9B00D3185D60D5E7102207
:104A300000211E4806F0A2FDCFE71A00153A082A09
:104A4000E8D8144A0399525C002AE3D13500152BAB
:104A500000D01500300003681A143A40152A0FD010
:104A60001D2A00D10025FFF71FFE0028F3D1002DDD
:104A700004D020002900FFF70BFE0400054BC6E719
:104A8000039A1B123B409A42EDD10500EBE7C0466A
:104A900000100020081100200011002000C0FEFFBF
:104AA00004C0020004110020D9D50000182F0020F6
:104AB00010B5FFF719FF10BDF0B585B003920322C2
:104AC0000333DC17294D1440E4182B68284F5A4251
:104AD000534180225B42D202A4103B409B18A21C8F
:104AE0000291244E910000910190316800980A18BB
:104AF000934215D2FFF7F8FE2B685A4253418022A9
:104B00005B421F40D202BF183368009A9B189F4235
:104B100006D2194800F0BCFE0025280005B0F0BD03
:104B2000029B356819066B461A7BA423DB051343E9
:104B3000FF222F00090C1943019B12041B04134090
:104B400019432800FFF75CFD0837281D2100376056
:104B5000FFF756FD002C04D00A9A21003800FFF719
:104B600075FD009B083BFF183760D6E70011002059
:104B700000C0FEFF04110020B3D5000070B59AB04C
:104B8000FFF74AFEFF221E4CD2000021200006F053
:104B9000F5FCFF25FFF794FE0026002814D1020043
:104BA000C300E3580130591E8B41D218FF28F7D1BA
:104BB000144901A807F026F801A800F069FE124880
:104BC00000F066FE1AB070BD03681A142A400A2A63
:104BD0000AD11A122A40FF2A03D0D200A1180B7161
:104BE000A050FFF761FDD8E7132AFAD11B122B4022
:104BF000FF2BF6D0DB00E2181671E650F1E7C04655
:104C0000902500207FD6000093D600000021094B9C
:104C1000094A59600131516059680029FCD00021CE
:104C20001961012393600222044B8131FF315A50F4
:104C30001A607047FC1000400010004000E100E0E6
:104C40000222064B0121DA670022054B5A61054A10
:104C500011615A69002AFCD07047C04604E100E0A7
:104C6000FC1000400010004010B5044C2378002BCD
:104C700001D0FFF7E5FF0020207010BD09120020D1
:104C8000802301205B055B6E5B00184370470000CA
:104C90000120024B1B685B00184370478C120020F8
:104CA0000120024B1B685B00184370472400002062
:104CB0000120024B1B685B001843704790120020D4
:104CC00070B504000D001600FEF75EF98023012187
:104CD0005B055A6E2670002653006170E1706272A7
:104CE000010A5A0A6071A171A272010C5A0C000EDD
:104CF0005B0EA6702571E1712072E272237370BDA4
:104D000010B5044C200006F0C3FF01002000FEF7A0
:104D1000FDFD10BD951200200E4B10B51B680E4C0A
:104D20005A1C0FD00D4C002B0CD00D4C012B09D070
:104D30000C4C022B06D0094C042B03D00A4C052B3B
:104D400000D1074C200006F0A3FF01002000FEF771
:104D5000DDFD10BD2800002024D70000ACCF0000EE
:104D60002FD70000B3CF000029D7000070B5214C29
:104D70002278002A3DD1204B01215A608022D205A1
:104D800011605A68002AFCD0002207201B4B1C49E6
:104D900001255A500439585008315A5019481A49B7
:104DA00058501A491A485A501A495A50A622D20045
:104DB0009D50082218495A50043158500220174972
:104DC0005850174917485850174804395850182058
:104DD00016495850C12189005A500539FF39585891
:104DE000921802435A501249124A9950FFF70EFF87
:104DF000257070BD09120020FC000040001000402A
:104E00000C050000746962751C0500002405000093
:104E1000200004022C0500001405000034050000E9
:104E20003C050000FFFF00002110010054050000B8
:104E30000A1200200405000070B50E4B06001B7816
:104E4000002B01D1FFF792FF00200B4D2C788442FC
:104E50000ED00A4B202219780323091B1940084B56
:104E60004901C918300006F06DFB0120013C2C708F
:104E700070BDC046091200209412002008120020C4
:104E80000A120020002370B588B0984235DD0D6805
:104E900001262C0034409C422FD12300042D2CD914
:104EA0000F222B681A402300092A26D16A683F2A5C
:104EB00023DD6846FFF7C0FF230000281DD06B46A6
:104EC00019783300A14203DB6B461B5D5B00334363
:104ED000A200AA1801349360202CF2D10921694460
:104EE0004A780B7812021A438B781B041A43CB784A
:104EF0001B061343024A13600423180008B070BD58
:104F00009012002070B5454B8AB01B78002B01D160
:104F1000FFF72CFF02AC2000FFF78EFF002802D124
:104F200000200AB070BD23780B2BF9D96378012BD0
:104F3000F6D1E378012BF3D100231120384E394DFF
:104F400033602B7068442379374A417813600278C4
:104F500009021143827812041143C27812060A43EF
:104F600032490A60002B0ED1152169444A780B782A
:104F700012021A438B781B041A43CB781B06134387
:104F80003360002318E0012B1AD1152169444A78B7
:104F90000B7812021A438B781B041A43CB781A2120
:104FA0001B06134333600E23627C6944934200DD89
:104FB000130000229A422CD100220420EA54B0E7C8
:104FC000022B03D1627B10331621EEE7042B0DD1A7
:104FD000152108226944684606F0B4FA0098019940
:104FE00002F034FD06F060F93060CAE7052BC8D145
:104FF000152108226944684606F0A4FA0098019930
:1050000002F024FD06F050F93060627D0A231E2173
:10501000CBE7885CA8540132CCE7C04609120020D7
:105020008C120020951200202800002090120020F1
:1050300010B5134B04001B78002B01D1FFF796FE2F
:10504000FFF7FEFD00200F4A0F49104B54505860E7
:105050000130106058680028FCD000201861013031
:10506000906018690028FCD0094B0A481B785B0146
:105070001B185350FFF7E4FDFFF7C8FD10BDC046F5
:10508000091200200010004004050000FC10004040
:10509000081200200A12002010B588B000281DDD7B
:1050A0000A68012113000B4018D1042A16D90F20D9
:1050B00014682040092811D150683F280EDD98005F
:1050C000101880680024084201D04010C4B268461D
:1050D000C4540133202BF2D1FFF7AAFF002008B0FF
:1050E00010BD000010B5002813DD0C68E30710D5D3
:1050F0006410532C0DD8084B1B78002B01D1FFF7FF
:1051000035FEFFF79DFDA123044ADB00D450FFF7D5
:105110007DFD002010BDC046091200200010004097
:1051200010B500280EDD0C68E3070BD56410FF2CCA
:1051300008D8054B1B78002B01D1FFF717FE034A57
:10514000034BD450002010BD091200200010004075
:105150002405000013B5002814DD0C68E30711D501
:10516000094B64100093094B0193072C0AD8084B94
:105170001B78002B01D1FFF7F9FD6B46054A195743
:10518000054BD150002016BDE2ECF0F4F8FC000411
:1051900009120020001000400C05000070B588B016
:1051A000002820DD0124086804401CD104281AD9F5
:1051B0000F2302681340042B15D1FEF787F9060070
:1051C00006F066FD0500122800D912252A000221EA
:1051D0000D326846FFF774FD6B465D73A54205DC32
:1051E0006846FFF725FF002008B070BD2300325D40
:1051F0006B449A730134F1E7F0B50D008BB00128D0
:1052000032DD08680122040014402DD104282BD976
:105210000F2301680B40042B26D16B68134223D067
:10522000FEF754F96E6807007310019306F030FD25
:1052300005000E2800D90E252A000121113202A8EE
:10524000FFF73EFD6A46127902AB5A7302AA731247
:105250009373019B76141B0ED67313745574A54279
:1052600005DC02A8FFF7E4FE00200BB0F0BD3A5DBC
:1052700002A963189A740134F1E730B589B00028A7
:1052800014DD0C68E30711D5102268460021FFF7F2
:1052900017FD6B466A4665105D73684663122D0EF6
:1052A00064149373D4731574FFF7C2FE002009B021
:1052B00030BD0000174B184A5968002903D000215F
:1052C000596001319160196900291FD000201861CF
:1052D0008023DB00D3581149012B18D1A923DB000F
:1052E000D3585B420B600E490B78032B01D8013376
:1052F0000B7003200B490B78013303400B700A49F4
:105300005B015B18094953500123936070470860A3
:10531000FAE7C046FC1000400010004024000020C6
:1053200094120020081200200A1200200405000038
:1053300010B5034A1021034800F0B4F810BDC04670
:10534000A4D600009BD60000044A05491368C8543F
:1053500001339B059B0D13607047C046C4160020A7
:10536000C412002070B5114C114A2368834202DC3C
:105370000023236016E0155C411C2E00FA3E012E2E
:1053800005D899420FDA555C013D1F2D01D908005F
:10539000ECE70100151A565C6E5401318B42FADCC1
:1053A000181A206070BD1570FAE7C046D01A0020A8
:1053B000D016002010B5FDF7DDFD064B1A688242BD
:1053C00001D900221A601B68C31A03489842804121
:1053D000404210BDC0120020204E000010B5094C04
:1053E000094A23681268934200D110BD074AD05C75
:1053F000FDF7EEFF0028F8D0236801339B059B0DD5
:105400002360ECE7C8160020C4160020C412002058
:1054100010B50400064B074A1B6812689B1ADB4351
:105420009B059B0DA34200DB10BDFFF7D7FFF1E703
:10543000C4160020C8160020F7B505005668019173
:10544000B000441C06301700FFF7E2FFFB20FFF717
:105450007BFF1C20FFF778FFE8B2FFF775FFE0B293
:105460002412FFF771FFE0B2FFF76EFF6B46187969
:10547000FFF76AFF0025AE4200DCF7BDAB00FB186A
:105480009C680135E0B2FFF75FFF2012C0B2FFF762
:105490005BFF2014C0B2FFF757FF200EFFF754FF49
:1054A000E9E7000070B5074E33680B2B08DC0C25CC
:1054B0005D43054C0133285164196160A26033607B
:1054C00070BDC046CC160020282F002010B5FBF779
:1054D000F7FDFFF749F8FBF71BFEFDF70DFFFEF7A1
:1054E000C5FBFEF703FCFFF723FF00F023FF01F0ED
:1054F0002BF901F075FB10BD962210B512010021A9
:10550000034806F03BF80022024B1A6010BDC0466B
:10551000301C0020CC050020064B074A1B6812688F
:105520009B1ADB439B059B0D0122834200DC00227A
:1055300010007047C4160020C8160020F8B50500FA
:105540000C0016001F1E0ED10320FFF7E5FF0028F8
:1055500008D0FA20FFF7F8FEE8B2FFF7F5FEE0B258
:10556000FFF7F2FEF8BD501DFFF7D6FF0028F9D077
:10557000FB20FFF7E9FEE8B2FFF7E6FEE0B2FFF737
:10558000E3FEF0B2FFF7E0FE3012C0B2FFF7DCFE40
:105590003C00E31B9E42E5DD2078FFF7D5FE013499
:1055A000F7E7000070B50024F0250B4B1B68A34201
:1055B00002DCFFF7A1FF70BD2B006343074A9B1875
:1055C0001A78002A05D05978002311201A00FFF715
:1055D000B5FF0134E9E7C046CC050020301C0020AF
:1055E000F8B507000024F0252B0063430C4A013472
:1055F0009E18B74211D0317800290BD00133D15C0D
:10560000002311201A00FFF799FF2A000021300023
:1056100005F0B4FF0A2CE7D1F8BD024B1C60F9E796
:10562000301C0020CC050020F0B5150001222F0011
:10563000754C1740A54401900291002F11D005AB85
:105640001A706A105A70120E1A7105226912997036
:105650006D140299DD70FFF771FFCF239B009D440D
:10566000F0BD042D1ED90F202A681040042826D131
:10567000022304AA28001371FDF728FF040006F096
:1056800007FB624B984200D91800B84204DC421C68
:1056900005AB02990198DEE701377B1EE35C05AAA2
:1056A000D355F2E7042D00D0A9E0032304AA043D5A
:1056B00013716B425D4105AB55710222E9E7092880
:1056C0007ED1042205AB1A706A68511000916946B8
:1056D000521209789A70009A59701F2A01DD20220F
:1056E00000926A46127806ACDA70009BBB4202DC7C
:1056F00005ABE21ACDE70126BB00EB18986806401F
:1057000006D1042837D90F210368194002290CD18A
:10571000012323704310637042121B0E4014A270C9
:10572000E070237105340137DFE7042921D102231A
:105730002370FDF7CBFE039006F0AAFAA31C0C28F9
:1057400009D86070864201D19C19ECE7039A925DFA
:105750009A550136F6E70C226270039A925D9A55CB
:105760000136092EF9D12E23E372237363730E34AD
:10577000D9E7012907D10323043823704342584154
:1057800060700234CFE7092909D1042323704368EC
:105790005A1062705B12A370E6700434C3E70329E9
:1057A0000BD1052323700068020992B2430F9200C7
:1057B0000B40D31A63701B12EDE726700134B2E779
:1057C000032800D049E7052105AB1970110989B2FA
:1057D000520F890002408A1A111299705A701100F2
:1057E000642A00DD64210420D970C9B2041FA142DB
:1057F00001DC04324DE72C5C1C540130F6E7002D2F
:1058000000D02AE751E7C046C4FCFFFF2303000095
:1058100070B502000024F0210D4E0800604380198D
:105820004578954203D001340A2CF6D170BDF022A0
:10583000002105F0A3FE074A1368013BA34200D1F3
:105840001460002329001A001120FFF777FEEDE70E
:10585000301C0020CC05002010B5B2B002236A46EF
:105860000400137006F014FAC72800D9C7200023DB
:10587000984207DC421C6B46FE211420FFF75EFEB7
:1058800032B010BD694601335A1EA25CCA54EFE71C
:1058900030B5B3B002236A460500137006F0F8F97C
:1058A0000400C72800D9C72400239C420BDC200039
:1058B0003230FFF7ADFD621C6B46FF211420FFF76D
:1058C0003DFE33B030BD694601335A1EAA5CCA544E
:1058D000EBE70000F0B5BBB004900C00012803DC3E
:1058E0001B20FBF7E9FC51E02A4B08680293C30731
:1058F00009D4042807D90F2302681340042B02D1CE
:10590000FDF7E4FD0290234B60680393C30709D4BD
:10591000042807D90F2302681340042B02D1FDF796
:10592000D5FD039000271C4B1B680693069BBB42CA
:105930000BDC039B194A0093C821029B08A806F0C0
:105940002FF908A8FFF7A4FFCAE70C267E43144BE3
:105950000299F618306806F091F9051E05D17368B2
:10596000B6680793079B9D4201DB0137DEE730688D
:105970000399059606F082F90836002808D121001F
:105980000498059B083102385B6898473BB0F0BD2E
:105990000135E7E7B0D00000CC16002000D80000A9
:1059A000282F0020F7B5234B06001B68F021009339
:1059B0000023009A9A4211DC0024F0231A0062436B
:1059C000019201991C4A55182F78002F12D00134EA
:1059D0000A2CF3D11948FFF75BFF29E00A005A436C
:1059E000154882185078B04202D11278002A1FD18F
:1059F0000133DEE7F0223900280005F0BFFD022365
:105A00000D4A0199EB6053540D4AF1008A58009BEE
:105A10006E70AE70AA602F616F61A34202DC054B0D
:105A200001341C60002331001A001020FFF786FDAE
:105A3000F7BDC046CC050020301C002054DC00001F
:105A40009025002010B5FFF7ADFDFF24084AE300C4
:105A50005B429B18074AD35C043B012B03D8E0430D
:105A6000C0B2FFF79FFF013C002CEFD110BDC04634
:105A7000FC07000090250020F7B50F00FF247F25CC
:105A800001901E4AE300D31A1D4A9A181278062A7A
:105A900001D0032A20D1FF22D2009B181868836806
:105AA0002B401C2B18D1C3681A002A40042A13D19A
:105AB00002692A40192A0FD11B0A01339B000C30BE
:105AC000C018FDF703FD03780600002B10D006F088
:105AD000DFF80023B84209D0013C002CD1D1F7BD3A
:105AE000019AF15CD25C9142F6D101339F42F7DC1E
:105AF000E043C0B2FFF756FFEEE7C0469025002016
:105B0000FC07000070B50500FF24084AE3005B4273
:105B10009B18074AD35CAB4203D1E043C0B2FFF706
:105B200041FF013C002CF0D170BDC046FC070000D5
:105B300090250020F7B5FDF71DFA514B1A688242F7
:105B400001D900221A601A684E49821A8A4200D886
:105B500083E01860FDF718FA071E00D10137002016
:105B6000FDF704FB01900020FDF714FB019B009062
:105B7000454C464D002B14D02368002B00D07AE012
:105B80002B682760002B00D171E0414B01261B7868
:105B9000002B63D10920FFF7B5FF3E4B1E703C4B35
:105BA0001E70009B002B12D02B68002B0FD1236896
:105BB0002F60002B1ED0374B01261B78002B52D1B3
:105BC0000920FFF79FFF334B1E70314B1E70236877
:105BD000002B0FD02F4E3278002A0BD19F4200D2DB
:105BE00027602368FB1A312B04D90720FFF78AFFAF
:105BF000012333702B68002B0FD0254E3278002AFA
:105C00000BD1BB4200D92F602B68FF1A312F04D96A
:105C10000820FFF777FF012333702368002B0CD097
:105C2000019B002B09D11B4E3378002B02D107209A
:105C3000FFF768FF0023236033702B68002B0CD024
:105C4000009B002B09D1124C2378002B02D1082095
:105C5000FFF758FF00232B602370F7BD0720FFF7E5
:105C600051FF0C4B9CE70820FFF74CFFADE7009B72
:105C7000002B9CD1ABE7009A002A95D1AAE7C04639
:105C8000BC1200200F270000AC120020B41200202C
:105C9000B8120020B012002037B500240500FFF72D
:105CA00081FC01A80194FDF74FFA21002000FEF7C6
:105CB00007F9FEF707FBFDF7FBFAFDF715FBFEF70B
:105CC0004DFCFDF77DF9A54204D0FDF7ABFB024882
:105CD000FFF7DEFD37BDC04645DC000010B5FFF71D
:105CE00061FC0120FFF7D8FF0248FFF7D1FDFFF765
:105CF000A9FE10BD3ADC0000002310B501001A0017
:105D00001120FFF71BFC10BD07B56B4619706946E3
:105D10005A7013128B701314120ECB700A716B46EB
:105D2000010005221320FFF709FC07BD10B50A008A
:105D300001001220FFF778FC10BD70B505000800C7
:105D40000C003230FFF764FB2B00220000211B20E7
:105D5000FFF7F4FB70BD10B50C0003001100142018
:105D60002200FFF7EBFB10BD012370B5FF24084AAA
:105D700041185B42884201D3D84370BD06781D0AA2
:105D8000234073409B009B5801306B40F2E7C046B4
:105D90001CD8000013B50400FE2813D80A4BC2001B
:105DA000D05800280ED0436808309900FFF7DCFF78
:105DB00001900920FFF72CFB01AB042221001720E2
:105DC000FFF7BCFB13BDC04690250020F7B501903E
:105DD000FEF776FD01250400FF276D42002C01D15E
:105DE0002800FEBD266833143B40152B0DD1210041
:105DF0000198083105F042FF002801D135123D40DD
:105E00002000FEF751FC0400E8E71D2BF8D1012526
:105E10006D42F5E7F0B580279DB0FFF7DFFAA54C9E
:105E2000A54D2068FF00391A4019FDF7B7FA23681D
:105E30000600C3182360002B0ED11DB0F0BD2068F2
:105E4000391A2818FDF7AAFA236806001B182360E0
:105E5000FDF790F8994B1860002EF0DC2B78FA2BA8
:105E600000D037E12368022B07DCFFF7A3FA0028F4
:105E7000E3D00120FFF776FADFE76878AC780238E4
:105E800018282BD803F0A2F919002C003000340098
:105E9000370040002A004A007C0086008A00A000EB
:105EA000F10002012A002A002A002A002A002A0002
:105EB0002A002A002A002A001001FF2C0ED0200000
:105EC000FFF7A6FC00227E4BE100CA505B181A7156
:105ED0002100009213001320FEF7EEFD0320C9E716
:105EE0002000FFF75FFDF9E72000FFF791FCF5E7E1
:105EF000FFF7A8FDF2E7FFF755FB0020FFF7CCFE08
:105F00007048FFF7C5FCE9E7632CE7D86E4BA200A9
:105F1000D25821001520FFF787FBDFE7FEF7D0FC02
:105F2000FF270400002CD9D025682B143B40152BEB
:105F300004D02000FEF7B8FB0400F3E7200008308F
:105F400005F0A6FE06000530FFF762FAFB20FFF71A
:105F5000FBF92D121D20FFF7F7F9E8B2FFF7F4F96E
:105F6000F0B2FFF7F1F93012C0B2FFF7EDF92500FA
:105F70002B1B9E42DDDD287AFFF7E6F90135F7E7B6
:105F800000211D2000910B000A00FEF795FDFDF792
:105F900049FAA3E72000FFF7FDFE9FE7FCF7FCFFAF
:105FA00003AC4A4A64210090494B200005F0F8FDFB
:105FB00002232000237005F06BFE23000200002165
:105FC0001620FFF7BBFA89E700243D4AE300D558C5
:105FD000002D27D06B689E00701DFFF719FA2B006B
:105FE00000253200083321000120FFF7A7FA2F0017
:105FF000FEF766FC2E00002818D1002F04D03A00CE
:1060000001212000FFF718FA002D04D02A000221F8
:106010002000FFF711FA002E04D0320000212000EA
:10602000FFF70AFA0134FF2CCFD157E7FF210368AD
:106030001A120A40A24209D11A140A400B2A08D1A6
:106040000B400CD0012B0CD0022B0CD0FEF72CFBFC
:10605000D1E7132AFAD100252F002E00F6E706001B
:10606000F4E70700F2E70500F0E70024FFF79AFAEB
:106070002200210000942300DA20FEF71DFDFF22FC
:106080002100D2000E4805F079FA80E7012C02D1F8
:10609000FEF734FB22E7022C02D1FEF709FD1DE7D3
:1060A0000120FFF7F9FD19E7002321001A001A204B
:1060B00087E7C046D01A0020D0160020C01200206A
:1060C000902500201CDC0000882D002033DC00001F
:1060D0002EDC0000FB2B00D0CBE62268042A00DC7B
:1060E000C3E62E79E878574B360206439E4200DD20
:1060F000BFE6331D9A4200DCB7E6EB5CFE2B00D016
:10610000B7E66B78AC78771E1B2B61D019D8072BBC
:1061100047D0082B1CD0012B18D1FF2C16D0200003
:10612000FFF776FB6D79484AB31E009221002A00E2
:106130000A20FEF7C1FC454BE400E0501B191D711D
:1061400004E01D2B56D048D31E2B6AD0701D91E65B
:10615000632CFBD86A79022A13D0032A1BD0012AA8
:10616000F4D1E979AB79090219432B7AA4001B0415
:1061700019436B7A1B060B435B001343344AA3504D
:10618000E4E7002FE2DDB11E2F48FDF7BFFB304BE7
:10619000A400E050DAE7AB79A4005A1E93419B00BB
:1061A000ECE7632FD2DC03AD3A002A49280005F062
:1061B000C9F900232800EB55FFF708FE0028C5DBCE
:1061C000234B8000C25821001520FFF72DFABDE7B0
:1061D00039002048FFF750FCB8E7FF2CB6D06A79A9
:1061E000022AB3D818490B2000912100B31EFEF7F4
:1061F00063FCABE7632F00DD6327002303A99F4205
:106200000ADCFB430022DB173B40CB181A70152039
:1062100000917B1C2100EAE7EA185279CA54013345
:10622000EDE7012C92D1002F90DD6B79002B03D08C
:106230001C00322B00DD322464235C43064B1C60BF
:1062400084E7C046F6030000D61600209025002003
:10625000882D0020D5160020040000200122094BC3
:106260001A60094A1368002BFCD00322074B1B68F5
:10627000D8171040C018012380100638400018437A
:106280007047C04600C0004000C1004008C5004043
:106290000120704710B5064C200000F0D7FD0549DD
:1062A000200000F0FBFD0122034B1A6010BDC04628
:1062B000001B0020801A0600D41A002010B501210E
:1062C0000D20FCF76FFE01210E20FCF76BFE002174
:1062D0000F20FCF767FE044C200000F0F3FC1021B7
:1062E000200000F00BFD10BDE01A002010B504687E
:1062F0000D20E30703D56410FF2C03D91720FAF70C
:10630000DBFF10BDFFF7DAFFE1B2024800F018FD35
:106310000020F6E7E01A002010B5FFF7CFFF0021BC
:10632000034800F00DFD43000120184310BDC04696
:10633000E01A002010B5034A08210348FFF7B2F81D
:1063400010BDC0466CDC0000ACDC00000D4B70B52D
:106350001B6804000E001500002B01D1FFF79AFF07
:10636000E1B2094C200000F030FEF1B2200000F054
:1063700033FDE9B2200000F02FFD200000F090FE78
:1063800070BDC046D41A0020001B002010B50124A7
:106390000368234205D04168214202D0826822422C
:1063A00003D10D20FAF788FF10BD5810802801D9BD
:1063B0001520F7E74910FF2901D91620F2E75210FE
:1063C000FF2A01D91720EDE7FFF7C0FF0020EBE718
:1063D000F7B501221400904222DD0D682A421FD039
:1063E0001D4B15411B684C68002B01D1FFF752FF74
:1063F000E9B201272500194E3D40300000F0E5FDCF
:10640000002D0FD03C413000E1B200F0E5FC30003F
:1064100000F046FE0024A04202D02320FAF74CFFF1
:106420002000FEBD042CF2D90F2322681340092B53
:10643000EDD163685B100193019BAB42E7DDAB00DC
:10644000E3189968394204D04910C9B2300000F00D
:10645000C3FC0135F0E7C046D41A0020001B002021
:10646000154B70B51B6805000E00002B01D1FFF71E
:1064700011FF124CEDB22900200000F0A6FDF1B290
:10648000200000F0A9FC0021200000F0A9FD002858
:1064900001D0404270BD72B601222900200000F0F8
:1064A0008FFD62B6200000F088FC0028F2D02000AA
:1064B00000F088FCEEE7C046D41A0020001B002044
:1064C00010B501240368234202D04168214203D160
:1064D0000D20FAF7F1FE10BD5810802801D91520C3
:1064E000F7E74910FF2901D91620F2E7FFF7B8FFB7
:1064F00040002043EFE7000010B50D211D20FFF7FD
:10650000AFFF164C5A2809D101222A2122703D38AA
:10651000FFF71CFF0122124B1A6010BD0F2119203A
:10652000FFF79EFF332805D102235F22237020212D
:106530001A38EDE70D211E20FFF792FFC7280AD178
:10654000032300222A21A9382370FFF7FFFE1B2214
:106550002A211E20DCE700232370DBE72C0000202B
:10656000D81A0020204B10B51B680400002B01D165
:10657000FFF7C2FF1D4B1B785BB2022B0AD0032B27
:1065800029D0012B2CD121001D200124FFF768FF09
:10659000644205E0012C13D129211920FFF760FF87
:1065A0007F2801DD0138FF3803007F3301DA7F20C7
:1065B0004042C8237F21584302F09CFE604310BD37
:1065C000032C0BD12B211920FFF74AFF043CE7E7EE
:1065D0002D211920D9E721001E20D6E7052CF7D060
:1065E000012400206442E4E7D81A00202C00002097
:1065F00010B50120FFF7B6FF43000120184310BD7E
:1066000010B50320FFF7AEFF43000120184310BD73
:1066100010B50520FFF7A6FF43000120184310BD69
:10662000144B70B51B68002B02D10120FFF79AFFB5
:10663000114B1B785BB2013301D1FFF75DFF0120E5
:10664000FFF790FF04000320FFF78CFF05000520F3
:10665000FFF788FF6D43644340436419201804F03A
:1066600059FE01F023FB04F01FFE430001201843F4
:1066700070BDC046D81A00202C000020F8B50123B8
:106680001C0098422BDD0F683B4228D04E68350035
:106690001D4024D1042E22D90F2231680A40092A34
:1066A0001DD173685C10202C00DD2024144B1B6866
:1066B000002B01D1FFF7EEFD72B67F10F9B2114F3A
:1066C0002200380000F07CFC62B6A54214DA3800E3
:1066D00000F073FB002804D101246D002C4320003E
:1066E000F8BD380000F06EFB0122AB004000F3184B
:1066F00010439860AD18E8E764000125EEE7C04656
:10670000D41A0020001B0020002070470120704791
:10671000002070470020704701207047002070471C
:10672000002070470020704700207047002070470D
:1067300000207047002070470020704700207047FD
:10674000704770477047000010B5034A0E21034898
:10675000FEF7A8FE10BDC046FCDC00006CDD0000AA
:106760000378013B1F2B00D970470130F8E710B5C3
:10677000FFF7F6FF0378002B0BD00130222B11D14D
:106780000378002B03D0421C222B03D11000FFF70B
:10679000E7FF10BD5C2B03D14378002B00D0821C97
:1067A0001000EDE73A2BF2D02C2BF0D07B2B0BD145
:1067B000FFF7D6FF0378002BE9D07D2B01D1013004
:1067C000E5E7FFF7D4FFF5E720225B2B14D1FFF7B5
:1067D000C7FF0378002BDAD05D2BF0D0FFF7C7FF9F
:1067E000F7E7202BD3DD2C2BD3D0190091435D2963
:1067F000CFD0222BCDD001300378002BF1D1C6E7CA
:10680000002210B5904216D0FFF7AAFF03780422A9
:10681000222B10D0023A7B2B0DD0013A5B2B0AD0F1
:10682000190030390232092905D92D2B05D14178BB
:10683000303909290AD8100010BD0522742BFAD06E
:106840000132662BF7D001326E2BF4D0581E8341F3
:106850005A42F0E770B5FFF783FF037801222D2B32
:1068600001D18018023A00230A2502E06B4301306F
:10687000CB1801783039CCB2092CF7D95A43100023
:1068800070BDF8B50C001500FFF76AFF0378222BE6
:1068900002D000232370F8BD0D236A1E21000825B5
:1068A0000C260A279C4601300378222B02D10023B4
:1068B0000B70F0E7002BFAD0441C5C2B0BD1437813
:1068C000841C622B0ED0662B0ED06E2B0ED0722B3A
:1068D0000ED0742B0ED0002AE9DD0B70013A013185
:1068E0002000E1E72B00F6E73300F4E73B00F2E796
:1068F0006346F0E70923EEE710B50400FFF737FF22
:10690000A04202D90378202B00D910BD0138F7E747
:1069100010B5002815D00378002B13D0FFF720FF07
:106920002021037802008B4300205D2B09D010004A
:10693000FFF71DFF03782C3B5A425341C018FFF765
:106940000FFF10BD1800FCE70300002070B50C001D
:1069500081420EDD1A785B2A0BD1581CFFF700FF2D
:106960000125AC4205D0FFF7D3FF002801D0013547
:10697000F7E770BD70B50C001500002901D00023A9
:106980000B70002820D00378002B1ED0FFF7E8FE04
:10699000037806002C2B03D10130FFF7E1FE06003F
:1069A000337800207D2B0FD0844204D02A002100B0
:1069B0003000FFF766FF3000FFF7D9FE03783A2B6F
:1069C00002D10130FFF7CCFE70BD1800FCE7F0B536
:1069D0000D0004009DB02E78002E35D02E21280009
:1069E00005F03EF9071E14D0431B0193303E092EDB
:1069F00014D82800FFF72EFF01002000FFF7A4FFA6
:106A00000400002C20D0002F1ED0019B0133ED1874
:106A1000E1E7280005F03CF90190E7E723787B2BBC
:106A200011D1601C642203A9FFF7A4FF041E0BD040
:106A3000019A290003A805F032F90028E1D02000CE
:106A4000FFF795FEEEE7002420001DB0F0BD70B505
:106A5000050000200C0081421DDD2800FFF7D0FE5C
:106A60000300681C012B14D00020022B13D100223C
:106A7000681C1100FFF77EFF012C0CD0FFF748FFC8
:106A800000221100FFF776FF013CF5E7FFF740FF1A
:106A9000013C012CFAD170BDF8B5050000200C00B6
:106AA00016001F0081420DDD2800FFF7A9FE03003C
:106AB0000020022B06D1681C3A003100FFF75AFF74
:106AC000012C00D1F8BDFFF723FF3A003100FFF79A
:106AD00051FF013CF4E710B50024A04218D0FFF7A5
:106AE0003FFE03787B2B0AD1013000221100FFF713
:106AF00041FF00280CD0FFF73AFE0134F5E75B2B8D
:106B000006D10130FFF704FF002801D00134F9E776
:106B1000200010BDF8B5002816DD0D68EB0713D571
:106B20006D10013D0124FDF7CBFE0026FF276442D6
:106B300000280CD1002E21D0300005F0A9F801006A
:106B40003000FCF7E3FEF8BD01256D42EAE703687B
:106B50001A143A40152A0BD11B123B409C4200DA12
:106B60001C009D4201D106000836FDF79DFDDFE7C0
:106B70001D2AFAD1012400266442F6E701200134DF
:106B800064002043DFE7000010B508680C00FCF744
:106B90009DFCFFF71BF9002803DB6268024B8000B5
:106BA000C250002010BDC046882D002010B50868D6
:106BB000FCF78CFCFFF70AF90123002802DB024BEB
:106BC0008000C358180010BD882D002010B508683B
:106BD000FCF77CFCFFF7FAF8C043C00F800010BD43
:106BE00010B5034A04210348FEF75CFC10BDC04603
:106BF000FCDD0000F5DD000010B5FCF789FBFCF7BB
:106C000037FCFEF763FC0448FEF742FEFDF7B6FFD3
:106C1000FEF718FF10BDC0464BDE000010B5FCF7B4
:106C200081F810BD70B5002504AC24780573A94225
:106C300005D10A4B0A4A23210A4804F015FC0160D9
:106C40000949920052589B0002715B58A40083715D
:106C50006358856043710223C37170BD63DE000019
:106C6000C2DE000071DE000020DF0000037B002B8D
:106C700004D14373837303610133037370470000CE
:106C80001FB50191A02100240068C900D2B2445070
:106C9000012A10D0A24209D0032A0AD0074A835001
:106CA000074B019AC250012343501FBD02221343D8
:106CB000F4E70422FBE70622F9E7C046540500008A
:106CC0002405000010B50400FFF7D0FFA1222368BF
:106CD000A179D20099506179064A20009950217912
:106CE00004329950044B19685A689B68FFF7C8FF33
:106CF00010BDC0460C050000F41A00204BB2002B5A
:106D00000FDB80233F290FD81F290FD80F290FD859
:106D100007290FD803290FD81B060168074A8B5093
:106D2000704780239B04F8E7DB04F6E71B05F4E7D4
:106D30005B05F2E79B05F0E7DB05EEE724050000C5
:106D40000368074A99501A00FC32D1680029FCD028
:106D5000A321C90058580023C0B2D3607047C04671
:106D60001C05000007B58022074BD2051A600022DF
:106D70009A6002321A710F230C3200930349023BCE
:106D80000348FFF74FFF07BDF41A00200030004012
:106D9000E01A0020F8B505000E0017000024BC42E0
:106DA00008D02B68315D1B6828009847002801D067
:106DB0000134F4E72000F8BD704710B51C3000F036
:106DC000A9F910BD10B51C3000F096F910BD10B532
:106DD0001C3000F0A5F910BD70B5437E0D00002BEE
:106DE00001D1002070BD6430040000F0A2F9002839
:106DF000F7D12000290000F070F90120F2E700002F
:106E0000F7B50193FA23002504009B0083600D4B26
:106E10004560083303601C300F00160000F052F983
:106E20002000643000F04EF9074A2761B600B358DD
:106E300020006375019B9B009B586576A576A37522
:106E4000FEBDC04600DF000020DF00000123A022BD
:106E5000C375837D0E49C133FF33D2059B00995022
:106E6000437DC133FF339B009950CC220169094B0C
:106E70005204CA5005220169243BCA50827D01692F
:106E80000833CA500269417D034BD1507047C04658
:106E90000C060000240500000C050000A0220023C1
:106EA00010B50469D200A3500A4CA1420FD90A4C74
:106EB0008C425B4109495B420B40CD21C9045B1800
:106EC00004690749635005210369995010BDCC231B
:106ED0005B04F5E7A086010090D00300000098FD58
:106EE00024050000F7B5040000200D000193824244
:106EF00065D01600402A00D9402627001C373800EC
:106F000000F0F6F8B1232269DB00D550802201237E
:106F1000216992008B50A27E002A03D1226913625C
:106F2000226913600025731EAB4207D1019B002B21
:106F300004D0802202212369920099500122236902
:106F40001A622369FC33DA68002A02D19A6A002A9D
:106F5000F9D09A6A002A0BD1DA60A3232269DB00F8
:106F6000D1583800C9B2013500F0B7F8B542DAD3CC
:106F7000019B2269002B0FD11300FC339B6A002B6D
:106F80000AD10133A376D3612369FC33DA6C002A7A
:106F9000FCD00022DA640AE000230121A3765161CB
:106FA0001A002369FC3399680029FCD09A60236990
:106FB000FC339A6A002A01D000229A62E8B2FEBD30
:106FC00010B50123FFF78EFF10BD0300AC3310B5E1
:106FD00004001970643000F08BF80123637610BD53
:106FE0000023020070B5AC3243760D001178B12257
:106FF00004000069D20081508022216992008B50E8
:1070000022690133136222699360260064363000DE
:1070100000F080F8002812D0300000F06DF81E4B10
:107020002269D0502369FC331A6A002A02D19A6A75
:10703000002AF9D09A6A002A01D11A62E5E7236989
:107040000122002D0DD11900FC31896A002908D1D7
:10705000DA612369FC33DA6C002AFCD00022DA649E
:1070600007E05A612369FC339A68002AFCD00022A9
:107070009A6000202369FC339A6A82420BD098629E
:107080002169064A8B588B501800022B03D0181F19
:10709000431E9841033070BD1C050000C40400006D
:1070A00010B50121FFF79CFF10BD000010B51323A0
:1070B000142202490248FFF7A3FE10BD0040004021
:1070C000001B002010B540220021040004F056FAF5
:1070D000002320002364636410BD10B53F24026CBC
:1070E000531C2340446C9C4201D08154036410BD66
:1070F0000023036443647047436C026C934206D0E0
:107100003F21C25C01330B404364100070470120F3
:107110004042FBE7036C406C181A00D540307047C2
:10712000436C026C934201D0C05C70470120404226
:10713000FBE73F22036C406C01331340181A4342B3
:107140005841C0B27047000003210A4802680A4350
:107150000260094802680A4302600849084A094B6C
:107160009B1A03DD043BC858D050FBDC00F012F83A
:10717000F8F7CAFF240500405405004074E40000FD
:107180000000002064020020FEE7FEE7FEE7FEE7C5
:10719000FEE7FEE72D4B10B51A68D2B2012A0FD1D7
:1071A0002B4A126812070BD12A4AE0241168F022F8
:1071B0000800104021422DD12749096811422CD0E6
:1071C0001A68D2B2012A12D12149096809070ED1E1
:1071D000F020204909680140402908D11E4909686A
:1071E000014204D18020C121C005C90042501B6862
:1071F000DBB2012B0DD1164B1B681B0709D1154BB8
:107200001A68F0231A40A02A0FD1134A12681A42B2
:107210000ED010BD3028CFD0D2E7104A10491160EF
:107220008021104A09021160CAE7D02AF1D1ECE7A7
:107230000D4B1A68012A04D00C4A1A601A68012AF8
:10724000FCD1C0220A4B1A60E3E7C046E00F00F011
:10725000E40F00F0E80F00F0EC0F00F00405004030
:10726000DFFF07C0186C004000EC0640759300007B
:1072700014EC06400120704710B503681322DB6947
:10728000984710BD70470000054B0269D150036953
:10729000FC331A6A002AFCD0002201201A627047CF
:1072A0001C050000030010B55C331A781F231A4038
:1072B0001E3B19009140114AD167C2220421046982
:1072C0009200A150026953600269D360A02300229A
:1072D0000169DB00CA5001230169094A5B428B50F6
:1072E0000169084A8B5001690C3A8B5001690832D8
:1072F0008B501430FFF7FCFE10BDC04604E100E0E7
:107300000C0500001405000010B51430FFF702FF53
:1073100010BD10B51430FFF703FF10BD10B51430C9
:10732000FFF7EAFE10BD0000030070B55E331A7867
:107330000469724BE25003005D331A780469704BA4
:10734000E250030061331C7802696E4B012C00D0BF
:107350009EE005005F352E78A225ED005651020013
:1073600060321578A1220669D200B5500269D45066
:107370009623DB00994200D88CE096231B019942AA
:1073800000D88AE096235B01994200D888E09623D2
:107390009B01994200D885E0E1239B01994200D8E6
:1073A00082E09623DB01994200D880E0E123DB01F3
:1073B000994200D87DE096231B02994200D87AE0DA
:1073C000E1231B02994200D877E096235B029942A1
:1073D00000D874E0E1235B02994200D871E0E12318
:1073E0009B02994200D86EE0474B994200D86CE06E
:1073F000E123DB02994200D86AE0E1220023120374
:107400008A425B41414A5B421340802252059B18ED
:1074100001693F4A8B50A02304220169DB00CA5056
:1074200000210369FC33D9600369FC33196201232D
:1074300001690B6001698B60C12104698900625098
:107440001F215C3002780A4093406231314AFF319B
:1074500053500021415600293CDA0F230B40083BD2
:107460002D4C9B089B001B1903242140A140FC3498
:107470008C40DD69A5432C00C0258D4029002143A7
:10748000D9611F23017819401E3B8B40136070BDEA
:1074900000246CE79E23DB02BAE79D231B03B7E7BA
:1074A0001E4BB5E71E4BB3E7EC239B03B0E71D4B28
:1074B000AEE71D4BACE71D4BAAE71D4BA8E71D4BE4
:1074C000A6E71D4BA4E71D4BA2E78023DB049FE743
:1074D0001B4B9DE78C080F4BA400E41803230B40C3
:1074E000FF21C025DB009940AD0066598E43310075
:1074F000C0269E4033000B436351C2E70C050000D9
:10750000140500006C05000090D0030000D0BEFE02
:107510002405000000E100E000ED00E000B01300F1
:107520000050270000A04E0000F0750000509D00A4
:1075300000F0EB0000903A0100E0D70100B0AF038B
:1075400000705F07F7B5009308AB1B780025019327
:10755000FA2304009B0083600E4B456008330360F0
:1075600014300F001600FFF7ADFD23005C332761D8
:107570001E70009B084A9B00995823005D331970C8
:10758000019B20009B009A5823005E33DD701A7027
:10759000FEBDC046A4DF000020DF0000036910B577
:1075A0001A00FC32D2680400002A0AD0A322D200BA
:1075B00099581430C9B2FFF790FD00222369FC33BB
:1075C000DA6010BD10B50248FFF7E8FF10BDC046F5
:1075D000B81B0020162307B5022200930249013B85
:1075E0000248FFF7AFFF07BD00200040B81B002096
:1075F00010B5002801D004F07DFA10BD70470000DE
:1076000010B500F011F8FFF7F9FF012000F000FAC3
:10761000FFF7F2FAFFF702FB024B002BFAD000E073
:1076200000BFF7E700000000C420114B80001A588B
:1076300010491140C02212020A431A50C021802270
:10764000490092025A501A608023A3220021DB05D0
:10765000D20099500122F9309A60074BFF3019503F
:10766000C120023180001950403019501A60704713
:1076700000E100E0FF00FFFF00100140014B186037
:107680007047C04678000020F7B5002320285AD85C
:10769000384B8000C258042A5BD007D8022A54D045
:1076A00055D80423012A09D000234CE0062A54D0DF
:1076B00051D31A2A53D002231B2AF5D12E4A11681E
:1076C00008294ED909294FD00A240226A0200125D5
:1076D0002A4AC00015502A482A4D07681C20BF00BE
:1076E00007402948019700685759009027481B0216
:1076F00007401F43C02300989B020340FF205751BF
:107700005759000207401F43019B1F43009B58012C
:107710006023184007433E43565101251C4B15601A
:1077200058680028FCD000205860A1230125DB0008
:10773000D3585560A025ED0050511BB2A14202D094
:1077400015D2611ACB401800FEBD0823B6E71023FE
:10775000B4E72023B2E74023B0E78023AEE701235C
:10776000ACE708240026B1E70C000126AEE7091BB0
:107770008B40E8E720DF000074000020007000402C
:10778000300000200405000034000020FF00FFFF4F
:10779000FC700040F0B520285BD8364B8000C25802
:1077A000354B1E68002E30D1C227344BBF00D8594C
:1077B000334C03250440C02000022043D851C0248C
:1077C00080206400800018512E4F18602E4B803CA2
:1077D000D859FF3CA043D8510437D859A843204377
:1077E000D8510837D8590C35A84384460720654638
:1077F0002843D851A820C0001E50C12080268000F8
:1078000076021E501C601C4B1C60142500202B00AF
:107810001E4C2E0046433659771C1BD14343E25081
:10782000A0230325C132FF329200DB05D550184B4F
:107830001A68082A14D114234343E3189A6812489B
:107840005132FF32920059601150DA68C1239B0017
:10785000C250F0BD9642E1D001300328D9D1F8E7FB
:10786000082A02D9083AD140E5E708239A1A91403C
:10787000E1E7C04620DF00001C1C002000E100E022
:10788000FF00FFFF040500000090004038000020CA
:10789000780000202149F0B54A6C2148002A14D014
:1078A000A025A12600230124ED05F600C258571C8F
:1078B00006D0C7187F68002F02D027009740AF512D
:1078C00014333C2BF2D100234B64A0230121DB05B0
:1078D00000260F009C4614234B43C3181A1F12683E
:1078E000104C0E4D920014195219526C002A10D0EF
:1078F0001A00143A1268551C09D0103B1B68FF2B64
:1079000005D03B00934065461A00074BEA50FC3413
:10791000666401310429DED1F0BDC046FC90004010
:1079200038000020009000400C05000000B5202821
:1079300010D80C4A8000835803290BD8A0220800D5
:10794000C133FF33D2059B0001F036FC0209050765
:107950000021D15000BD0C21FBE70421F9E70321F0
:10796000F7E7C04620DF000020280AD8074B800038
:10797000C25801239340A022D205002902D1044914
:1079800053507047A121C900FAE7C04620DF00002C
:107990000C05000003000020202B0AD8A021A22201
:1079A000C905D2008858034A9B009B58D840012340
:1079B0001840704720DF0000F7B506000D000C00EE
:1079C0008B180193019B671B9C4207D03368217879
:1079D0001B683000984701340028F3D13800FEBD01
:1079E0000849094A094B10B51B688858FA22190A38
:1079F0001B0618439200002301F0B4FD4904C00B9C
:107A0000084310BD0010014004050000201C0020A8
:107A100070B5041E09D0FFF7E3FF050000F014F86D
:107A2000FFF7DEFF401BA042F8D370BD0022044BDD
:107A30009A60044A13680133DBB213607047C04692
:107A4000FC100140201C002070470000F0B5C64625
:107A500000B5CB0F9846404A4B005B0D9A1882B098
:107A60000D000400132A2FDC002A49DB3B4F17418D
:107A70003E000E40064323D07F08390029400C43C6
:107A80000AD03749BD438C4663445C425C41802345
:107A9000DB021341E4071D434146CE0031492B0070
:107AA0008E192200346875682000290001F000FF5B
:107AB000009001910098019922002B0003F090F8AA
:107AC00002B004BC9046F0BD332A08DD8023DB0001
:107AD0009A42F5D102000B0001F0EAFEF0E7224ADB
:107AE0009446012263445242DA400242E8D05208EE
:107AF0000242D1D094438022D2051A411443CBE7ED
:107B00004B005B080343DBD00B031B0B1C4363429E
:107B1000234380244D0C24031B0B23406D042B4373
:107B200019004346DA000F4B9B181C685D68020081
:107B30000B002000290001F0BBFE0090019100988D
:107B4000019922002B0003F04BF842464B005B08E2
:107B5000D60733431900B3E701FCFFFFFFFF0F0017
:107B6000EEFBFFFFD8DF0000EDFBFFFFF8B5274A73
:107B70004B005B0D9A180C000700132A10DC002A3A
:107B800036DB234B13410B423AD0802424031441AB
:107B9000002064189C430600250030002900F8BD31
:107BA000332A0EDD80230600DB000D009A42F4D15B
:107BB00002000B003800210001F07AFE06000D00E3
:107BC000EBE7144D0600AC46012563446D42DD40F1
:107BD000AC4663460D000342DFD033239A1A323B92
:107BE00093401818874200D94C1C63469843D2E74B
:107BF000C90FCC070020531CCDD1074B1C43CAE74B
:107C000006000D000028C0D1C7E7C04601FCFFFFF9
:107C1000FFFF0F00EDFBFFFF0000F03F30B5214AF2
:107C20004B0087B05B0893421EDD1F4A934205DD7F
:107C300002000B0002F0D4FF07B030BD02AA00F032
:107C400095F803231840049A059B012813D00228B5
:107C50001DD0002814D00298039900F06FFB8023F8
:107C60001B069C466144E7E70023002200930023A3
:107C700001F0DEF8E0E70298039900F05FFBDBE734
:107C8000012402980399009401F0D2F8D4E701246A
:107C900002980399009401F0CBF880231B069C46C0
:107CA0006144C9E7FB21E93FFFFFEF7FF0B547469D
:107CB000CE4680B58DB004000D0000F067FA294B68
:107CC00006001B780F005BB29846013310D02200EB
:107CD0002B002000290003F0CBFA8146002807D1B1
:107CE000002200232000290001F014FC002806D106
:107CF000300039000DB00CBC90469946F0BD012310
:107D00000293194B0694079503934B460A934346F7
:107D100004940595002B15D00023002219001000B3
:107D200002F0E2F8434608900991022B0ED103F0CD
:107D3000B9FB212303600A9B0193002B0CD1089E01
:107D4000099FD5E7002300240893099402A801F0B5
:107D5000C1F90028EFD1EAE703F0A4FB0A9B0193E5
:107D60000360ECE77C000020E8DF0000F0B54E4641
:107D70004546DE465746E0B5E14B4C008FB0904695
:107D8000894664089C4200DC87E0DE4B9C4222DC92
:107D9000DD4A002900DC92E0DC4B02F021FFDB4BE6
:107DA00006000F009C4200D17EE1D94AD94B02F077
:107DB00017FF02000B00414630000A604B6039009B
:107DC00002F00EFFD34BD24A02F00AFF43460125D0
:107DD0009860D9606BE0D04B9C4200DC8FE0CF4BC9
:107DE0009C4200DD55E1CE4A231592469A44514605
:107DF0000905631A19001D00040003F055FA03F089
:107E000089FA02000B00200029000892099302F071
:107E1000E7FE0022C34B02F071FC0F00060003F0E6
:107E200043FA03F077FA04000D0002000B00300063
:107E300039000A940B9502F0D3FE0022B94B02F0F0
:107E40005DFC002200230C900D9101F05DFB0028E9
:107E500000D192E1002300222000290001F054FB10
:107E6000434243410133B04A41460192022208A8ED
:107E70000092524600F07CFB4B460500002B16DAC0
:107E8000802243461206944642465B68454263445C
:107E90005360D3686344D36009E00B00020041469D
:107EA0000A604B600022002300258A60CB60280016
:107EB0000FB03CBC90469946A246AB46F0BD934BF2
:107EC00001F0F6FC914B06000F009C4200D13DE111
:107ED0008F4A904B01F0ECFC02000B004146300051
:107EE0000A604B60390002F07BFE894A894B01F041
:107EF000DFFC012543466D429860D960D7E701F069
:107F000049F88A4A8A4B06000F0002F0F7FB00226C
:107F1000884B01F0CDFC03F0C7F9050003F0FAF936
:107F2000794A7A4B0490059102F0E8FB02000B00BD
:107F30003000390002F054FE754A06000F00049824
:107F40000599744B02F0DAFB029003911F2D00DCBF
:107F5000C7E0029A039B3000390002F041FE8346DD
:107F60008A4653465B0024155B0DE31A102B6CDD2B
:107F700004980599D322674B520502F0BFFB02001B
:107F80000B00300039000292039302F029FE0A0030
:107F9000010013000691079202003900300002F040
:107FA0001FFE029A039B02F01BFE06000F000498BE
:107FB0000599614A614B02F0A1FB32003B0002F0DF
:107FC0000FFE069E079F0B00020039003000029250
:107FD000039302F005FE4B005B0D83468A46E41ACC
:107FE000312C32DD04980599B822544B920502F0E9
:107FF00085FB03000C000200029303940B0006981B
:10800000079902F0EDFD02000B0006000F00069834
:10801000079902F0E5FD029A039B02F0E1FD484A50
:108020000290039104980599464B02F067FB029A6F
:10803000039B02F0D5FD02000B00300039000292D4
:10804000039302F0CDFD83468A465A465346414685
:1080500030000A604B60390002F0C2FD029A039BB7
:1080600002F0BEFD44460B000200A260E3604B46F6
:10807000002B00DB1BE75B46236080231B06534479
:10808000636080231B069C466144A060E1606D42F2
:108090000DE70B00020002F0A3FD434600259860A7
:1080A000D9601860596002E7D3221A4B520502F0DA
:1080B00097FD214A214B0D00040002F091FD0200C2
:1080C0000B00414620000A604B60290002F088FD49
:1080D0001A4B194A02F084FD434601259860D96085
:1080E000E5E602000B003000390002F079FD6B1E5E
:1080F000154A9B009B5883468A46A342A5D130E788
:10810000FB21E93F7BD9024000004054FB21F93FAD
:108110003163621A61B4D03DFB213941FFFFEF7F2B
:10812000EAFBFFFF0000704170E0000083C8C96DEA
:10813000305FE43F0000E03F7370032E8A19A33BD9
:10814000C14920259A837B39F0DF0000D3220C4BF4
:10815000520501F0ADFB0B4A0B4B04000D0001F082
:10816000A7FB02000B00414620000A604B6029007B
:1081700002F036FD034A044BB9E6032373E6C0461A
:1081800061B4D03D7370032E8A19A33BF8B54746FE
:10819000CE46674B80B50A000F0019000500394034
:1081A000994200D19BE004000100002F69DD3F15DA
:1081B00000D1B4E05F4B12039C468023120B5B039B
:1081C00013435B00CA0F67449B184A00F80703D5A6
:1081D000D20F5B009B188A0079108C46002180200A
:1081E0001624894680030D189D4202DC29185B1B6A
:1081F0008144D50F5B00013C5B1952004008002C04
:10820000F1D100208046802020250027000609E0CB
:108210008B425CD0D40F5B00013DE3185200400854
:10822000002D16D0C4198B42F2DD27180E00002C49
:1082300049DB5B1AA242894149425B1A121BD40FE7
:108240005B00013D80443100E31852004008002DDE
:10825000E8D113434ED143465B0837494A46884626
:10826000494652104244C90702D5802109060B43F2
:1082700061460F05BD18180029000CBC90469946B0
:10828000F8BD7B005B0803433900002BF5D0002FBD
:108290003CD1E30A153A6405002BFAD08020400354
:1082A00003423FD1002700E00F005B00791C03422E
:1082B000FAD0250020208D40401A2900D71B22002B
:1082C000C2401A4376E7FE43F60F8E19B1E7944297
:1082D000A0D82718002CF6DB1E000023AEE7020012
:1082E0003B002800390002F009FA2A003B0001F0A7
:1082F000DFFAC2E74346013303D0434601335B084C
:10830000ABE7012398460023C144A6E73B000200E7
:1083100002F066FC02000B0001F0E6FDADE7130081
:108320000022BBE70127210020207F42C6E7C0468C
:108330000000F07F01FCFFFF0000E03FF0B5474682
:10834000CE4680B587B000920193754B4F008146B1
:1083500088467F089F4263DC02F0A6FF002800D118
:10836000D4E04A4643464846414602F0C7F9040075
:108370000D006C4A6C4B02F0C1F96C4A6C4B01F079
:1083800097FA22002B0002F0B9F96A4A6A4B02F010
:1083900027FC22002B0002F0B1F9684A684B01F07B
:1083A00087FA22002B0002F0A9F9664A664B02F018
:1083B00017FC22002B0002F0A1F9644A644B01F083
:1083C00077FA22002B0002F099F902900391002223
:1083D000604B2000290002F091F9029A039B0600ED
:1083E0000F002000290002F089F9009A019B040087
:1083F0000D004846414602F081F902000B002000C2
:10840000290002F0EDFB02000B003000390002F001
:10841000E7FB02000B0000204F4902F0E1FB70E097
:1084200002000B0002F06AF904000D003D4A3E4BC9
:1084300002F064F93D4A3E4B01F03AFA22002B006B
:1084400002F05CF93B4A3C4B02F0CAFB22002B00D5
:1084500002F054F9394A3A4B01F02AFA22002B0073
:1084600002F04CF9374A384B02F0BAFB22002B00DD
:1084700002F044F9354A364B01F01AFA2B0022007B
:1084800002F03CF9354B029003919F429FDD344B43
:1084900000229F423DDC334900207B182E49160004
:1084A0001F0002F09DFB049005910022294B200043
:1084B000290002F023F932003B0002F091FB029AFE
:1084C000039B06000F002000290002F017F9009A14
:1084D000019B04000D004846414602F00FF90200DE
:1084E0000B002000290002F07BFB02000B00300093
:1084F000390002F075FB02000B000498059902F0A8
:108500006FFB07B00CBC90469946F0BD00201249A5
:10851000F7E7154B002604920593144FC5E7C046B4
:10852000FFFF3F3ED43888BEE9FAA8BDC4B1B4BD50
:108530009EEE213EAD529C804F7E923E9015CB190F
:10854000A001FA3E7751C1166CC1563F4C555555A6
:108550005555A53F0000E03F0000F03F3233D33FC8
:108560000000E93F0000E0FF0000E73F0000D23FCD
:10857000F0B5DE464E4645465746E0B5DC4CA544D0
:108580000D9114001900A49A0993DA4B9200D65861
:108590004D1E03901821E01E0696029500F0AAFEDB
:1085A000C3430100DB1719404B1C9A009B1ADB00E8
:1085B0001B190B9105934C1B771918D4A59BA5008B
:1085C0009C463F1922AE6544013707E0286802F057
:1085D000A1FE013403C60435BC4208D0002CF5DAF4
:1085E00000200021013403C60435BC42F6D1069BAD
:1085F000002B01DA00F0FDFB069B03990133DB0041
:108600009A46099BDA00944600920022914672AA8B
:108610000492B94A6144934688469AAB63449B44AA
:10862000029B002B00DABCE15D4600260027039C7C
:108630004D442A686B6803CC02F060F802000B001E
:108640003000390001F034F9083D06000F004445C0
:10865000EFD1049B4B441E605F6008239C46E144BD
:10866000D145DDD10EA804218446494261448C469F
:10867000069A93009C44614684460A910399083BFC
:1086800063448C460C93009B009263449B46009A83
:108690000498D10003008C46634408911E685F680B
:1086A000002A33DD954980468C466244D3009844C5
:1086B00070AB9A460EAB99460022914B30003900C0
:1086C00002F01CF802F0F0FD02F024FE00228D4BB7
:1086D00004000D0002F012F802000B003000390017
:1086E00002F07EFA02F0E0FD4B4601C39946434694
:1086F00020001A685B68290001F0DAF808235B4261
:108700009C46E04406000F00D045D5D1059B3000C3
:108710001A003900984600F0DFFCFF2300229B0579
:1087200004000D0001F0EAFF00F038FC0022764B57
:1087300001F0E4FF02000B002000290002F050FAD3
:108740000D00040002F0B0FD814602F0E3FD0200DE
:108750000B002000290002F043FA060040460F00FB
:10876000002800DCEEE0009B18215A1E92000EABA0
:108770009B58091A1D000D41A9448D405D1B0EAB8D
:108780009D5017231B1A1D41002D2DDD01239C46F2
:10879000009BE144002B00DC1CE20E9C0123002C1A
:1087A00000D0B5E0009A012A09D099000EAA5458C9
:1087B0000133002C00D0ACE0009A9A42F5D1059B21
:1087C000002B0EDD012B00D1A8E1022B09D1009B6B
:1087D0000EA95A1E92000EAB9B5807939B029B0A50
:1087E0008B50022D00D1C1E000230022300039005F
:1087F00000F08AFE009B002800D194E2069A591EE0
:108800008A4210DC414A0A9894460EAA6344944670
:1088100000229B0063441C68043B22438342FAD13C
:10882000002A00D0C0E0069B0EAA013B9B00D35853
:10883000002B00D0B3E001220C9B043B59680132AD
:108840000029FAD0009B9C466244110007921A004E
:1088500001338B4246DC0B9863468046A59C43441B
:10886000A046099C9B00A1464A449844D30022AAF2
:108870009146049A99449446089BA59A6344844679
:10888000614494469A468B0063440093434658687B
:1088900002F040FD4B4618605960029B002B24DB20
:1088A0004D46039C0026002701E0286869680CCC2F
:1088B00001F024FF02000B003000390000F0F8FF47
:1088C000083D06000F005C45EFD153469E60DF6017
:1088D00004239C460433E0449C46009BE144E2446C
:1088E0009845D3D1079B0093D1E600260027ECE7FB
:1088F00094FDFFFFB8E1000018FEFFFFFFFFFF1F20
:108900000000703E0000704100002040FFFFFF3F6C
:10891000002180225204141B0EAA5450009999423F
:108920000EDD0EA884469B000EAA8900D258614431
:108930006344CF4800E01A68821A04C38B42FAD11C
:1089400001243CE7059B002B06D1009B0EAA013BAE
:108950009B00D558ED1517E70022C64B300000F0FC
:10896000F7FD002800D024E100253DE732003B0060
:108970000020C14902F034F906000F00002C00D19C
:1089800032E7059A0020BC4900F0A6FB02000B006C
:108990003000390002F024F906000F0024E701221C
:1089A00050E70026002754E64B46059A0793884671
:1089B0008B000EA9CB58183A08950592002B0DD1C3
:1089C0008C464146AD4B43449B006344043B58688E
:1089D0000139183A0028F9D088460592059A0020F6
:1089E000A54900F079FB434604000D00002B00DA96
:1089F00005E29E000EAB9C464346DB0066449C4667
:108A0000059370AB9946049F67440097306802F065
:108A100081FC22002B0001F071FE00223860796099
:108A2000974B2000290001F069FE083F04000D006B
:108A3000043EB945EAD14AAB03939B4600239A46CC
:108A4000069B4246994643460132029204934B46A6
:108A5000002B00DAAAE080208A4B009D9846C005D2
:108A6000894900260027002408E008239C46083591
:108A7000E044544511DC4346186859682A686B681D
:108A800001F03CFE02000B003000390000F010FF46
:108A9000013406000F00A145E7DA5B46C0C39B46E0
:108AA00001239C46009BE244083B0093029B9A45AD
:108AB000CDD1049B9846A49B022B00DD8EE0002BB9
:108AC00037DC1FD1059B00271D00039B00249C461B
:108AD0001E006544083E2A686B683800210000F0DB
:108AE000E7FE083D07000C00AE42F4D1089B002BC6
:108AF00003D080231B069C4664443A0023000D9952
:108B00000A604B600720079B18409B239B009D44F5
:108B10003CBC90469946A246AB46F0BD009B0EA9D0
:108B20005A1E92000EAB9B5807935B025B0A8B5058
:108B300057E64346002B00DA70E100200021DB00FD
:108B40004AAAD61848AF32687368083E00F0B0FEF3
:108B5000B742F8D1089B002B00D025E10B000200A2
:108B60004A984B990D9C2260636002F039F84346A5
:108B700007000C00002B13DD01254CAEB146380078
:108B80002E0021004C4601360CCC00F091FEA1468F
:108B9000B045F7DA089B07000C00002B00D015E168
:108BA0003A0023000D998A60CB60ABE700260027CE
:108BB00073E701239C46009BE1440225002B00DD66
:108BC000EBE532003B0000202B4902F009F80600DB
:108BD0000F0009E60024F2E54AAB0393A49B032BA4
:108BE00000D08FE74346002B00DC14E1039ADB0042
:108BF0009B46130091465B441E685F68234B4344C9
:108C00000293DB00994448AB9A464B465C681B686C
:108C10001800210032003B000090019100F048FE56
:108C200004000D0002000B000098019901F0D8FF2C
:108C30003B00320000F03CFE4B469860D9601C605F
:108C40005D6008235B429C46E14426002F00CA4534
:108C5000DBD14346012B00DCE3E0039A13005B44C5
:108C60001E685F68029BDB0099464A44904610E00C
:108C7000FFFFFF000000E03F0000F03FFFFFFF3F6D
:108C80000000703E78E10000FB21F93FFFFFFF1F6D
:108C9000984643465C681B681800210032003B0080
:108CA0000090019100F004FE04000D0002000B0092
:108CB0000098019901F094FF32003B0000F0F8FDAC
:108CC0004346039A9860D9601C605D60083B2600AB
:108CD0002F009A42DCD14D46944600260024474698
:108CE000083565442A686B683000210000F0E0FD1B
:108CF000083D06000C00AF42F4D1039B4A9F5D681B
:108D00009968D868089B002B65D08022120694468B
:108D10000D9B6544604464441F605D609960D86049
:108D20001E615C61EEE69A464B460793059B300058
:108D30005A423900089500F0CFF900223A4B06005C
:108D40000F0000F005FC002824D0384B0022300032
:108D5000390001F0D3FC02F0A7FA52460400950056
:108D600002F0D8FA0022304B01F0C8FC02000B00E0
:108D70003000390001F034FF02F096FA0EAA50518B
:108D80000122059B524418339046059393000EAA86
:108D9000D45023E65346300039009C0002F084FA98
:108DA0000EAB1851D04619E680230D9A1B06CB183E
:108DB000106053600B0002004A984B9901F010FFBD
:108DC000434607000C00002B00DDD5E680231B0680
:108DD0009C466444E4E62B003A000D9D2A606B60DB
:108DE0000A000300AA60EB60320023002A616B6175
:108DF00088E6099BDB00009372AB049332E4A49BEA
:108E0000022B00DDE8E6002B00DD92E600D079E6DB
:108E1000002700246AE6002600246EE700200021D7
:108E200098E60026340068E7000070410000703EBC
:108E3000F0B5CE46474680B587B000920193474AC9
:108E40004B00814688465B08934207DC4146484612
:108E500002F02AFA4146031E484666D04A46434677
:108E60004846414601F04AFC04000D0002000B0098
:108E70004846414601F042FC394A3A4B06000F0091
:108E80002000290001F03AFC374A384B01F0A8FED7
:108E900022002B0001F032FC354A364B00F008FD71
:108EA00022002B0001F02AFC334A344B01F098FEDB
:108EB00022002B0001F022FC314B324A00F0F8FC7A
:108EC0000E9B02900391002B34D000980199002250
:108ED0002D4B01F013FC029A039B04900591300086
:108EE000390001F00BFC02000B000498059901F019
:108EF00077FE22002B0001F001FC009A019B01F09B
:108F00006FFE224A04000D00214B3000390001F0B1
:108F1000F5FB02000B002000290000F0C9FC020054
:108F20000B004846414601F05BFE07B00CBC904682
:108F30009946F0BD02000B002000290001F0DEFB85
:108F4000124A134B01F04CFE32003B0001F0D6FBFD
:108F50004A46434600F0ACFCE7E7C046FFFF3F3E11
:108F60007CD5CF5A3AD9E53DEB9C2B8AE6E55A3EB3
:108F70007DFEB157E31DC73ED561C119A0012A3F4F
:108F80001111813FA6F810110000E03F49555555D9
:108F90005555C53F49004B0819007047474AF0B581
:108FA0004F4691464B005B0D99444646D6464A468D
:108FB000C0B505000C000E0088460700132A27DC08
:108FC000002A4BDB3E4B13419A460B00524613409E
:108FD000034318D03B4A3C4B2800210000F068FCBA
:108FE0000022002300F0AAFA002847D0002C04DA5F
:108FF00080234A465B031341984446465346002764
:109000009E43380031001CBC90469946A246F0BDF4
:10901000332A08DD8023DB009945F4D102000B00E0
:1090200000F046FCEFE7294A94460122634452428D
:10903000DA4092460242E6D0224A234B2800210021
:1090400000F036FC0022002300F078FA002815D04A
:10905000002C1EDB534646469F430FE0194A1A4B2D
:109060002800210000F024FC0022002300F066FA12
:10907000002803D0002C04DB002700263800310034
:10908000C1E76400640825430027002DF6D0104E88
:10909000F4E74B46142B0BD03422D21A0123934011
:1090A0005D19BD4208D201239C462F00E044D1E760
:1090B000133B9C46E044CDE72F00CBE701FCFFFFCC
:1090C000FFFF0F009C7500883CE4377EEDFBFFFF3F
:1090D0000000F0BF002070474B0070B55B0D14001E
:1090E0000A00002B1AD14B005B08034315D0234B19
:1090F000002201F003FB224B9C422DDB0A004B00B7
:109100005B0D363B1F4DE318AB422ADC002B0DDD17
:109110001D4C1B0522401A43110070BD1B4DAB4274
:10912000F0D102000B0000F0C3FBF6E71D0035355F
:1091300019DA174B02009C4209DD0B00154816494D
:1091400000F032F8134A144B01F0D8FAE5E70B00AF
:109150001248134900F028F8104A114B01F0CEFADA
:10916000DBE70200E9E7084C363322401B051343D6
:10917000190000220B4B01F0C1FACEE7000050436A
:10918000B03CFFFFFE070000FFFF0F80FF0700005D
:1091900050C300009C7500883CE4377E59F3F8C248
:1091A0001F6EA5010000903C30B54A00DB0FDB07C5
:1091B00052081A43110030BD02B4714649084900F3
:1091C000095C49008E4402BC7047C04603B4714636
:1091D000490840004900095A49008E4403BC7047C1
:1091E000002243088B4274D303098B425FD3030AE6
:1091F0008B4244D3030B8B4228D3030C8B420DD3F9
:10920000FF22090212BA030C8B4202D31212090286
:1092100065D0030B8B4219D300E0090AC30B8B42C4
:1092200001D3CB03C01A5241830B8B4201D38B0372
:10923000C01A5241430B8B4201D34B03C01A524117
:10924000030B8B4201D30B03C01A5241C30A8B425A
:1092500001D3CB02C01A5241830A8B4201D38B0245
:10926000C01A5241430A8B4201D34B02C01A5241E9
:10927000030A8B4201D30B02C01A5241CDD2C3095B
:109280008B4201D3CB01C01A524183098B4201D3D7
:109290008B01C01A524143098B4201D34B01C01AC2
:1092A000524103098B4201D30B01C01A5241C3083A
:1092B0008B4201D3CB00C01A524183088B4201D3A9
:1092C0008B00C01A524143088B4201D34B00C01A95
:1092D0005241411A00D20146524110467047FFE701
:1092E00001B5002000F0F0F802BDC0460029F7D01B
:1092F00076E7704703460B437FD4002243088B4236
:1093000074D303098B425FD3030A8B4244D3030B0C
:109310008B4228D3030C8B420DD3FF22090212BAD1
:10932000030C8B4202D31212090265D0030B8B424D
:1093300019D300E0090AC30B8B4201D3CB03C01A37
:109340005241830B8B4201D38B03C01A5241430B12
:109350008B4201D34B03C01A5241030B8B4201D302
:109360000B03C01A5241C30A8B4201D3CB02C01A6D
:109370005241830A8B4201D38B02C01A5241430AE5
:109380008B4201D34B02C01A5241030A8B4201D3D4
:109390000B02C01A5241CDD2C3098B4201D3CB017B
:1093A000C01A524183098B4201D38B01C01A52412A
:1093B00043098B4201D34B01C01A524103098B422E
:1093C00001D30B01C01A5241C3088B4201D3CB0019
:1093D000C01A524183088B4201D38B00C01A5241FC
:1093E00043088B4201D34B00C01A5241411A00D2AC
:1093F00001465241104670475DE0CA0F00D0494215
:10940000031000D34042534000229C4603098B4284
:109410002DD3030A8B4212D3FC22890112BA030A0C
:109420008B420CD3890192118B4208D3890192118E
:109430008B4204D389013AD0921100E08909C30913
:109440008B4201D3CB01C01A524183098B4201D315
:109450008B01C01A524143098B4201D34B01C01A00
:10946000524103098B4201D30B01C01A5241C30878
:109470008B4201D3CB00C01A524183088B4201D3E7
:109480008B00C01A5241D9D243088B4201D34B0002
:10949000C01A5241411A00D20146634652415B1044
:1094A000104601D34042002B00D549427047634625
:1094B0005B1000D3404201B5002000F005F802BD6A
:1094C0000029F8D016E770477047C046D0400B1C03
:1094D0001141203A03D49C4613411843634652423B
:1094E000934018437047C0468446101C62468C4621
:1094F000191C634600E0C0461FB501F097F800282C
:1095000001D40021C8421FBD10B500F0EFFF40425A
:10951000013010BD10B501F089F8002801DB0020F2
:1095200010BD012010BDC04610B501F07FF8002825
:1095300001DD002010BD012010BDC04610B501F0B6
:1095400011F8002801DC002010BD012010BDC0462C
:1095500010B501F007F8002801DA002010BD012045
:1095600010BDC046F0B5CE46474615042D0C2E0062
:1095700080B50704140C3F0C9946030C7E435D43F1
:10958000674363437F19340CE4199C46A54203D911
:1095900080235B029846C4444B4643435143250C09
:1095A00036046544360C2404A4195B1959182000AC
:1095B0000CBC90469946F0BDF0B54E465746454620
:1095C000DE46E0B543025B0A450083B00F1C9946B6
:1095D0002D0EC60F002D57D0FF2D24D08020DB008C
:1095E000C0041843002381469A469B467F3D7C0277
:1095F0007A00FB0F640A120E984623D0FF2A4BD044
:10960000E30080240020E4047F3A1C43AD186B1C67
:1096100047460193534677403A000F2B48D87D497F
:109620009B00CB589F46002B00D085E008339A461C
:10963000063B9B467C027A00FB0FFF25640A120E54
:109640009846DBD1002C00D090E0524601231A430B
:1096500092460120DBE74C4658461700022824D0EA
:10966000032800D1CFE00022002301284DD1580269
:10967000D205400AFF071043384303B03CBC904674
:109680009946A246AB46F0BD002B5BD104239A4617
:10969000033B00259B46AAE7FF35002C60D15246CC
:1096A00002231A4392460220B1E7FF220023DEE79D
:1096B0004B461B0C9C464B462604360C1804614650
:1096C0003300220C6446000C43434E435043544342
:1096D00080191A0C1218964203D9802149028C462F
:1096E00064441B041B0C1004C01883015E1EB341AC
:1096F000800E1843130C1B199B0103431C0023010C
:1097000079D5012362081C401443019A7F32002A54
:109710004DDD630704D00F232340042B00D0043415
:10972000230103D53C4B019A1C408032FE2ABCDC4D
:10973000A3015B0AD2B29AE70C239A46093BFF25A4
:109740009B4654E7180001F071FE4A46431F7625F8
:109750009A4000236D4291462D1A9A469B4646E751
:10976000524603231A439246032050E7200001F09B
:109770005DFE431F2D1A9C40763D002047E7802365
:109780000027DB03FF2272E7424666E74C463200C1
:10979000584662E780234A46DB031A4222D01C4225
:1097A00020D123435B025B0A4746FF225FE7012388
:1097B0009A1A1B2A21DC23000199D3409E318C4048
:1097C0001A0023005C1EA34113435A0704D00F2242
:1097D0001A40042A00D004335A0111D49B015B0AB9
:1097E000002244E780234A46DB0313435B025B0A03
:1097F0003700FF223BE7019587E70022002336E789
:109800000122002333E78023DB0323435B025B0A4F
:10981000FF222CE7C8E10000FFFFFFF770B500282A
:109820003DD0C317C5185D40C40F280001F0FEFDF0
:109830009E22121A962A07DCD2B2082833DD083895
:1098400085406802400A23E0992A0BDD05232900A0
:109850001B1AD94003001B339D402B005D1EAB41FA
:1098600019430D00052801DD431F9D402B000F49C2
:109870000B406E0709D00F263540042D05D0043368
:109880005D0102D59F220B40121A9B01580AD2B2E9
:109890004002D205400AE4071043204370BD002473
:1098A00000220020F4E76802400AF1E7FFFFFFFB17
:1098B000F0B54F464646D6460C000903C0B5490AE6
:1098C000470F5E0039431F03DB0F9C4665007B0A90
:1098D000570F1F436D0DE40F760DA146C000B8462B
:1098E000D200AB1B64457BD0002B5FDD002E00D087
:1098F000A4E03E00164300D112E15E1E002E00D00F
:109900009EE1871A4346B84280410125C91A404268
:10991000091A0B0200D431E149024E0A002E00D18F
:109920006EE1300001F082FD0300083B1F2B00DDDB
:1099300061E120223900D21A9E40D1409F400E435F
:109940009D4200DD51E15D1B6B1C1F2B00DD7CE1A6
:109950002021C91A3D0030008F408840DD40791E2B
:109960008F41310007222843D940002507433A4060
:10997000002A09D00F233B40042B05D03B1DBB42DE
:10998000BF417F42C9191F000B0200D426E26A1CA6
:10999000C64B55056D0D9A4200D106E1C44AFF0839
:1099A0000A40530752023B43120B8EE0002B00D0BB
:1099B000B8E06B1C5B055B0D012B00DC30E1871A06
:1099C0004346B842B641CB1A76429E1B330200D5BD
:1099D0004CE13B003343A1D100220024002570E07C
:1099E000002B00DCE5E0002E00D183E0AF4EB54255
:1099F00060D0802636043743B846382B00DC3EE181
:109A0000434613431F007A1E97413F188742804107
:109A1000404209180B0200D4B0E0A44B01359D422E
:109A200000D1C3E0A24A7B080A4001210F401F4336
:109A30005108D30707221F433A4099E79B4EB5428E
:109A400038D0802636043743B846382B00DDDCE0BA
:109A50001F2B00DC30E11E004746203EF740BC468D
:109A6000202B04D04026F31A46469E40324317006E
:109A700063467A1E97411F43CCE0002B00D104E2DD
:109A80004346134300D159E14B07C00818438023D4
:109A9000C9081B03194208D04546ED081D4204D1F0
:109AA0004346D008590708432900420FC9007F4D9B
:109AB0001143C0004B07CA087C49C00803438D42CC
:109AC00068D012036D05120B6D0D002112031800F2
:109AD000130B0A0D12051A43764B2D0513402B4329
:109AE0005B00E4075B08234319001CBC90469946C1
:109AF000A246F0BD3E00164312D05E1E002E00D0DE
:109B000000E18718874280414144404209180125FD
:109B10000B0233D5022585E7644633004146100029
:109B20001D00C7E7002D00D0DAE00C000443F3D09D
:109B30005C1C00D19FE15D4CA64200D12FE1DB43CC
:109B4000382B00DD66E11F2B00DD83E120240500BA
:109B5000E41A0F00DD40D940A0404346A7405B1AFD
:109B6000441EA04198462F433843171ABA429241E7
:109B700043465242991A64463500CAE607223A40E3
:109B8000002A00D0F6E64B07CA084849FF083B43C5
:109B90008D4296D11900114300D19EE18021090325
:109BA0000A431203120B414D8FE7150000220023D8
:109BB0008BE7002B00D0C7E06B1C5F057F0D012FEA
:109BC00000DCF1E0394DAB4200D1B9E085180A0064
:109BD000854289414244494251180722CF076D0806
:109BE0002F4349083A401D00C2E607223049ED1ACA
:109BF00031403A40BCE63E002838864000279FE6C8
:109C0000380001F013FC20308EE6434613431F005A
:109C10007A1E9741C71BB84280414042091A78E634
:109C20000E003B0006431343002D61D1002E00D0EF
:109C3000F4E0002B00D11BE164463900100039E745
:109C40001A4FBB427AD03300FFE630001F3DE84098
:109C5000202B03D04021CB1A9E4037437B1E9F41CF
:109C6000072207433A400021002589E7171A434697
:109C7000BA42B641591A76428E1B64464EE61F2BF5
:109C800000DDADE020264746F61AB740B94617007A
:109C9000B246DF404E463E4337005646B240561E5F
:109CA000B24117434246DA408918AEE6FF0700008A
:109CB000FFFF7FFFFFFF0F8020264746F61AB740C1
:109CC000B9461700B246DF404E463E43370056467F
:109CD000B240561EB24117434246DA40891A99E70C
:109CE0007F4CA6425BD0802424045B42214327E7BB
:109CF000002E0CD1002B00D1CBE0644639001000BF
:109D0000774DD7E6764FBB4218D0330075E6002B6F
:109D100014D04B07C00818438023C9081B031942FD
:109D200007D0FC081C4204D17907D0080843E1465B
:109D300021004C46420FC9001143C000684DB9E6EE
:109D40001D0000220023C0E6002D5BD10D0005435D
:109D500000D1E2E65D1C00D1B0E0614DAE421FD003
:109D6000DB43382B71DC1F2B00DD96E020250F0034
:109D7000ED1AAF40B9460700AA46DF404D463D43C5
:109D80002F005546A840D940451EA84188440743A6
:109D9000BF18974292415142414435003AE6644629
:109DA00035004146100085E60B000343002D00D02E
:109DB00063E6002BF5D04346134300D17AE68718BB
:109DC0008742804107224144404209183A400B0231
:109DD00000D4D5E6434B01351940C9E5380069E6A2
:109DE0001E004746203EF740BC46202B04D04026AC
:109DF000F31A46469E403243170063467A1E974147
:109E00001F4302E6364DAE42CAD080252D045B4288
:109E10002943A6E70843411E8841A6E6002B00D14E
:109E200048E6871A4346B842B641CB1A76429E1B93
:109E300033024BD5171A4346BA429241591A52423D
:109E4000891A072264463A4092E501430F00791EC1
:109E50008F419DE71C000F00203CE740202B03D0E2
:109E60004024E31A99400843411E884138437CE668
:109E70000022002425E6171A4346BA429241591A95
:109E80005242891A6446350043E541461000144D9C
:109E900010E680220024120380E61D000F00203D02
:109EA000EF40BC46202B03D04025EB1A99400843D5
:109EB00007006346781E87411F4369E7871897426A
:109EC0009B4141445B42C9183500A3E53B00334345
:109ED000CED0072231003A4052E600231A00F4E5C2
:109EE000FF070000FFFF7FFFF0B55746DE464E46F6
:109EF0004546E0B5834607000E03480085B092460C
:109F00001C00360B400DCD0F002800D19DE0954B75
:109F1000984239D08023F6001B041E43924A7B0FDF
:109F2000334399469446030063440093002300267C
:109F3000FF00029323031B0B98466300E40F524675
:109F40005B0D019400D1B3E086498B4200D19EE0C5
:109F50004246D100802212040A435146490F114360
:109F60008B46814952468C4600996344CB1A0021A6
:109F7000D20000932B0063409A460F2E00D905E1D2
:109F80007A4BB6009B599F465B463343994600D0B7
:109F9000B8E002230826002700900293CAE7CB46C8
:109FA0003A0002990195019B9A46022927D003297C
:109FB00000D180E2012944D06D49009B8C46634466
:109FC0001C00002C38DD530700D013E2D2085B469A
:109FD000DB0109D55946674B19408B468021C900E2
:109FE0008C46009B63441C00634B9C4207DC5B4631
:109FF00064055F075B0217431B0B620D02E0002341
:10A000000027584A00211B031C0B0B0D1B05234383
:10A0100014055A4A380013401C4353466400DB07BA
:10A0200064081C43210005B03CBC90469946A246FA
:10A03000AB46F0BD0122524201231B1B382B00DC32
:10A04000ADE1002200230027DCE75B46334399465D
:10A050005ED0002E00D18AE1300001F0E7F9030064
:10A060000B3B1C2B00DD7BE11D22D31A5A4601005D
:10A07000DA4008398E4013005F46334399468F40DB
:10A080003F4B00261B1A00930023029352E74146E0
:10A0900053460B433B499B468C46009B63440093CD
:10A0A0005B46002B3BD1022300221E43022161E7C5
:10A0B000434613439B4637D04346002B00D162E111
:10A0C000404601F0B3F903000B3B1C2B00DD53E1CC
:10A0D00002004146083A914088461D21CB1A51465C
:10A0E000D9400B0041460B439B46534693401A0010
:10A0F000009B25499C46604403008C4663440093C2
:10A10000002137E70323B14600900C26029311E7A4
:10A110000023009301330426002702930AE7032358
:10A12000C3461E43032125E701331E4300220121BC
:10A1300020E700239A46802300271B03094A61E792
:10A14000802349461B03194200D1E2E059461942D7
:10A1500000D0DEE00B431B0317001B0BA246014A95
:10A1600050E7C046FF07000001FCFFFF08E20000C7
:10A17000FF030000FFFFFFFEFE070000FFFF0F8050
:10A180000DFCFFFF01F8FFFFF3030000D94500D9E4
:10A19000CBE000D1C6E03C0048460027009B013BD5
:10A1A00000935B46160E1B021E43130298463304AF
:10A1B0001B0C9946310C0191FFF798F84A4642432F
:10A1C0000B04210C050019438A4207D98919013D66
:10A1D0008E4203D88A4201D9851E8919881A0199AD
:10A1E000FFF784F809048C464A462104644642433A
:10A1F000090C030021438A4204D98919013B8E428C
:10A2000000D8F1E02D041D43AB464346891A42466F
:10A21000280C12041D0C5B46140C22001B041B0CA2
:10A220005A4303946B434443029568431B19150C2E
:10A23000EB189C4203D980246402A44660441C0CA1
:10A2400015041B042D0C20185D19814277D373D09F
:10A250000C1AA24A7D1BAF42BF419446009B7F422D
:10A260006344E01B1C00864200D1DBE00199FFF74C
:10A270003DF84A4642430B04290C070019438A4221
:10A2800007D98919013F8E4203D88A4201D9871E16
:10A290008919881A0199FFF729F809044A4689465D
:10A2A00029044D464243090C030029438A4207D939
:10A2B0008919013B8E4203D88A4201D9831E89192C
:10A2C0003F04891A3A00039F1A43380013041B0CF9
:10A2D000584381460298150C6F4343434543484613
:10A2E000000C8446DB1963449F4203D9802040025E
:10A2F0008446654448461F0C00041B04000C7D196D
:10A300001818A94200D284E000D17FE001231A434B
:10A3100057E680234A461B0313431B031B0BAA4625
:10A320006F4A6FE6BA4200D935E74B46DC0758085A
:10A330007B081C43FF0734E70024AF4289D247441F
:10A340004745A4415B466442A4196418013BA642F8
:10A350001ED2A0426DD800D1B6E0241A9B4678E701
:10A3600003005A46283B9A400027914688E6584603
:10A3700001F05CF8203072E603005246283B9A4018
:10A3800093460022B4E6504601F050F820309AE699
:10A39000A642E2D1B845DCD9341A9B4659E71F2BB7
:10A3A00065DC504C0099A4465C46614408008C4032
:10A3B00011008240D940501E82410C4314435A463A
:10A3C000DA401300620709D00F222240042A05D088
:10A3D0002200141D9442894149425B181A0262D539
:10A3E0000122002300270DE68A4200D80AE7831ED7
:10A3F000891907E70F231340042B00D1E6E5171D49
:10A400009742924153429B44FA08E0E5002800D16C
:10A41000D7E57118531EB14227D3A94215D358D09E
:10A420001A0073E7002B00DC04E6012300229B44A2
:10A43000CDE502234744474589415B429C4649425A
:10A4400089190C19E344241A03E743465F00474582
:10A450009B41B8465B429E19023A8919A94200D035
:10A4600054E7404500D051E7ABE51A00F6E71F215D
:10A470005F4649420C1BE740202B07D01A49009B3E
:10A480008C46634418005B4683401A43501E824149
:10A490003A4307270023174009D00F21002311401A
:10A4A0001400042995D122005F075B021B0BD20820
:10A4B00017430022A6E5802359461B030B431B03C9
:10A4C00017001B0B064A9DE5BD42B2D89B460024EF
:10A4D000BFE68045B9D31A00C3E7C046FF030000BA
:10A4E000FF0700001E0400003E040000F0B54F46C8
:10A4F0004646D6468446C0B58046194E18030F031B
:10A500004D00000B5C0082463F0B6D0DC90F91465C
:10A51000640DDB0F0120B5420AD0B44203D0A5423E
:10A5200001D157450CD01CBC90469946A246F0BDBF
:10A5300066463E43F7D1AC42F5D154461443F2D1BE
:10A540000120C845EFD1994207D0002DEBD16346D9
:10A550001F433800471EB841E5E70020E3E7C04647
:10A56000FF070000F0B54F464646D6464D00C0B541
:10A570000E03C90F8A462C491F035C008046360B28
:10A580006D0D91463F0B640DDB0F8D421ED08C424A
:10A5900016D0002D1ED130438446002C01D13A4301
:10A5A00023D06246002A1AD09A4529D0514602206B
:10A5B0000139084001381CBC90469946A246F0BDBE
:10A5C00039001143E5D002204042F4E73043FAD18C
:10A5D000AC420FD0002C0FD13A43E7D00CE001225F
:10A5E000013B934318000130E5E763460020002B50
:10A5F000E1D0DBE73A43E6D19A45D7D1A542D5DC95
:10A60000A54205DBBE42D1D808D00020BE42D2D23E
:10A6100050460123013898430130CCE7C845C5D8DE
:10A620000020C845F4D3C6E7FF070000F0B54F4649
:10A630004646D6464D00C0B50E03C90F8A462E4980
:10A640001F035C008046360B6D0D91463F0B640D79
:10A65000DB0F8D4218D08C4211D0002D18D1304321
:10A660008446002C1ED13A431CD163460020002BA7
:10A6700030D0514602200139084001382AE0390023
:10A680001143EAD0022025E03043FBD1AC4226D072
:10A69000002C26D13A4324D15146022001390840EA
:10A6A000013817E06246002A0FD09A45E1D1A54251
:10A6B00005DBBE42DDD819D00020BE420AD250468A
:10A6C000012301389843013004E00122013B934308
:10A6D000180001301CBC90469946A246F0BD3A4392
:10A6E000D0D19A45C5D1A542C3DCE0E7C845C0D862
:10A6F0000020C845E3D3EDE7FF070000F0B557465B
:10A70000DE464E464546E0B5834606000F03480048
:10A7100087B092461D003F0B400DCC0F002800D1A2
:10A720006FE0DE4B984238D08023FF001B041F43AC
:10A73000730F3B430193DA4B0027994600239B4656
:10A74000F60081442B0369001B0B52469846490DC5
:10A75000ED0F002900D185E0D04B994200D173E084
:10A760004346DA0080231B0413435246CC48520F61
:10A7700084461343524600206144D200894421009C
:10A78000694000918C46012149448A460F2F00D927
:10A7900090E0C449BF00CF59BF465B463B4301939D
:10A7A00000D06AE102230827002681469B46C9E7BC
:10A7B00032005846019B61460091022800D175E0A5
:10A7C000032800D1FEE1012800D02CE1002300275E
:10A7D000002600253F032A0D3F0BB34812053A43DC
:10A7E00002401B051343009A5B00D1075B080B4333
:10A7F0003000190007B03CBC90469946A246AB46D3
:10A80000F0BD5B463B43019300D12FE1002F00D107
:10A81000A5E1380000F00AFE03000B3B1C2B00DD15
:10A8200096E11D22D31A5A460100DA405E460839E5
:10A830008F4013008E403B4301939C4B00271B1A13
:10A84000994600239B467DE7414653460B43934977
:10A850008C46E144002B00D01AE10222022017436B
:10A8600000228CE7134300D10DE14346002B00D1B9
:10A8700081E1404600F0DAFD02000B3A1C2A00DDBF
:10A8800072E10100434608398B4098461D239A1A0D
:10A890005346D3401A004346134352468A40494622
:10A8A000081A824989468144002068E77B4B0027CB
:10A8B00000268EE7140C1204120C1100370C36041B
:10A8C000350C794328008C462E0060436044834653
:10A8D00056432100300C804658467943404402914B
:10A8E000844506D98846802149028C46E044414689
:10A8F00002913604010C360C00048B4681191E0CA3
:10A900001B041B0C0391190079438C4628007543E6
:10A910006544A8465843050C45447743A94203D9EA
:10A92000802149028C466744290C8C46390000047A
:10A93000000C2D042D186144AB4405915946049137
:10A9400001990F043F0C080C3900514342439046D3
:10A9500002008C46090C8B4662437C4344445C44B1
:10A96000A04503D98021490288464244210C8846EB
:10A9700061460904090C8C4639005943434370432E
:10A980007E430F0CF6182404BE19644442448C46DE
:10A99000B34203D980235B0298464044029B614640
:10A9A0009846049B370443449B46AB45AD416B42FC
:10A9B0000D0405992D0C8C467F196744FD18A84697
:10A9C0005D462D19A542A44193466442A446C34462
:10A9D000DC448F42BF4198459B4193459241A44539
:10A9E000A4415B427F421F43360C52426442BF196E
:10A9F0002243BF18624638184302D20D039913430D
:10AA00006A020A43501E82416146ED0D2A434E02FE
:10AA10003243D90100D4B3E001265008324002434A
:10AA2000DE0732435B08224C5444002C62DD5107A0
:10AA300009D00F201040042805D0101D90429241EB
:10AA400052429B180200D90104D580241948E40021
:10AA5000034054441848844200DD27E75E075B0248
:10AA6000D2081F0B630516435B0DB2E6002399461F
:10AA70000133042700269B4664E6032301978146A1
:10AA80000C279B465EE6012201201743002276E652
:10AA9000032303201F43434671E6C046FF0700001F
:10AAA00001FCFFFF48E20000FFFF0F800DFCFFFFED
:10AAB000FF030000FFFFFFFEFE07000000238027CA
:10AAC00000933F030026434B83E6019B3200A446DC
:10AAD000584670E6AC466EE6802701993F0339423E
:10AAE0002DD03B422BD11F433F033F0B0095160057
:10AAF000384B6EE601252D1B382D00DD66E61F2D37
:10AB000040DC35481C005044160082408440EE4032
:10AB1000501E824134431443EB40620709D00F2298
:10AB20002240042A05D02200141D94428041404254
:10AB30001B181A023ED501230027002649E680276C
:10AB4000019B3F031F433F033F0B0094214B40E613
:10AB500003005A46283B9A40002601926DE658466B
:10AB600000F064FC203057E603005246283B9A4030
:10AB70001300002293E6504600F058FC20307BE69C
:10AB8000CA4650E71F201E004042041BE640202D0D
:10AB900003D0124C5444A3401A43501E8241324306
:10ABA00007260027164009D00F200023104014006C
:10ABB0000428B9D122005E075B021F0BD20816439E
:10ABC000002306E680273F031F433F033F0B160089
:10ABD000004BFEE5FF0700001E0400003E040000DD
:10ABE000F8B557464E464546DE460C000903E0B52B
:10ABF000490A460F5F0031431E03DB0F760A9B466E
:10AC0000530F3343C84E6500C000E40FD2006D0DF2
:10AC1000A24681467F0D9C469046B74200D1B9E0DE
:10AC20005B46012673409B46EE1BA34500D183E0A3
:10AC3000002E63DD002F00D0B1E06346134300D146
:10AC400023E1731E002B00D0BAE1861A6346B0429E
:10AC500080410125C91A4042091A0B0200D447E17C
:10AC600049024B0A98464346002B00D189E14046F1
:10AC700000F0DCFB0300083B1F2B00DD7CE1202201
:10AC80003000D21A4146D040994002009E400A430B
:10AC90009D4200DD6AE15D1B6B1C1F2B00DD94E112
:10ACA000202110003500C91A8E40DA408840DD406E
:10ACB000711E8E41110007222843002506433240B1
:10ACC000002A09D00F233340042B05D0331DB34293
:10ACD000B641764289191E000B0200D43DE26A1C7F
:10ACE000914B55056D0D9A4200D119E18F4AF60836
:10ACF0000A40570752023743120B9BE0002E00D048
:10AD0000C5E06E1C7605760D012E00DC48E1674635
:10AD1000861ACB1BB042BF417F42B8461F00434654
:10AD2000FF1A3B00B8461B0200D55FE137439AD1BA
:10AD300000220024002579E0002E00DCFAE0002F3C
:10AD400000D18DE0784B9D4267D0802367461B047D
:10AD50001F43BC46382E00DC52E1634613435A1EA3
:10AD600093411E1886428041404209180B0200D4CC
:10AD7000BEE06D4B01359D4200D1D2E06B4A7308B5
:10AD80000A4001210E401E435108D30707221E43EB
:10AD9000324095E71E00164300D045E740E7624B7E
:10ADA0009D423AD0802367461B041F43BC46382E81
:10ADB00000DDEBE01F2E00DC3AE133006746203B6C
:10ADC000DF403B00202E05D04027BF1B6646BE401B
:10ADD000324390464646721E96413343DAE0002BDA
:10ADE00000D114E26346134300D168E180234E078B
:10ADF000C008C9081B030643194208D06046C008B2
:10AE0000184204D163460100D2085E071643F300DE
:10AE10009946C900720F444D11434B46DE08424B20
:10AE20004F073743CA089D4200D16EE012036D05FB
:10AE3000120B6D0D00211203130B0A0D12051A439C
:10AE40003B4B2D0513402B435B00E4075B0823437A
:10AE5000380019003CBC90469946A246AB46F8BD66
:10AE60006346134311D0731E002B00D007E18618F0
:10AE70008642804161444042091801250B0237D5C2
:10AE800002257BE73E00614691463500C5E75C46FA
:10AE9000002D00D0E1E00B000343F3D0731C00D180
:10AEA000ACE1214B9F4200D13AE1F343382B00DD66
:10AEB0006FE11F2B00DD8CE120250E00ED1AAE4066
:10AEC000B0460600AA46DE40454635432E005546AC
:10AED000D940A8406346451EA8415B1A9C463043B2
:10AEE000161AB242924163465242991A3D00B4E6A4
:10AEF00007223240002A00D0E4E60B4BF6084F0749
:10AF00003743CA089D4200D090E73B00134300D16D
:10AF1000A6E180231B031A431203120B024D89E79B
:10AF200015000022002785E7FF070000FFFF7FFFD5
:10AF3000FFFF0F80002E00D0C7E06B1C5E05760D72
:10AF4000012E00DCF0E0C84DAB4200D1B9E085181D
:10AF50000A00854289416244494251180722CE07BE
:10AF60006D082E43490832401D00A9E6BF49ED1A7D
:10AF7000114007223240A3E63200283882400026E2
:10AF800086E6300000F052FA203073E66346134341
:10AF90005A1E9341C61AB04280414042091A5CE6EB
:10AFA0000E00674606431743002D5ED1002E00D0E9
:10AFB000F3E0002F00D11EE15C46614691462CE78C
:10AFC000A94FBE427BD01E00F1E610001F3DE840B5
:10AFD000202B03D04021CB1A9A401643731E9E416A
:10AFE0000722064332400021002583E7161A6346F4
:10AFF000B2428041591A40420B1A98465C4632E6EA
:10B000001F2E00DDABE02027BB1B9A466346574648
:10B01000BB40994613004F46F3401F433B00574641
:10B02000BA40571EBA4113436246F240891898E667
:10B030002027BB1B9A4663465746BB4099461300E0
:10B040004F46F3401F433B005746BA40571EBA4194
:10B0500013436246F240891A9CE7834B9F425FD0BC
:10B0600080252D047342294320E7002E0CD1002FA8
:10B0700000D1D0E05C46614691467B4DCDE67A4FEB
:10B08000BE421CD01E0065E6002F18D0C0084E0737
:10B0900006438020C9080003014208D06346DC084B
:10B0A000044204D12100DA46D2085E071643F300B9
:10B0B000994601245346C900720F11431C406A4D42
:10B0C000ABE61D0000220027B4E6002D59D10B008D
:10B0D000034300D1D6E6731C00D1B2E0624B9F421D
:10B0E0001ED0F343382B6FDC1F2B00DD97E02025AB
:10B0F0000E00ED1AAE40B0460600AA46DE404546B8
:10B1000035432E005546A840D940451EA8418C44E1
:10B110000643B61896429241514261443D0025E6ED
:10B120003D006146914678E60B000343002D00D0B8
:10B1300055E6002BF5D06346134300D16DE6861823
:10B140008642804161444042091800220B0200D42B
:10B15000D0E6464B01351940B2E5B1465DE6330015
:10B160006746203BDF403B00202E05D04027BF1B19
:10B170006646BE40324390464646721E9641334371
:10B18000EFE5394B9F42CBD080252D0473422943F4
:10B19000A8E70843411E8841A2E6002F00D13CE603
:10B1A0006346861ACF1AB0429B415B42FB1A98460F
:10B1B0001B024ED5161A6346B2429241591A5242A8
:10B1C000891A5C4600227BE501430E00711E8E4108
:10B1D0009FE71D000E00203DEE40B046202B04D01E
:10B1E0004025EB1A99400843814648464346411E94
:10B1F0008841184374E60022002417E6161A6346B5
:10B20000B2429241591A5242891A3D0025E56146DF
:10B210009146154D01E680220024120379E61D00B7
:10B220000E00203DEE40B046202B04D04025EB1A06
:10B230009940084381464E464346711E8E411E4347
:10B2400067E7861896429B4161445B42C9183D00FE
:10B250008CE547463743CED007224146324049E687
:10B2600000273A00E6E5C046FF070000FFFF7FFF2A
:10B2700070B50C4E0D031C0349005B002D0B490DEE
:10B28000240B5B0DB14208D0064900208B4203D14C
:10B2900014432000441EA04170BD05430120002D31
:10B2A000FAD1F1E7FF07000030B5144D0A034B0057
:10B2B000120B5B0DC90F0024AB4211DD104CA342F1
:10B2C00010DC8024640322430E4CE41A1F2C0CDD96
:10B2D0000D48C31ADA4013005C42002900D11C005B
:10B2E000200030BD094BCC18FAE7094DE040AC46D0
:10B2F00063449A4013000343EEE7C046FE03000098
:10B300001D0400003304000013040000FFFFFF7F52
:10B31000EDFBFFFF70B500282DD0C317C5185D40A9
:10B32000C40F280000F082F8154B1B1A5B055B0D5B
:10B330000A2815DD0B38854000222D032D0B002136
:10B3400010002D030A0D2D0B12052A430D4D1B0570
:10B350002A4013435B00E4075B082343190070BDD8
:10B3600002002900153291400A000B21081AC5403D
:10B370002D032D0BE3E70024002300250022DEE748
:10B380001E040000FFFF0F804100090E4B1C70B52A
:10B39000DBB24602750AC40F012B14DDE0239B00CB
:10B3A0006D07360BCB1800210A0D280012051C4D25
:10B3B00032435B052A405B0813435B00E4075B08EC
:10B3C0002343190070BD002914D1002D1ED0280080
:10B3D00000F02CF80A281CDC0B232A001B1ADA4088
:10B3E000030015339D400F4B12031B1A5B05160B10
:10B3F0005B0DD8E7002D06D0320B802636036D0793
:10B400001643094BCFE7084B0026CCE70023002664
:10B41000C9E703002A000B3B9A400025E3E7C0463A
:10B42000FFFF0F8089030000FF0700001C2101239C
:10B430001B04984201D3000C10391B0A984201D317
:10B44000000A08391B09984201D30009043902A2F5
:10B45000105C40187047C04604030202010101015C
:10B46000000000000000000030B51C00094B050082
:10B470001B6885B0D868084B002A01D1074B1A0019
:10B480000292019300912B002200054900F026F85A
:10B4900000F0A6FD8000002088E20000B0D000008F
:10B4A00095E20000014B18687047C04680000020FC
:10B4B000084B10B50400002B02D0002100E000BFB3
:10B4C000054B1868836A002B00D09847200001F0D4
:10B4D0005DFBC04600000000C4E200000EB403B5EE
:10B4E000010003AB044804CB0068019300F076F838
:10B4F00002B008BC03B018478000002070B50026D9
:10B500000C4D0D4C641BA410A64209D1002601F07D
:10B510003FFB0A4D0A4C641BA410A64205D170BD26
:10B52000B300EB5898470136EEE7B300EB58984765
:10B530000136F2E7500200205002002050020020A5
:10B5400060020020002310B59A4200D110BDCC5CEF
:10B55000C4540133F8E710B5884202D98B189842D9
:10B5600003D3002307E08B5C8354013AFBD210BD68
:10B57000CC5CC45401339A42FAD1F8E703001218A4
:10B58000934200D1704719700133F9E7936810B501
:10B59000013B9360002B04DA9469A34207DB0A297C
:10B5A00005D01368581C10601970080010BD00F019
:10B5B0004BFC0100F9E7F8B506000F001400D518A0
:10B5C000AC4201D1002007E021783A003000FFF7BB
:10B5D000DDFF0134431CF3D1F8BD0000F0B59FB08E
:10B5E00002900F0016000593002805D0836904938C
:10B5F000002B01D100F0F4FD7B4B9F425BD1029BFD
:10B600005F68BB891B0762D53B69002B5FD00023B5
:10B6100006AC6361203363761033A37635002B7854
:10B62000002B01D0252B5CD1AB1B04930CD0320036
:10B6300039000298FFF7BFFF431C00D1C4E06269E4
:10B64000049B9446634463612B78002B00D1BBE0DC
:10B65000012200235242626002A9543252186E1C29
:10B660002360E360A3601370A365317805225F480F
:10B6700000F0D4FE751C002835D12268D30604D50D
:10B68000532302A95B1820211970130704D55323F3
:10B6900002A95B182B21197033782A2B2CD0350086
:10B6A00000210A20E3682A786E1C303A092A64D9FE
:10B6B00000292ED026E04E4B9F4202D1029B9F686C
:10B6C0009FE74C4B9F429CD1029BDF6899E7390072
:10B6D000029800F00FFC002899D0012040421FB0D2
:10B6E000F0BD01359BE7414B2268C01A012383401E
:10B6F000134323602E00B8E7059B191D1B680591B5
:10B70000002B01DB099304E05B42E3600223134357
:10B7100023602B782E2B0AD16B782A2B35D1059BF1
:10B7200002351A1D1B680592002B2BDB0793324E46
:10B7300029780322300000F071FE002806D0402353
:10B74000801B834022680135134323602978062239
:10B750002A486E1C217600F061FE00283AD0284B62
:10B76000002B25D10722059B07339343083305930C
:10B770006369039A9B18636150E7434301219B1857
:10B78000350090E701235B42D0E700230A201A002E
:10B790000135636029786E1C3039092903D9002BE3
:10B7A000C5D00792C3E74243012352183500F1E7A1
:10B7B00005AB00933A00134B2100029800E000BF54
:10B7C0000390039B0133D3D1BB895B0600D584E78B
:10B7D0000B9884E705AB00933A000A4B21000298CE
:10B7E00000F080F8ECE7C0461CE30000C8E200006F
:10B7F0003CE30000FCE20000CEE20000D2E20000E8
:10B8000000000000B7B50000F7B5150001938A6885
:10B810000B6900900C00934200DA130022002B60A9
:10B8200043321278002A01D001332B6023689B0633
:10B8300002D52B6802332B60062723681F4027D0D0
:10B84000230043331B785A1E93412268920630D45A
:10B850002200019943320098089EB047431C25D02E
:10B86000062320682A68E16803400025042B03D1E1
:10B870008D1AEB43DB171D40A3682269934201DD5B
:10B880009B1AED180027BD4220D1002010E001379F
:10B89000E3682A689B1ABB42D2DD220001231932D9
:10B8A00001990098089EB047431CF0D10120404206
:10B8B000FEBD3020E1184331087021005A1C45318B
:10B8C0000978A218433202331170C1E72200012324
:10B8D0001A3201990098089EB047431CE6D0013700
:10B8E000D1E70000F0B589B004920A004332059315
:10B8F000039002920A7E0C000E9B6E2A00D186E015
:10B900001FD8632A33D008D8002A00D18CE0582AE7
:10B910004DD0250042352A7030E0642A01D0692AD2
:10B92000F7D1196825680A1D280629D508681A6004
:10B93000002803DA2D23029A404213706B4E0A2727
:10B940004FE0732A74D008D86F2A1FD0702AE0D134
:10B95000202209680A43226003E0752A16D0782A5B
:10B96000D7D12200782145321170614E22E02500A6
:10B970001A684235111D196013682B70012365E0A8
:10B9800008681A606906D3D500B2D1E7196825683E
:10B99000081D186008682E0605D5544E08276F2A22
:10B9A0001BD00A2719E06D06F7D580B2F5E74531BF
:10B9B0004E4E0A7018682268011D0068196015064D
:10B9C00021D5D30702D520231A432260102700284F
:10B9D00003D1202322689A432260230000224333AC
:10B9E0001A706368A360002B58DB0422216891431E
:10B9F0002160002854D1029D002B5AD025003378B5
:10BA000042352B7055E05506DBD580B2D9E71A6870
:10BA10000D68101D4969186013682E0601D519605C
:10BA200002E06D06FBD519800023029D23614FE0E3
:10BA30001A68111D1960156800216268280000F05D
:10BA4000EDFC002801D0401B606063682361002387
:10BA5000029A13703CE023692A0004990398059D1B
:10BA6000A847431C3ED023689B0715D4079BE0687A
:10BA7000984239DA180037E022000123193204997C
:10BA80000398059EB047431C2CD00135E368079A04
:10BA90009B1AAB42F0DCE9E70025F7E70028ADD0C0
:10BAA000029D3900FDF722FC735C013D2B700028DC
:10BAB000F7D1082F09D12368DB0706D5636822690F
:10BAC000934202DC3023013D2B70029B5B1B236100
:10BAD000059B07AA00932100049B0398FFF794FE9F
:10BAE000431CB8D10120404209B0F0BDD9E20000AA
:10BAF000EAE200000D4B70B51C680500A36B002B3B
:10BB00000FD1182000F06EFC094BA0630360094BB5
:10BB100001224360084B83600B2383810023026171
:10BB200043610022A36B1D615A6170BD800000203B
:10BB30000E33CDAB34126DE6ECDE0500124B10B5C2
:10BB40001C68A36B002B0FD1182000F04BFC0F4B8F
:10BB5000A06303600E4B012243600E4B83600B23F6
:10BB60008381002302614361A46B0B4A20696169F0
:10BB70000A4BFDF7F7FC0122002380185941206190
:10BB800061614800400810BD800000200E33CDAB3D
:10BB900034126DE6ECDE05002D7F954C2DF45158E6
:10BBA0000CB430B5164B9DB00C1E1D6808DA8B2303
:10BBB00001202B6040421DB030BC08BC02B01847C9
:10BBC000822302A99B008B810023029008619C4282
:10BBD00000D0631E8B604B6101235B42CB81209AB6
:10BBE00021AB2800019300F055FD431C01DA8B23A3
:10BBF0002B60002CDFD00023029A1370DBE7C046D5
:10BC0000800000200EB400B50B499CB01DAB029023
:10BC10000690079104910948094904CB05910068F1
:10BC200002A9019300F036FD0023029A13701CB0A4
:10BC300008BC03B01847C046FFFFFF7F800000200C
:10BC40000802FFFF020010B51378541C002B05D129
:10BC5000CC5CD4540133002CFAD110BD2200F3E7A0
:10BC6000C9B20378002B04D08B4200D17047013059
:10BC7000F7E74B42594149420840F7E702780B7811
:10BC8000002A03D0013001319A42F7D0D01A704710
:10BC90000023C25C0133002AFBD1581E70470023E9
:10BCA00030B59A420AD0013AC45CCD5CAC4204D1B2
:10BCB000934202D00133002CF6D1631B180030BD33
:10BCC00030B50500002A00D130BD0C78013A6B1C5C
:10BCD0002C700131002C05D19A189A42F4D01C70B6
:10BCE0000133FAE71D00EDE710B50378002B0FD103
:10BCF0000B785A4253415B42184010BD0023CA5C86
:10BD0000002AFAD0C45C944201D10133F7E7013034
:10BD10000378002BF2D11800EFE70000F0B51F0008
:10BD20000E0087B00590019102920C98347800F0D3
:10BD3000EAFA082200194378751C134036D12D2CDD
:10BD400036D1B51C74780126002F62D0102F09D18E
:10BD5000302C07D120222B789343582B54D1102715
:10BD60006C7802352D4B3900F31818000393FDF75A
:10BD7000BDFA049101210023494202008C461800BB
:10BD80002100303909291AD80C00A74223DD591C9B
:10BD900009D06346824206D302D10499A14202DB54
:10BDA0000123784320182C780135E9E72E00BCE701
:10BDB0002B2C01D01E00C7E7B51C7478FAE72100D0
:10BDC0004139192901D8373CDFE7210061391929A8
:10BDD00001D8573CD9E75A1C08D1059A2333136080
:10BDE000029B0398002B09D107B0F0BD002E00D0B4
:10BDF0004042029A002AF7D0002B01D06B1E01931B
:10BE0000029B019A1A60EFE73024002FAAD108277D
:10BE1000A8E7302C9ED00A27A4E7C046FFFFFF7F8B
:10BE200037B51300064A05001068046A002C00D1DB
:10BE3000044C0A0000942900FFF770FF3EBDC04685
:10BE400080000020E4000020F8B505000E0014007A
:10BE5000002804D08369002B01D100F0C1F9224BE6
:10BE60009C422DD16C68A369A360A3891B0731D5BF
:10BE70002369002B2ED023682269F7B2981A6369D0
:10BE8000F6B2834205DC2100280000F03BF90028CF
:10BE900026D1A3680130013BA36023685A1C2260AD
:10BEA0001F706369834204D0A389DB071AD50A2E69
:10BEB00018D12100280000F025F9002812D00FE049
:10BEC0000A4B9C4201D1AC68CDE7094B9C42CAD1D8
:10BED000EC68C8E72100280000F00CF80028CAD060
:10BEE000012676423000F8BD1CE300003CE3000070
:10BEF000FCE20000364B70B51D6806000C00002DFA
:10BF000005D0AB69002B02D1280000F069F9314B54
:10BF10009C420FD16C680C23E25E93B219072DD4BA
:10BF2000D90611D409230120336037331343A38189
:10BF3000404270BD284B9C4201D1AC68EBE7274BD7
:10BF40009C42E8D1EC68E6E75B0713D5616B0029FA
:10BF500008D023004433994202D0300000F06AFA3E
:10BF6000002363632422A3899343A3810023636096
:10BF7000236923600823A2891343A3812369002B2B
:10BF80000BD1A0218022A389890092000B4093420B
:10BF900003D02100300000F0E1F90123A289134011
:10BFA00011D00023A36063695B42A3610020236971
:10BFB0008342BED10C23E25E1306BAD5402313435D
:10BFC000A3810138B5E7920700D46369A360EDE768
:10BFD000800000201CE300003CE30000FCE20000C5
:10BFE00010B5062000F090FC012000F0CFFD00000D
:10BFF000F7B58A8905000C00130760D44B68002B45
:10C0000004DC0B6C002B01DC0020FEBDE76A002F76
:10C01000FAD000232E682B6080235B01216A1A402E
:10C0200034D0606DA3895B0706D56368C01A636B63
:10C03000002B01D0236CC01A0200216A00232800C3
:10C04000E76AB847A189431C06D12B681D2B30D85D
:10C050002B4ADA40D3072CD5002363602369236081
:10C06000CB0405D5431C02D12B68002B00D16065A1
:10C07000616B2E600029C7D023004433994202D05F
:10C08000280000F0D7F900206063BEE701232800F4
:10C09000B847431CC6D12B68002BC3D01D2B01D041
:10C0A000162B01D12E60AFE74023A2891343A38151
:10C0B000ABE740230B430120A3814042A5E70F6972
:10C0C000002FA1D00B680F60DB1B019300239207A8
:10C0D00000D14B69A360019B002B00DC94E7019B1E
:10C0E0003A00216A2800A66AB047002803DC4023F2
:10C0F000A2891343DFE7019B3F181B1A0193EAE76C
:10C10000010040200B6970B505000C00002B01D127
:10C11000002070BD002804D08369002B01D100F0FD
:10C120005FF80B4B9C4209D16C680C22A35E002B7C
:10C13000EED021002800FFF75BFFEAE7054B9C42A9
:10C1400001D1AC68F1E7044B9C42EED1EC68ECE71E
:10C150001CE300003CE30000FCE20000002310B5FB
:10C16000040003604360836081814366C281036190
:10C1700043618361190008225C30FFF7FFF9054B2A
:10C1800024626362044BA362044BE362044B2363A7
:10C1900010BDC04649C9000071C90000A9C900000E
:10C1A000D5C9000010B5024900F08CF810BDC0469A
:10C1B00005C1000070B568254A1E55430E002900D0
:10C1C000743100F081F9041E08D000212A000160BA
:10C1D00046600C30A0606832FFF7D0F9200070BDD7
:10C1E000836913B50400002B28D18364C3640365FD
:10C1F000134B144A1B6882620193984201D10123B8
:10C200008361200000F020F86060200000F01CF83E
:10C21000A060200000F018F80022E06004216068AF
:10C22000FFF79CFF01220921A068FFF797FF022278
:10C230001221E068FFF792FF0123A36113BDC046FE
:10C24000C4E20000A5C10000F8B51C4B07001E6841
:10C25000B369002B02D13000FFF7C2FF4836B46843
:10C260007368013B04D53368002B07D03668F6E7C6
:10C270000C22A55E002D0DD06834F2E704213800B1
:10C28000FFF798FF30600028F0D10C2304003B60DA
:10C290002000F8BD20000A4B656625606560A5603A
:10C2A000E36025616561A561082229005C30FFF724
:10C2B00065F96563A563A564E564E9E7C4E2000088
:10C2C0000100FFFFF7B50400070000260191483484
:10C2D000002C01D13000FEBD6368A5680093009B6F
:10C2E000013B009301D52468F2E7AB89012B08D903
:10C2F0000E22AB5E013304D029003800019B984721
:10C3000006436835EBE7EC300068704770B50E0007
:10C310001D000E23C95E96B01400002907DA002321
:10C320002B60B3891B0611D48023DB000FE06A4623
:10C3300000F088FB0028F2DBF022019B1202134080
:10C34000054A9B185A4253412B60EDE740230020D9
:10C35000236016B070BDC04600E0FFFFF7B50226AF
:10C360008B8905000C00334206D02300473323603D
:10C37000236101236361F7BD01AB6A46FFF7C6FF86
:10C3800000990700280000F09FF8002808D10C222F
:10C39000A35E9A05EFD4032293431E43A681E4E7EC
:10C3A0000F4BAB628023A28920601343A381009BC3
:10C3B00020616361019B002B0DD00E23E15E2800FC
:10C3C00000F052FB002806D00322A38993431A00F1
:10C3D00001231343A381A0893843A081CBE7C04642
:10C3E000A5C1000010B5034B0100186800F06CF8FF
:10C3F00010BDC0468000002082B0002900D101A9F4
:10C40000101E06D0002B06D013780B601078431E48
:10C41000984102B0704702204042FAE7C9B2821840
:10C42000904201D10020704703788B42FBD001304D
:10C43000F6E7000070B50500002910D00C1F236836
:10C44000002B00DAE418280000F034FB1D4A1368C2
:10C45000002B05D163601460280000F02CFB70BD38
:10C46000A34209D9216860188342F3D118685B6838
:10C4700041182160EEE713005A68002A01D0A24259
:10C48000F9D919685818A0420BD120680918581812
:10C4900019608242E0D110685268411819605A60F0
:10C4A000DAE7A04202D90C232B60D5E72168601897
:10C4B000824203D1106852684118216062605C605A
:10C4C000CAE7C046241C0020032370B5CD1C9D4341
:10C4D000083506000C2D1ED20C25A9421DD83000AF
:10C4E00000F0E8FA254A14682100002919D1244CEB
:10C4F0002368002B03D1300000F0CAF92060290026
:10C50000300000F0C5F9431C2BD10C233000336000
:10C5100000F0D1FA03E0002DDFDA0C2333600020B5
:10C5200070BD0B685B1B19D40B2B03D90B60CC18A7
:10C53000256003E04B688C420DD11360300000F0A1
:10C54000BAFA200007220B30231D9043C31AE7D00C
:10C550005A42E250E4E763600C00EFE70C004968E0
:10C56000C3E70323C41C9C43A042E1D0211A30003E
:10C5700000F08EF9431CDBD1C7E7C046241C002025
:10C58000281C0020F8B507000D001600002905D171
:10C590001100FFF799FF04002000F8BD002A03D125
:10C5A000FFF748FF3400F7E700F086FA2C00B042AE
:10C5B000F2D231003800FFF787FF041EECD02900CB
:10C5C0003200FEF7BFFF29003800FFF733FFE3E733
:10C5D000F0B58E6885B007000C00039201939E426F
:10C5E0003CD890238A89DB001A4234D0032509699C
:10C5F00023685B1A0293636902985D43EB0F5D1930
:10C60000019B6D1001331B18AB4200D91D0053056F
:10C6100032D529003800FFF757FF061E09D10C2339
:10C620003B6040230120A28940421343A38105B00F
:10C63000F0BD029A2169FEF785FFA389144A1A40CA
:10C6400080231343A381029B2661F618266065614F
:10C65000019EED1AA560019B9E4200D9019E320009
:10C6600003992068FEF777FFA36800209B1BA36057
:10C6700023689E192660DAE72A003800FFF782FF58
:10C68000061EE0D121693800FFF7D4FEC7E7C04697
:10C690007FFBFFFFF0B59FB0029005938B890F00E1
:10C6A00016001B0611D50B69002B0ED14021FFF798
:10C6B0000BFF38603861002805D10C23029A01383D
:10C6C00013601FB0F0BD40237B61002306AC6361A3
:10C6D000203363761033A37635002B78002B01D0FE
:10C6E000252B46D1AB1B04930CD0320039000298A5
:10C6F000FFF76EFF431C00D1AEE06269049B9446D5
:10C70000634463612B78002B00D1A5E00122002354
:10C710005242626002A9543252186E1C2360E360D8
:10C72000A3601370A365317805225448FFF776FEA5
:10C73000751C00281FD12268D30604D5532302A9F3
:10C740005B1820211970130704D5532302A95B1825
:10C750002B21197033782A2B16D0350000210A209E
:10C76000E3682A786E1C303A092A4ED9002918D07D
:10C7700010E00135B1E7414B2268C01A0123834024
:10C78000134323602E00CEE7059B191D1B680591FE
:10C79000002B01DB099304E05B42E36002231343B7
:10C7A00023602B782E2B0AD16B782A2B35D1059B51
:10C7B00002351A1D1B680592002B2BDB0793304EA8
:10C7C000297803223000FFF729FE002806D04023F5
:10C7D000801B834022680135134323602978062299
:10C7E00028486E1C2176FFF719FE00283CD0264B06
:10C7F000002B25D10722059B07339343083305936C
:10C800006369039A9B18636166E7434301219B18A0
:10C810003500A6E701235B42D0E700230A201A0077
:10C820000135636029786E1C3039092903D9002B42
:10C83000C5D00792C3E74243012352183500F1E700
:10C8400005AB00933A00114B2100029800E000BFB5
:10C850000390039B0133D3D1BB890B985B0600D4B3
:10C860002FE7012040422CE705AB00933A00074B2D
:10C8700021000298FFF736F8EAE7C046C8E2000058
:10C88000CEE20000D2E2000000000000D1C50000AE
:10C89000002370B5064C05000800236000F060F925
:10C8A000431C03D12368002B00D02B6070BDC04611
:10C8B000B82F002070B504000D001F2904D91623DD
:10C8C00003600120404270BD436C002B04D08A00FD
:10C8D0009B181A68002A08D1200000F031F82A00BD
:10C8E0000100200000F01AF8EDE70020012AEAD04C
:10C8F000511C03D1162301302360E4E700242800F3
:10C900001C6090472000DEE710B5034B010018685B
:10C91000FFF7D0FF10BDC04680000020002370B597
:10C92000064C050008001100236000F001F9431CCB
:10C9300003D12368002B00D02B6070BDB82F0020DE
:10C9400010B500F0E5F810BD70B50C000E25495F7C
:10C9500000F0BAF8002803DB636D1B18636570BD37
:10C96000A389024A1340A381F9E7C046FFEFFFFF06
:10C97000F8B51F008B8905000C001600DB0505D5F6
:10C980000E23C95E0022022300F080F8A389054A25
:10C9900028001340A38132000E23E15E3B0000F02B
:10C9A0002BF8F8BDFFEFFFFF70B50C000E25495FB7
:10C9B00000F06CF8A389421C03D1054A1340A381FF
:10C9C00070BD802252011343A3816065F8E7C04621
:10C9D000FFEFFFFF10B50E23C95E00F021F810BD78
:10C9E0000B1E04D0FF2A04D98A2303608B3B180056
:10C9F00070470A700123FAE770B5050008001100BE
:10CA00000022064C22601A0000F0B8F8431C03D143
:10CA10002368002B00D02B6070BDC046B82F0020CB
:10CA2000002370B5064C05000800236000F060F894
:10CA3000431C03D12368002B00D02B6070BDC0467F
:10CA4000B82F0020002370B5064C05000800110027
:10CA5000236000F055F8431C03D12368002B00D05D
:10CA60002B6070BDB82F0020002370B5064C050068
:10CA70000800236000F054F8431C03D12368002B06
:10CA800000D02B6070BDC046B82F002070B50500E7
:10CA9000080011000022064C22601A0000F050F835
:10CAA000431C03D12368002B00D02B6070BDC0460F
:10CAB000B82F0020704770470B1F1B68181F002BF2
:10CAC00001DA0B58C018704770B505000800110056
:10CAD0000022064C22601A0000F03AF8431C03D1F1
:10CAE0002368002B00D02B6070BDC046B82F0020FB
:10CAF00058220120014B40421A607047B82F002095
:10CB000058220120014B40421A607047B82F002084
:10CB100058220120014B40421A607047B82F002074
:10CB20005822024B00201A607047C046B82F0020E0
:10CB300058220120014B40421A607047B82F002054
:10CB400058220120014B40421A607047B82F002044
:10CB500058220120014B40421A607047B82F002034
:10CB6000044A1368002B00D1034B181810601800FA
:10CB70007047C0462C1C0020C02F002058220120E6
:10CB8000014B40421A607047B82F0020FEE7C046B4
:10CB9000F8B5C046F8BC08BC9E467047F8B5C0461C
:10CBA000F8BC08BC9E4670476461746100000000D8
:10CBB0002CCC0000EF01000035CC0000E3020000A7
:10CBC0003DCC00000909000044CC0000190A000017
:10CBD00049CC00003105000054CC00005303000094
:10CBE00059CC0000710C000065CC00001F02000051
:10CBF0006FCC0000110800007DCC0000BD060000D5
:10CC00008ACC0000F104000072616E646F6D0061F7
:10CC10006C6C006C6173740066616C736500747297
:10CC2000756500252E3135732E2E2E006D616B65D6
:10CC30004C697374006164644C6173740064656C66
:10CC4000657465006A6F696E00636F707946726F14
:10CC50006D546F0066696E64006A6F696E5374721A
:10CC6000696E677300756E69636F64654174007502
:10CC70006E69636F6465537472696E67006E657781
:10CC800042797465417272617900667265654D65BD
:10CC90006D6F727900000000FDCC0000D91000001B
:10CCA00002CD0000F71000003DCC0000FB1000009A
:10CCB00008CD0000DD10000012CD0000FF100000C4
:10CCC0001BCD00000311000025CD0000071100005E
:10CCD00030CD00000B1100003CCD0000E110000041
:10CCE00045CD0000EF1000004FCD0000E510000022
:10CCF0005ACD0000F310000066696C65006F706526
:10CD00006E00636C6F736500656E644F6646696C98
:10CD10006500726561644C696E65007265616442AC
:10CD20007974657300617070656E644C696E65003E
:10CD3000617070656E6442797465730066696C65D4
:10CD400053697A650073746172744C697374006E10
:10CD5000657874496E4C6973740073797374656D8A
:10CD6000496E666F00000000381300004813000091
:10CD700062130000E0130000181400004E140000BD
:10CD800086140000AC140000E81400002A1500000E
:10CD900080150000C4150000301600007816000051
:10CDA0009E160000D61600001C1700004217000057
:10CDB000701700009E170000D417000058180000DC
:10CDC0002019000096190000061A0000521A0000EF
:10CDD000721A0000941A0000461B00008C1B000011
:10CDE000041C0000321C0000621C0000981C0000A3
:10CDF000001D0000801D0000C61D00000E1E00006A
:10CE0000841E0000FA1E0000421F0000881F000060
:10CE1000BE1F0000042000004A20000092200000F5
:10CE2000E62000004421000082210000EC210000E7
:10CE3000222200006A220000B2220000FA22000032
:10CE4000342300007C230000C423000030250000B0
:10CE500070170000381300002C2400003813000065
:10CE6000622400008E240000C4240000F02400008E
:10CE70003813000038130000381300003813000086
:10CE8000AA250000EC2500003226000082260000C2
:10CE9000AE260000FE2600002427000052270000D6
:10CEA00076270000381300007E270000AE27000020
:10CEB000DE270000142800003E280000742800002F
:10CEC0009E280000C6280000EE280000542900001B
:10CED00084290000AE290000D8290000082A00009B
:10CEE000322A000038130000381300003813000005
:10CEF0003813000038130000622A00008E2A000058
:10CF0000BA2A0000E62A0000122B0000482B00007D
:10CF10007E2B0000B42B0000EA2B0000162C000032
:10CF2000422C0000782C0000381300003813000059
:10CF300038130000381300003813000038130000C5
:10CF400038130000381300003813000038130000B5
:10CF500038130000381300003813000038130000A5
:10CF6000A42C0000DA2C00005B2564206974656D38
:10CF7000206C6973745D0028256420627974657380
:10CF80002900286F626A65637420747970653A209D
:10CF900025642900537461636B20756E6465726645
:10CFA0006C6F7700626F6F6C65616E006E756D629D
:10CFB000657200737472696E67006C6973740062E5
:10CFC00079746520617272617900000007000000C9
:10CFD0000300000026D00000FD2D00002ED0000030
:10CFE000AD2E000037D00000572F000040D00000C9
:10CFF000012E000049D000005B2F000051D000003E
:10D00000452F0000000000000100000002000000A9
:10D0100003000000040000000A0000006D69637254
:10D020006F3A62697400686173546F6E6500706C6A
:10D030006179546F6E6500686173536572766F0035
:10D04000736574536572766F00646163496E6974C9
:10D0500000646163577269746500474320746F6FA1
:10D060006B2025642075736563733B20667265656C
:10D0700020256420776F726473003C496E74656785
:10D0800065723E003C4C6973743E003C4F626A65B9
:10D0900063743E003C4279746541727261793E006E
:10D0A0000D0A564D2050616E69633A2025730D0AB2
:10D0B000006D697363000000EDD00000193C0000B2
:10D0C000F6D00000A93B0000FAD00000FD3A0000B5
:10D0D00002D10000A33A00000CD10000393A000050
:10D0E00018D100003B3900006E756C6C00686578E3
:10D0F000546F496E740073696E006A736F6E476592
:10D1000074006A736F6E436F756E74006A736F6E2E
:10D1100056616C75654174006A736F6E4B65794139
:10D120007400000080D10000853C000088D1000020
:10D13000893C000092D10000A73C00009BD1000078
:10D14000B13C0000A6D10000BB3C0000B2D1000001
:10D15000C53C0000C7D10000CF3C0000DCD100007E
:10D16000D93C0000E8D10000E33C0000F8D1000009
:10D17000933C000004D200009D3C00006E657400EA
:10D1800068617357694669007374617274576946C0
:10D19000690073746F7057694669007769666953EF
:10D1A0007461747573006D7949504164647265737C
:10D1B0007300687474705365727665724765745253
:10D1C00065717565737400726573706F6E64546F0A
:10D1D0004874747052657175657374006874747006
:10D1E000436F6E6E65637400687474704973436F47
:10D1F0006E6E6563746564006874747052657175F1
:10D200006573740068747470526573706F6E7365C3
:10D21000001A1B1C03040607090A1718190000004E
:10D22000000008080800080A4A4000000A5FEA5F98
:10D23000EA0ED92ED36E19324489330C924C924D9A
:10D240000808000000048808080408048484880092
:10D250000A448A4000048EC4800000000488000054
:10D260000EC000000000080001224488100C9252F9
:10D27000524C048C84848E1C824C901E1EC244929C
:10D280004C06CA525FE21FF01EC13E02448ED12EF0
:10D290001FE24488100ED12ED12E0ED12EC488004C
:10D2A0000800080000048004880244880482000EFC
:10D2B000C00EC008048244880ED126C0040ED135A9
:10D2C000B36C0C925ED2521C925C925C0ED0101029
:10D2D0000E1C9252525C1ED01C901E1ED01C901030
:10D2E0000ED013712E12525ED2521C8808081C1FD9
:10D2F000E242524C1254981492101010101E113B1E
:10D3000075B131113935B3710C9252524C1C925C8B
:10D3100090100C92524C861C925C92510ED00C8252
:10D320005C1FE4848484125252524C1131312A44DD
:10D33000113135BB7112524C9252112A4484841E11
:10D34000C488101E0EC808080E10080482410EC2C0
:10D3500042424E048A400000000000001F08048082
:10D360000000000ED2524F10101C925C000ED01024
:10D370000E02424ED24E0C925C900E06C81C8808DB
:10D380000ED24EC24C10101C92520800080808021F
:10D390004002424C10149814920808080806001B1A
:10D3A00075B131001C925252000C92524C001C92EA
:10D3B0005C90000ED24EC2000ED010100006C804C1
:10D3C0009808080EC807001252524F0011312A4423
:10D3D00000113135BB00124C8C9200112A44980088
:10D3E0001EC4881E06C48C8486080808080818080D
:10D3F0000C881800000C8360000000000100000091
:10D40000020000000300000004000000050000000E
:10D4100006000000070000000800000009000000EE
:10D420000A0000000B0000000C0000000D000000CE
:10D430000E0000000F0000001000000012000000AD
:10D440001400000016000000180000001A00000080
:10D450001C0000001E00000020000000230000004F
:10D4600026000000290000002C0000002F00000012
:10D4700032000000360000003A0000003E000000CC
:10D4800042000000460000004B0000005000000079
:10D49000550000005A000000610000006800000014
:10D4A0006F000000760000007D0000008400000096
:10D4B0008B0000009200000099000000A000000016
:10D4C000A7000000AE000000B5000000BC00000096
:10D4D000C3000000CA000000D1000000D800000016
:10D4E000DF000000E6000000ED000000F400000096
:10D4F000FB000000FF00000048D50000053D0000D3
:10D5000053D50000994200005DD50000C13E0000E7
:10D510006AD500000941000071D5000059410000A2
:10D520007AD50000A941000086D50000A140000086
:10D5300097D50000313F0000A4D500003140000025
:10D54000646973706C6179006C696768744C6576A6
:10D55000656C006D62446973706C6179006D624442
:10D560006973706C61794F6666006D62506C6F74A0
:10D57000006D62556E706C6F74006D6244726177FD
:10D580005368617065006D625368617065466F72C3
:10D590004C6574746572006E656F506978656C5384
:10D5A000656E64006E656F506978656C5365745084
:10D5B000696E004E6F7420656E6F75676820726FBC
:10D5C0006F6D206576656E20616674657220636F8D
:10D5D0006D70616374696F6E00436F6D7061637429
:10D5E000656420466C61736820636F6465207374A2
:10D5F0006F72650A2564206279746573207573659E
:10D600006420282564252529206F66202564004292
:10D610006164207265636F726420666F756E64204A
:10D62000647572696E6720696E697469616C697A84
:10D630006174696F6E0025642025642025642028AC
:10D64000256420776F7264732900256420726563F6
:10D650006F7264732C20256420776F7264732C20A2
:10D660006D617849442025642C20636F6D7061637F
:10D6700074696F6E206379636C6573202564005252
:10D680006573746F726564202564207363726970BA
:10D690007473005374617274656400726164696FBD
:10D6A0000000000034D70000694C000041D70000A2
:10D6B000054F000051D70000854E00005FD70000E5
:10D6C000995000006AD70000914C00007AD7000002
:10D6D000194D00008ED70000014D00009DD70000BD
:10D6E0007B520000A9D70000F9510000B2D700001A
:10D6F0009D510000BDD70000E5500000C8D70000D4
:10D7000021510000D1D7000055510000DAD70000A8
:10D71000A14C0000E9D70000814C0000F2D70000C6
:10D72000B14C00006E6F6E65006F746865720070BA
:10D730006169720064697361626C65526164696FEA
:10D74000006D6573736167655265636569766564CD
:10D75000007061636B65745265636569766500701E
:10D7600061636B657453656E6400726563656976A9
:10D770006564496E74656765720072656365697694
:10D7800065644D6573736167655479706500726592
:10D79000636569766564537472696E670073656E5C
:10D7A00064496E74656765720073656E6450616983
:10D7B000720073656E64537472696E67007365748A
:10D7C0004368616E6E656C0073657447726F757047
:10D7D00000736574506F776572007369676E616C72
:10D7E000537472656E677468006465766963654931
:10D7F00044006C6173744D657373616765494400DF
:10D80000556E6B6E6F776E207072696D6974697694
:10D8100065205B25733A25735D0000000000000061
:10D82000963007772C610EEEBA51099919C46D072D
:10D830008FF46A7035A563E9A395649E3288DB0E88
:10D84000A4B8DC791EE9D5E088D9D2972B4CB6096B
:10D85000BD7CB17E072DB8E7911DBF906410B71D48
:10D86000F220B06A4871B9F3DE41BE847DD4DA1A81
:10D87000EBE4DD6D51B5D4F4C785D38356986C13B2
:10D88000C0A86B647AF962FDECC9658A4F5C01142B
:10D89000D96C0663633D0FFAF50D088DC8206E3B09
:10D8A0005E10694CE44160D5727167A2D1E4033C1B
:10D8B00047D4044BFD850DD26BB50AA5FAA8B53542
:10D8C0006C98B242D6C9BBDB40F9BCACE36CD83231
:10D8D000755CDF45CF0DD6DC593DD1ABAC30D926D8
:10D8E0003A00DE518051D7C81661D0BFB5F4B421DB
:10D8F00023C4B3569995BACF0FA5BDB89EB80228D8
:10D900000888055FB2D90CC624E90BB1877C6F2F5C
:10D91000114C6858AB1D61C13D2D66B69041DC7657
:10D920000671DB01BC20D2982A10D5EF8985B17130
:10D930001FB5B606A5E4BF9F33D4B8E8A2C90778DF
:10D9400034F9000F8EA8099618980EE1BB0D6A7F76
:10D950002D3D6D08976C6491015C63E6F4516B6B2F
:10D9600062616C1CD83065854E0062F2ED95066CE4
:10D970007BA5011BC1F4088257C40FF5C6D9B06559
:10D9800050E9B712EAB8BE8B7C88B9FCDF1DDD62B6
:10D99000492DDA15F37CD38C654CD4FB5861B24D1C
:10D9A000CE51B53A7400BCA3E230BBD441A5DF4AE6
:10D9B000D795D83D6DC4D1A4FBF4D6D36AE96943A9
:10D9C000FCD96E34468867ADD0B860DA732D044454
:10D9D000E51D03335F4C0AAAC97C0DDD3C7105507F
:10D9E000AA41022710100BBE86200CC925B5685726
:10D9F000B3856F2009D466B99FE461CE0EF9DE5E6F
:10DA000098C9D9292298D0B0B4A8D7C7173DB3591F
:10DA1000810DB42E3B5CBDB7AD6CBAC02083B8EDB0
:10DA2000B6B3BF9A0CE2B6039AD2B1743947D5EABD
:10DA3000AF77D29D1526DB048316DC73120B63E3EC
:10DA4000843B64943E6A6D0DA85A6A7A0BCF0EE44B
:10DA50009DFF099327AE000AB19E077D44930FF006
:10DA6000D2A3088768F2011EFEC206695D5762F7FD
:10DA7000CB67658071366C19E7066B6E761BD4FE3A
:10DA8000E02BD3895A7ADA10CC4ADD676FDFB9F917
:10DA9000F9EFBE8E43BEB717D58EB060E8A3D6D6D9
:10DAA0007E93D1A1C4C2D83852F2DF4FF167BBD107
:10DAB0006757BCA6DD06B53F4B36B248DA2B0DD80A
:10DAC0004C1B0AAFF64A0336607A0441C3EF60DFAD
:10DAD00055DF67A8EF8E6E3179BE69468CB361CB96
:10DAE0001A8366BCA0D26F2536E2685295770CCCBB
:10DAF00003470BBBB91602222F260555BE3BBAC5FC
:10DB0000280BBDB2925AB42B046AB35CA7FFD7C2EC
:10DB100031CFD0B58B9ED92C1DAEDE5BB0C2649BDD
:10DB200026F263EC9CA36A750A936D02A906099C10
:10DB30003F360EEB8567077213570005824ABF9583
:10DB4000147AB8E2AE2BB17B381BB60C9B8ED29206
:10DB50000DBED5E5B7EFDC7C21DFDB0BD4D2D3865D
:10DB600042E2D4F1F8B3DD686E83DA1FCD16BE81D0
:10DB70005B26B9F6E177B06F7747B718E65A0888A1
:10DB8000706A0FFFCA3B06665C0B0111FF9E658F32
:10DB900069AE62F8D3FF6B6145CF6C1678E20AA0DC
:10DBA000EED20DD75483044EC2B30339612667A762
:10DBB000F71660D04D476949DB776E3E4A6AD1AEB1
:10DBC000DC5AD6D9660BDF40F03BD83753AEBCA940
:10DBD000C59EBBDE7FCFB247E9FFB5301CF2BDBDAD
:10DBE0008AC2BACA3093B353A6A3B4240536D0BAB6
:10DBF0009306D7CD2957DE54BF67D9232E7A66B353
:10DC0000B84A61C4021B685D942B6F2A37BE0BB4FF
:10DC1000A18E0CC31BDF055A8DEF022D416C6C20C9
:10DC20007461736B732073746F7070656400763009
:10DC30003838002025732025730052657374617293
:10DC400074696E67004D656D6F727920636C6561F4
:10DC5000726564004E6F2066726565207461736B37
:10DC600020656E747269657300000000B4DC00000A
:10DC700021660000C1DC00005D620000CDDC000018
:10DC8000F1650000D3DC000001660000D9DC000073
:10DC900011660000DFDC000091620000E9DC00009A
:10DCA0007D660000F1DC0000D163000073656E73D7
:10DCB0006F727300616363656C65726174696F6E26
:10DCC0000074656D70657261747572650074696C5D
:10DCD00074580074696C74590074696C745A0074D7
:10DCE0006F7563685265616400693263526561648F
:10DCF00000693263577269746500000070DD0000CE
:10DD0000096700007EDD00000D67000087DD000070
:10DD10001967000091DD00001D6700009ADD00001A
:10DD2000216700009FDD000025670000A4DD0000E2
:10DD300029670000B0DD00002D670000B7DD00009E
:10DD400031670000C0DD000035670000C5DD000060
:10DD500039670000D0DD00003D670000DADD00001B
:10DD600011670000E4DD00001567000074667400B0
:10DD7000656E61626C65446973706C61790067659A
:10DD80007457696474680067657448656967687486
:10DD900000736574506978656C006C696E6500721B
:10DDA00065637400726F756E6465645265637400B8
:10DDB000636972636C6500747269616E676C65009B
:10DDC0007465787400746674546F75636865640074
:10DDD000746674546F7563685800746674546F7514
:10DDE00063685900746674546F7563685072657324
:10DDF0007375726500766172730000001CDE0000AE
:10DE0000CD6B000026DE0000AD6B00002FDE0000B1
:10DE1000896B00003BDE0000156B000076617245E7
:10DE20007869737473007661724E616D6564007316
:10DE300065745661724E616D6564007661724E6103
:10DE40006D65466F72496E6465780057656C636FE7
:10DE50006D6520746F204D6963726F426C6F636BE8
:10DE6000732100705F73706920213D204E554C4C2A
:10DE7000002F686F6D652F6769742F2E706C617449
:10DE8000666F726D696F2F7061636B616765732F69
:10DE90006672616D65776F726B2D61726475696E04
:10DEA0006F6E6F726469636E7266352F6C69627231
:10DEB00061726965732F5350492F5350492E637017
:10DEC0007000535049436C6173733A3A535049435D
:10DED0006C617373284E52465F5350495F5479709A
:10DEE000652A2C2075696E74385F742C2075696EF4
:10DEF00074385F742C2075696E74385F7429000063
:10DF00000000000000000000D96D0000956D0000C9
:10DF1000BB6D0000C56D0000CF6D0000B96D000045
:10DF200003000000020000000100000004000000E7
:10DF300005000000110000000C0000000B000000B4
:10DF4000120000000A000000060000001A00000095
:10DF5000140000001700000016000000150000006B
:10DF600010000000FFFFFFFFFFFFFFFF00000000A9
:10DF70001E0000001900000018000000070000004B
:10DF800008000000090000000D0000000E00000065
:10DF90000F0000001C0000001B0000001D0000001E
:10DFA0001300000000000000000000008972000063
:10DFB000B9790000097300001D730000137300009D
:10DFC000857200007972000029730000A5720000BC
:10DFD00075720000000000000000000000003043E7
:10DFE00000000000000030C3737172740000000074
:10DFF000FB21F93FFB2109407CD91240FB2119404C
:10E000007A6A1F407CD92240BBFD2540FB21294074
:10E010003A462C407A6A2F405C4731407CD93240E6
:10E020009C6B3440BBFD3540DB8F3740FB213940D2
:10E030001BB43A403A463C405AD83D407A6A3F4089
:10E040004C7E40405C4741406C1042407CD942408D
:10E050008CA243409C6B4440AC344540BBFD4540E2
:10E06000CBC64640DB8F4740EB584840FB21494038
:10E0700083F9A200444E6E00FC291500D1572700F9
:10E08000DD34F50062DBC0003C999500419043000F
:10E090006351FE00BBDEAB00B761C5003A6E2400E1
:10E0A000D24D42004906E00009EA2E001C92D10040
:10E0B000EB1DFE0029B11C00E83EA700F5358200EB
:10E0C00044BB2E009CE98400B4267000417E5F00B2
:10E0D000D6913900538339009CF439008B5F84005A
:10E0E00028F9BD00F81F3B00DEFF97000F980500E0
:10E0F000112FEF000A5A8B006D1F6D00CF7E360086
:10E1000009CB2700464FB7009E663F002DEA5F000F
:10E11000BA277500E5EBC7003D7BF100F739070032
:10E1200092528A00FB6BEA001FB15F00085D8D0010
:10E13000300356007BFC4600F0AB6B0020BCCF00E8
:10E1400036F49A00E3A91D005E619100081BE60009
:10E1500085996500A0145F008D40680080D8FF009D
:10E1600027734D0006063100CA561500C9A8730072
:10E170007BE260006B8CC00000000040FB21F93F97
:10E18000000000002D44743E000000809846F83CDA
:10E190000000006051CC783B00000080831BF03908
:10E1A0000000004020257A38000000802282E336FB
:10E1B000000000001DF369350200000003000000AC
:10E1C0000400000006000000B09600005A9600000F
:10E1D0005A96000088970000569600005696000058
:10E1E0007E97000088970000569600007E970000FA
:10E1F00056960000889700008C9700008C970000CE
:10E200008C970000949700008CA10000FE9F0000F6
:10E2100042A00000A69F000042A0000032A1000022
:10E2200042A00000A69F0000FE9F0000FE9F00008D
:10E2300032A10000A69F00009E9F00009E9F00004C
:10E240009E9F000040A10000B4A80000B6A70000F7
:10E25000B6A70000D4AA0000B0A70000B0A7000035
:10E26000BCAA0000D4AA0000B0A70000BCAA00000D
:10E27000B0A70000D4AA0000CAAA0000CAAA0000E1
:10E28000CAAA0000D8AA00002C2066756E637469C3
:10E290006F6E3A2000617373657274696F6E20222D
:10E2A000257322206661696C65643A2066696C6535
:10E2B00020222573222C206C696E6520256425732D
:10E2C00025730A0084000020232D302B2000686C69
:10E2D0004C00656667454647003031323334353689
:10E2E00037383941424344454600303132333435C2
:10E2F00036373839616263646566000000000000EB
:10E30000000000000000000000000000000000000D
:10E3100000000000000000000000000000000000FD
:10E3200000000000000000000000000000000000ED
:10E3300000000000000000000000000000000000DD
:10E3400000000000000000000000000000000000CD
:10E350000000000000000000000000004300504FDB
:10E360005349580000202020202020202020282849
:10E370002828282020202020202020202020202085
:10E3800020202020208810101010101010101010C5
:10E3900010101010100404040404040404040410F5
:10E3A0001010101010104141414141410101010183
:10E3B000010101010101010101010101010101014D
:10E3C0001010101010104242424242420202020259
:10E3D000020202020202020202020202020202021D
:10E3E00010101010200000000000000000000000CD
:10E3F000000000000000000000000000000000001D
:10E40000000000000000000000000000000000000C
:10E4100000000000000000000000000000000000FC
:10E4200000000000000000000000000000000000EC
:10E4300000000000000000000000000000000000DC
:10E4400000000000000000000000000000000000CC
:10E4500000000000000000000000000000000000BC
:0CE46000000000000000000000000000B0
:08E46C009C1CFF7F0100000071
:10E47400FFFFFFFF4006000001000000E803DC0589
:10E48400DC05DC05DC050000FFFFFFFFFFFFFFFFED
:10E494001800000019FCFFFFFFFFFFFFFF00000052
:10E4A4000200000003000000FFFFFFFF0000000067
:10E4B400010000000000020001000000FFFFFFFF58
:10E4C4000000000002000000000004000200000040
:10E4D400FFFFFFFF00000000030000000000080031
:10E4E400030000000A000000080000000100000012
:10E4F40084000020000000001CE300003CE3000056
:10E50400FCE2000000000000000000000000000029
:10E5140000000000000000000000000000000000F7
:10E5240000000000000000000000000000000000E7
:10E5340000000000000000000000000000000000D7
:10E5440000000000000000000000000000000000C7
:10E554000000000043000000000000000000000074
:10E5640000000000000000000000000000000000A7
:10E574000000000043000000000000000000000054
:10E584000000000000000000000000000000000087
:10E594000000000043000000000000000000000034
:10E5A4000000000000000000000000000000000067
:10E5B4000000000043000000000000000000000014
:10E5C4000000000000000000000000000000000047
:10E5D40000000000430000000000000000000000F4
:10E5E4000000000000000000000000000000000027
:10E5F40000000000430000000000000000000000D4
:10E604000000000000000000000000000000000006
:10E6140000000000430000000000000000000000B3
:10E6240000000000000000000000000000000000E6
:10E6340000000000E1C90000F9C300000000000070
:10E6440064E300002ACC0000B0D00000B0D0000089
:10E65400B0D00000B0D00000B0D00000B0D00000B6
:10E66400B0D00000B0D00000B0D00000FFFFFFFF2A
:10E67400FFFFFFFFFFFFFFFFFFFF0000010041530B
:10E6840043494900000000000000000000000000B1
:10E6940000000000000000000000000000004153E2
:10E6A4004349490000000000000000000000000091
:10E6B4000000000000000000000000000000000056
:10E6C400E9000000656D0000AD700000D575000024
:04E6D400C100000081
:04000003000071493F
:00000001FF
